:100000000C9416250C9445250C9445250C944525F7
:100010000C9445250C9445250C9445250C944525B8
:100020000C9445250C9445250C9445250C944525A8
:100030000C9445250C949D450C9445250C94452520
:100040000C9445250C9445250C9445250C94452588
:100050000C9445250C9445250C9445250C94452578
:100060000C9445250C94CCD10C9445250C94F8D1D6
:100070000C9445250C94F99B0C9445250C9445252E
:100080000C9445250C9445250C9445250C94452548
:100090000C9445250C9445250C9445250C94452538
:1000A0000C9445250C9445250C9445250C94452528
:1000B0000C9445250C9445250C9445250C94FC4442
:1000C0000C9445250C9445250C9445250C94452508
:1000D0000C9445250C9445250C9445250C944525F8
:1000E0000C944525F3289D299D299A299A299D2913
:1000F0009D299D299D29392948299D299D29A02986
:10010000A029A029A029A029A029A0293229A02915
:10011000A029A029A029A029A029A0295129863FEA
:10012000AE3FB33F903FB83F05400540903FD63FBC
:100130000540DB3FE33FE83FED3FC23FC73FCC3FD9
:10014000903FD13F05408B3FBD3FF23FF73FFB3F24
:1001500005400540FF3F52885988628866885E885E
:1001600056886B887B887088B2A5B6A5BAA5BEA54F
:10017000C2A5DFA5C6A5DFA5DAA522A947A924A99E
:1001800027A92AA92FA934A939A940A976AE8AAEF0
:100190003DAF05AF30AFF8AEE4AED0AE4AAFC7AEBC
:1001A000B5AEB8AEBBAEBEAEC1AEC4AECDAECAAEDD
:1001B000F8B2FBB2FEB201B304B363B317B31AB320
:1001C00063B33CB344B363B35FB365B9A6B8C5B812
:1001D000D4B802B920B933B97FBA87BA8ABA94BA07
:1001E000A2BAEFBAA9BA03BB06BBE6BAD4BAD7BA69
:1001F000DABADDBAE0BAE3BAECBAE9BA29BB41BB74
:1002000044BB5FBB88BB93BBA5BB9DBBA0BB76BCFF
:1002100079BC7CBC82BC7FBC85BC88BC9BBCA5BCBB
:10022000ACBCD1BCD4BCDBBCE0BCDDBCE6BCE9BC36
:10023000F7BC05BD0FBD8FBD9ABDE0BDA5BDD5BD49
:10024000CABDABBDEEBD0FBED7C47DC587C58DC5CC
:1002500090C5A1C5B5C5E1C5E4C552C6FCC51CC65F
:100260003FC6494E56414C494420544F4F4C3A20CA
:10027000202020202020492072656365697665640E
:100280002061204C656674202020546F6F6C2063C1
:100290006F6D6D616E642C206275742049206F6EE5
:1002A0006C792068617665206F6E6520546F6F6C85
:1002B0002E2000494E56414C494420434F4D4D415C
:1002C0004E443A2020202049207265636569766596
:1002D00064206120636F6D6D616E64666F72206172
:1002E0002068656174656420706C6174652C20629F
:1002F0007574204920646F6E2774206861766520CC
:100300006F6E6500492074696D6564206F75742097
:100310007768696C65202020617474656D707469FC
:100320006E6720746F206865617420206D79206588
:10033000787472756465722E202020202020202081
:1003400000492074696D6564206F75742077686951
:100350006C65202020617474656D7074696E67200F
:10036000746F206865617420206D7920706C6174F1
:10037000666F726D2E2020202020202020005468DF
:100380006973206275696C6420697320666F7220DE
:100390002020616E6F7468657220626F742E205326
:1003A00065653A2020206D616B6572626F742E6303
:1003B0006F6D2F68656C7020202000546869732071
:1003C0006973206E6F7420746865207833672076B7
:1003D000657273696F6E204920776F726B2062655A
:1003E000737420776974682E20466F722068656C7C
:1003F00070207365653A206D616B6572626F742E53
:10040000636F6D2F68656C702020200052657374D7
:10041000617274696E6720746865204275696C64E6
:1004200000507265706172696E6720666F7220732A
:100430006C6565703A49276D20636F6F6C696E67F4
:10044000206D7920202020202068656174657273FA
:1004500020616E6420676F696E6720746F6D79200C
:100460007761697420706F736974696F6E2E2020D4
:100470002000507265706172696E6720666F72202D
:10048000736C6565703A49276D20636F6D706C659C
:1004900074696E6720616E79202071756575656479
:1004A000206D6F7665732E20202020202020004DA7
:1004B0007920686561746572732074696D65642064
:1004C0006F75744920616D206E6F7720696E2053BF
:1004D0006C65657020202028436F6C642050617526
:1004E0007365292E2020202020202020202020205D
:1004F000202020202020202020202020202020001C
:100500004368616E67696E672046696C616D656EF0
:10051000743A202049276D20676F696E6720746FD9
:10052000206D792077616974706F736974696F6E7B
:100530002E20202020202020202020200043686121
:100540006E67696E672046696C616D656E743A20EE
:100550002049276D20636F6D706C6574696E67202C
:10056000616E792020717565756564206D6F7665A3
:10057000732E202020202020200049207361772026
:100580006120676C6974636820696E206D795344DB
:1005900020636172642E2049662074686973206943
:1005A0007320746865206669727374206572726F57
:1005B000722C2074727974686973206D6F64656C35
:1005C00020616761696E2E202020005468652052EA
:1005D00065706C6963617430720049276D204361F6
:1005E0006E63656C6C696E672E2020202020506C35
:1005F0006561736520576169742E202020202020BA
:1006000020200048656174696E67204661696C75D9
:100610007265202335212049276D20726561646948
:100620006E67206F7574206F66202072616E67653B
:100630002074656D7065726174757265732E2043E8
:100640006865636B206D7920636F6E6E6563746996
:100650006F6E730048656174696E67204661696CEE
:1006600075726520233421204D792074656D706585
:100670007261747572652072656164736172652060
:100680006661696C696E672120506C6561736520D5
:10069000436865636B206D7920636F6E6E6563746C
:1006A000696F6E730048656174696E6720466169A1
:1006B0006C75726520233321204D79206578747222
:1006C000756465727320617265202020206C6F73E1
:1006D000696E672074656D70657261747572652EE0
:1006E00020436865636B206D7920636F6E6E656370
:1006F00074696F6E730048656174696E6720466146
:10070000696C75726520233221204D7920657874DB
:1007100072756465727320617265206E6F746865AE
:100720006174696E672070726F7065726C792E20CB
:100730002020436865636B206D7920636F6E6E6562
:100740006374696F6E730048656174696E672046F3
:1007500061696C7572652023312120536F6674774F
:100760006172652054656D70204C696D697420520A
:100770006561636865642120506C65617365202044
:1007800020202053687574646F776E206F7220523A
:1007900065737461727420004865617465727320BA
:1007A00073687574646F776E2020202064756520EF
:1007B000746F20696E616374697669747920202092
:1007C0000020009302690000006900EE016900004A
:1007D0000069002601B80100000000B807550000BC
:1007E000005500B909AB000000AB007D06550000C4
:1007F000005500C805550000005500B807AB0000C3
:1008000000AB00C805550000005500DD0455000090
:10081000005500C805550000005500B807550000F8
:100820000055007D065601000000003F0355000002
:10083000005500FA0C5500000055003F035500001C
:10084000005500B9095500000055003F0355000050
:100850000055002D095500000055003F03550000CC
:10086000005500EA0A5500000055003F03550000FE
:10087000005500B909AB0000000000C805C8000021
:10088000001400C805C80000001400C805C8000016
:10089000001400DD04B004000014007505C8000059
:1008A0000014007505C800000014007505C800009C
:1008B0000014009704B00400000000C00DC8000040
:1008C000001400C00DC80000001400910E9001003B
:1008D0000014005A10900100001400C00D20030005
:1008E00000000020065500000055002D08550000AE
:1008F0000055004D0A550000005500400CAB0000AB
:1009000000AB002D095500000055002D08550000D2
:100910000055004D0AAB000000550000000001C06A
:100920000D5500000055002D08560100000000C0C4
:100930000D20015311BC005B12B1010000000053F7
:100940004420436172642052656D6F766564202097
:1009500020200024F4D43050C38E20C2A24017823D
:100960008B7011127A910D816CD90AA861E108C7C8
:10097000586607615143061E4B5D05C145A7041A21
:10098000411104093D9803713931034036DB02659A
:10099000339102D4305402802E1D02632CEE017577
:1009A0002AC501B028A001102781018F2564012BE1
:1009B000244B01E0223401AC211F018D200D018068
:1009C0001FFC00841EED00971DDF00B81CD200E65E
:1009D0001BC600201BBC00641AB200B219A8000A92
:1009E00019A0006A189900D117910040178B00B523
:1009F00016840031167E00B31579003A157300C7CE
:100A0000146F0058146A00EE136600881363002503
:100A1000135E00C7125B006C12570015125400C120
:100A200011510070114F0021114B00D61049008D5B
:100A30001047004610440002104200C00F400080E2
:100A40000F3E00420F3C00060F3B00CB0E380093D8
:100A50000E37005C0E3500270E3400F30D3200C156
:100A60000D3100900D3000600D2E00320D2D00056F
:100A70000D2C00D90C2B00AE0C2900850C29005C34
:100A80000C2700350C27000E0C2600E80B2400C4B0
:100A90000B2400A00B23007D0B23005A0B210039EF
:100AA0000B2100180B2000F80A1F00D90A1E00BBFA
:100AB0000A1E009D0A1D00800A1D00630A1C0047D3
:100AC0000A1B002C0A1B00110A1A00F7091A00DD84
:100AD000091900C4091900AB091900920917007B14
:100AE000091800630917004C091600360916002082
:100AF0000916000A091500F5081500E0081400CCD5
:100B0000081400B8081400A4081400900813007D0D
:100B10000812006B0813005808120046081200342F
:100B2000081100230811001208110001081100F03B
:100B3000071000E0071000D0071000C0071000B039
:100B4000070F00A107100091070E0083070F007424
:100B5000070F0065070E0057070E0049070E003B00
:100B6000070D002E070E0020070D0013070D0006CD
:100B7000070D00F9060C00ED060D00E0060C00D490
:100B8000060C00C8060C00BC060C00B0060C00A445
:100B9000060B0099060C008D060B0082060B0077F1
:100BA000060B006C060B0061060A0057060B004C92
:100BB000060A0042060A0038060A002E060A002429
:100BC000060A001A060A001006090007060A00FDB8
:100BD000050900F4050900EB050900E2050900D943
:100BE000050900D0050900C7050900BE050900B5C3
:100BF000050800AD050800A50509009C050800943E
:100C00000508008C050800840508007C05080074B0
:100C10000508006C050700650508005D050700561E
:100C20000508004E05070047050700400508003885
:100C3000050700310507002A050700230507001CEA
:100C4000050600160507000F050700080506000247
:100C5000050700FB040600F5040700EE040600E8A3
:100C6000040600E2040700DB040600D5040600CFFA
:100C7000040600C9040600C3040600BD040600B74C
:100C8000040600B1040500AC040600A6040600A09A
:100C90000405009B04060095040500900406008AE4
:100CA00004050085040500800406007A040500752B
:100CB000040500700405006B04050066040500616E
:100CC0000405005C04050057040500520405004DAE
:100CD00004050048040500430405003E0404003AEE
:100CE00004050035040500300404002C0405002729
:100CF000040400230405001E0404001A0404001662
:100D0000040500110404000D040400090405000496
:100D100004040000040400FC030400F8030400F4CD
:100D2000030400F0030400EC030400E8030400E4FF
:100D3000030400E0030400DC030400D8030400D42F
:100D4000030400D0030400CC030400C8030300C55F
:100D500003030024F404D9201BC40C5C0E9804C4C3
:100D6000095F0265077101F405F900FB04B300484F
:100D7000048700C10369005803550003034500BE02
:100D8000023A008402310053022A0029022500049D
:100D9000022000E4011C00C8011900AF01170098EF
:100DA0000114008401130071011000610110005151
:100DB000010E0043010D0036010B002B010B00203A
:100DC000010B00150109000C01090003010800FBDB
:100DD000000800F3000800EB000700E4000600DE56
:100DE000000600D8000600D2000600CC000500C7AF
:100DF000000500C2000500BD000400B9000400B5F4
:100E0000000400B1000400AD000400A9000400A526
:100E1000000300A20003009F0004009B0003009851
:100E20000003009500020093000300900003008D72
:100E30000002008B0003008800020086000200848C
:100E4000000300810002007F0002007D0002007BA1
:100E500000020079000200770001007600020074B1
:100E600000020072000100710002006F0002006DBC
:100E70000001006C0002006A0001006900020067C6
:100E800000010066000100650001006400020062CC
:100E900000010061000100600001005F0002005DD0
:100EA0000001005C0001005B0001005A00010059D4
:100EB00000010058000100570001005600010055D4
:100EC00000010054000100530000005300010052D3
:100ED00000010051000100500001004F0001004ED0
:100EE0000000004E0001004D0001004C0001004BCD
:100EF0000000004B0001004A0001004900010048C9
:100F000000000048000100470001004600000046C4
:100F100000010045000000450001004400010043BD
:100F200000000043000100420000004200010041B7
:100F300000000041000100400001003F0000003FB0
:100F40000001003E0000003E0001003D0000003DA9
:100F50000001003C0000003C0000003C0001003BA0
:100F60000000003B0001003A0000003A0001003997
:100F7000000000390001003800000038000000388F
:100F80000001003700000037000100360000003685
:100F9000000000360001003500000035000000357B
:100FA0000001003400000034000000340001003370
:100FB0000000003300000033000100320000003266
:100FC000000000320001003100000031000000315B
:100FD0000001003000000030000000300001002F50
:100FE0000000002F0000002F0000002F0001002E45
:100FF0000000002E0000002E0001002D0000002D3A
:101000000000002D0000002D0001002C0000002C2D
:101010000000002C0000002C0001002B0000002B21
:101020000000002B0000002B0001002A0000002A15
:101030000000002A0000002A000100290000002909
:1010400000000029000000290000002900010028FC
:1010500000000028000000280000002800000028F0
:1010600000010027000000270000002700000027E3
:1010700000000027000100260000002600000026D6
:1010800000000026000000260001002500000025C9
:1010900000000025000000250000002500000025BC
:1010A00000010024000000240000002400000024AF
:1010B00000000024000100230000002300000023A2
:1010C0000000002300000023000000230000002394
:1010D0000001002200000022000000220000002287
:1010E0000000002200000022000100210000002179
:1010F000000000210000002100000021000000216C
:10110000000000210001002000000020000000205D
:10111000000000200000002000000020000000204F
:10112000000000200001001F0000001F0000001F41
:101130000000001F0000001F0000001F0000001F33
:101140000001001E0000001E0000001E0000001E26
:1011500000000099000000006E6F7A7A6C654361B0
:101160006C6962726174696F6E009600008600841B
:10117000035201000014008304A600000014008C38
:10118000000000000000000030F8FFFF0000000039
:10119000000000008B0000000000000000000000C4
:1011A000000000000000000000A60000008304DC36
:1011B0000500001400901F8C97340000F219000005
:1011C0000000000000000000000000008B40D9FF7C
:1011D000FFBFE6FFFF60EA00000000000000000023
:1011E00000800000009101149100149104149103F7
:1011F0001488001F026E008D0064005802880003EE
:1012000002E60088010302E60087006400580287B6
:10121000016400580291017F91007F91047F910346
:101220007F8BC8E7FFFF09EBFFFF680100000000AC
:10123000000000000000800000008BC8E7FFFF09ED
:10124000EBFFFF68010000E4FFFFFF000000000C5F
:101250000300008BC8E7FFFF09EBFFFFF000000071
:10126000D0FFFFFF000000003E0000008BC8E7FF3A
:10127000FF09EBFFFFF0000000B3FFFFFF000000DD
:1012800000850100008BF1D9FFFF09EBFFFFF000A3
:1012900000004FFEFFFF000000007F0300008BC82E
:1012A000E7FFFF88EEFFFFF00000007FFEFFFF007A
:1012B000000000D30000008BC8E7FFFF88EEFFFFAF
:1012C000F000000063FEFFFF000000008501000049
:1012D0008B67DDFFFF88EEFFFFF0000000FEFCFFE4
:1012E000FF00000000820300008BC8E7FFFF06F24A
:1012F000FFFFF00000002EFDFFFF00000000D800FF
:1013000000008BC8E7FFFF06F2FFFFF000000012AD
:10131000FDFFFF00000000850100008B67DDFFFF7F
:1013200006F2FFFFF0000000ADFBFFFF0000000031
:10133000820300008BC8E7FFFF85F5FFFFF0000088
:1013400000DDFBFFFF00000000D80000008BC8E7B5
:10135000FFFF85F5FFFFF0000000C1FBFFFF00006D
:101360000000850100008B67DDFFFF85F5FFFFF0C2
:101370000000005CFAFFFF00000000820300008B09
:10138000C8E7FFFF03F9FFFFF00000008DFAFFFF41
:1013900000000000D80000008BC8E7FFFF03F9FF42
:1013A000FFF000000070FAFFFF0000000085010060
:1013B000008B67DDFFFF03F9FFFFF00000000BF972
:1013C000FFFF00000000820300008BC8E7FFFF82E0
:1013D000FCFFFFF00000003CF9FFFF00000000D818
:1013E0000000008BC8E7FFFF82FCFFFFF000000059
:1013F0001FF9FFFF00000000850100008B67DDFF83
:10140000FF82FCFFFFF0000000BAF7FFFF000000C2
:1014100000820300008BC8E7FFFF00000000F0001F
:101420000000EBF7FFFF00000000D80000008BC8B1
:10143000E7FFFF00000000F0000000CEF7FFFF0014
:10144000000000850100008B67DDFFFF0000000049
:10145000F000000069F6FFFF0000000082030000BA
:101460008BC8E7FFFF7E030000F00000009AF6FF44
:10147000FF00000000D80000008BC8E7FFFF7E03DC
:101480000000F00000007DF6FFFF00000000850175
:1014900000008B67DDFFFF7E030000F000000019F5
:1014A000F5FFFF00000000820300008BC8E7FFFF8C
:1014B000FD060000F000000049F5FFFF00000000FD
:1014C000D80000008BC8E7FFFFFD060000F0000019
:1014D000002CF5FFFF00000000850100008B67DD98
:1014E000FFFFFD060000F0000000C8F3FFFF000052
:1014F0000000820300008BC8E7FFFF7B0A0000F0BA
:10150000000000F8F3FFFF00000000D80000008B8F
:10151000C8E7FFFF7B0A0000F0000000DBF3FFFFDD
:1015200000000000850100008B67DDFFFF7B0A00E3
:1015300000F000000077F2FFFF00000000820300CF
:10154000008BC8E7FFFFFA0D0000F0000000A7F2D3
:10155000FFFF00000000D80000008BC8E7FFFFFA83
:101560000D0000F00000008AF2FFFF00000000857F
:101570000100008B67DDFFFFFA0D0000F0000000A6
:1015800026F1FFFF00000000820300008BC8E7FF88
:10159000FF78110000F000000056F1FFFF0000008E
:1015A00000D80000008BC8E7FFFF78110000F000B2
:1015B000000039F1FFFF00000000850100008B678B
:1015C000DDFFFF78110000F0000000D5EFFFFF0005
:1015D000000000820300008BC8E7FFFFF714000043
:1015E000F000000005F0FFFF00000000D800000040
:1015F0008BC8E7FFFFF7140000F0000000E8EFFFE2
:10160000FF00000000850100008B67DDFFFFF7147D
:101610000000F000000084EEFFFF000000008203E5
:1016200000008B6AF5FFFF15F9FFFF68010000B4A9
:10163000EEFFFF000000000E0100008B6AF5FFFFC7
:1016400015F9FFFFF000000084EEFFFF000000002E
:101650009C0000008B6AF5FFFF15F9FFFFF000000A
:101660000067EEFFFF00000000850100008B6AF5B7
:10167000FFFFEB060000F000000003EDFFFF00009D
:1016800000007F0300008BE9F8FFFF15F9FFFFF072
:1016900000000033EDFFFF00000000D30000008BCE
:1016A000E9F8FFFF15F9FFFFF000000016EDFFFF5E
:1016B00000000000850100008BE9F8FFFF750300C2
:1016C00000F0000000B2EBFFFF000000008203000A
:1016D000008B67FCFFFF15F9FFFFF0000000E2EB55
:1016E000FFFF00000000D80000008B67FCFFFF1523
:1016F000F9FFFFF0000000C5EBFFFF0000000085D0
:101700000100008B67FCFFFF75030000F000000084
:1017100061EAFFFF00000000820300008BE6FFFF8C
:10172000FF15F9FFFFF000000091EAFFFF00000045
:1017300000D80000008BE6FFFFFF15F9FFFFF00067
:10174000000074EAFFFF00000000850100008BE646
:10175000FFFFFF75030000F000000010E9FFFF002D
:10176000000000820300008B6403000015F9FFFFF6
:10177000F000000040E9FFFF00000000D80000007A
:101780008B6403000015F9FFFFF000000023E9FF60
:10179000FF00000000850100008B6403000075035A
:1017A0000000F0000000BFE7FFFF00000000820320
:1017B00000008BE206000015F9FFFFF0000000EFCB
:1017C000E7FFFF00000000D80000008BE2060000E9
:1017D00015F9FFFFF0000000D2E7FFFF0000000056
:1017E000850100008BE206000075030000F0000098
:1017F000006EE6FFFF00000000820300008B610A1C
:10180000000015F9FFFFF00000009EE6FFFF00005A
:101810000000D80000008B610A000015F9FFFFF0FE
:1018200000000081E6FFFF00000000850100008B42
:10183000610A000075030000F00000001DE5FFFFD5
:1018400000000000820300008BDF0D000015F9FF8F
:10185000FFF00000004DE5FFFF00000000D8000091
:10186000008BDF0D000015F9FFFFF000000030E5F0
:10187000FFFF00000000850100008BDF0D000075F8
:10188000030000F0000000CCE3FFFF000000008236
:101890000300008B5E11000015F9FFFFF00000004F
:1018A000FCE3FFFF00000000D80000008B5E110089
:1018B0000015F9FFFFF0000000DFE3FFFF0000006C
:1018C00000850100008B5E11000075030000F00030
:1018D00000007BE2FFFF00000000820300008BDCC1
:1018E00014000015F9FFFFF0000000ABE2FFFF005D
:1018F000000000D80000008BDC14000015F9FFFF89
:10190000F00000008EE2FFFF0000000085010000F3
:101910008BDC14000075030000F00000002AE1FFDA
:10192000FF00000000820300008B5B18000015F927
:10193000FFFFF00000005AE1FFFF00000000D800A8
:1019400000008B5B18000015F9FFFFF00000003D60
:10195000E1FFFF00000000850100008B5B18000024
:1019600075030000F0000000D9DFFFFF0000000059
:10197000820300008BDA1B000015F9FFFFF0000066
:101980000009E0FFFF00000000D80000008BDA1B18
:10199000000015F9FFFFF0000000ECDFFFFF000082
:1019A0000000850100008BDA1B000075030000F0C9
:1019B00000000088DEFFFF00000000820300008BB3
:1019C000581F000015F9FFFFF0000000B8DEFFFF10
:1019D00000000000D80000008B581F000015F9FF20
:1019E000FFF00000009BDEFFFF000000008501000B
:1019F000008B581F000075030000F000000037DD69
:101A0000FFFF00000000820300008B581F000075DC
:101A1000030000F000000067DDFFFF000000000C85
:101A20000300008C581F000075030000F000000048
:101A30000000000000000000860189188BC8E7FF45
:101A4000FF3EEBFFFF680100000000000000000007
:101A500000DF0000008BC8E7FFFF3EEBFFFF6801DF
:101A6000000000000000E4FFFFFF0C0300008BC833
:101A7000E7FFFF3EEBFFFFF000000000000000D09A
:101A8000FFFFFF3E0000008BC8E7FFFF3EEBFFFFBC
:101A9000F000000000000000B3FFFFFF8501000020
:101AA0008B2AF2FFFF3EEBFFFFF00000000000007A
:101AB000004FFEFFFF820300008BC8E7FFFFB4EE7C
:101AC000FFFFF0000000000000007FFEFFFFD800D5
:101AD00000008BC8E7FFFFB4EEFFFFF0000000003E
:101AE00000000063FEFFFF850100008B2AF2FFFF6C
:101AF000B4EEFFFFF000000000000000FEFCFFFF5E
:101B0000820300008BC8E7FFFF2AF2FFFFF000000E
:101B100000000000002EFDFFFFD80000008BC8E78A
:101B2000FFFF2AF2FFFFF00000000000000012FD9E
:101B3000FFFF850100008B2AF2FFFF2AF2FFFFF072
:101B400000000000000000ADFBFFFF820300008BDF
:101B5000C8E7FFFF9FF5FFFFF00000000000000056
:101B6000DDFBFFFFD80000008BC8E7FFFF9FF5FFFC
:101B7000FFF000000000000000C1FBFFFF85010036
:101B8000008B2AF2FFFF9FF5FFFFF000000000002E
:101B900000005CFAFFFF820300008BC8E7FFFF151F
:101BA000F9FFFFF0000000000000008DFAFFFFD8F1
:101BB0000000008BC8E7FFFF15F9FFFFF0000000F1
:101BC0000000000070FAFFFF850100008B2AF2FF81
:101BD000FF15F9FFFFF0000000000000000BF9FF07
:101BE000FF820300008BC8E7FFFF8BFCFFFFF000C4
:101BF0000000000000003CF9FFFFD80000008BC887
:101C0000E7FFFF8BFCFFFFF0000000000000001F5B
:101C1000F9FFFF850100008B2AF2FFFF8BFCFFFF1D
:101C2000F000000000000000BAF7FFFF8203000090
:101C30008BC8E7FFFF00000000F00000000000007C
:101C400000EBF7FFFFD80000008BC8E7FFFF0000A4
:101C50000000F000000000000000CEF7FFFF85014B
:101C600000008B2AF2FFFF00000000F000000000DF
:101C700000000069F6FFFF820300008BC8E7FFFF4A
:101C800075030000F0000000000000009AF6FFFF5E
:101C9000D80000008BC8E7FFFF75030000F00000CC
:101CA00000000000007DF6FFFF850100008B2AF296
:101CB000FFFF75030000F00000000000000019F5B0
:101CC000FFFF820300008BC8E7FFFFEB060000F078
:101CD0000000000000000049F5FFFFD80000008B65
:101CE000C8E7FFFFEB060000F00000000000000066
:101CF0002CF5FFFF850100008B2AF2FFFFEB0600A9
:101D000000F000000000000000C8F3FFFF820300A5
:101D1000008BC8E7FFFF610A0000F0000000000030
:101D20000000F8F3FFFFD80000008BC8E7FFFF6159
:101D30000A0000F000000000000000DBF3FFFF8558
:101D40000100008B2AF2FFFF610A0000F000000092
:101D50000000000077F2FFFF820300008BC8E7FF5E
:101D6000FFD60D0000F000000000000000A7F2FF09
:101D7000FFD80000008BC8E7FFFFD60D0000F00081
:101D80000000000000008AF2FFFF850100008B2A9E
:101D9000F2FFFFD60D0000F000000000000000265A
:101DA000F1FFFF820300008BC8E7FFFF4C1100002A
:101DB000F00000000000000056F1FFFFD800000016
:101DC0008BC8E7FFFF4C110000F00000000000008E
:101DD0000039F1FFFF850100008B2AF2FFFF4C1153
:101DE0000000F000000000000000D5EFFFFF8203BC
:101DF00000008BC8E7FFFFC2140000F000000000E5
:101E000000000005F0FFFFD80000008BC8E7FFFFCF
:101E1000C2140000F000000000000000E8EFFFFF27
:101E2000850100008B2AF2FFFFC2140000F00000C1
:101E3000000000000084EEFFFF820300008B9FF58E
:101E4000FFFFB4EEFFFF6801000000000000B4EEE9
:101E5000FFFFCE0000008B9FF5FFFFB4EEFFFFF009
:101E60000000000000000084EEFFFF9C0000008BDB
:101E70009FF5FFFFB4EEFFFFF00000000000000040
:101E800067EEFFFF850100008B9FF5FFFF15F9FF4F
:101E9000FFF00000000000000003EDFFFF820300E0
:101EA000008B15F9FFFFB4EEFFFFF000000000000B
:101EB000000033EDFFFFD80000008B15F9FFFFB4E1
:101EC000EEFFFFF00000000000000016EDFFFF85B0
:101ED0000100008B15F9FFFF15F9FFFFF00000006E
:101EE00000000000B2EBFFFF820300008B8BFCFFC1
:101EF000FFB4EEFFFFF000000000000000E2EBFF87
:101F0000FFD80000008B8BFCFFFFB4EEFFFFF0005A
:101F1000000000000000C5EBFFFF850100008B8B77
:101F2000FCFFFF15F9FFFFF000000000000000615A
:101F3000EAFFFF820300008B00000000B4EEFFFF09
:101F4000F00000000000000091EAFFFFD800000050
:101F50008B00000000B4EEFFFFF000000000000066
:101F60000074EAFFFF850100008B0000000015F9F6
:101F7000FFFFF00000000000000010E9FFFF8203F7
:101F800000008B75030000B4EEFFFFF000000000BE
:101F900000000040E9FFFFD80000008B750300003F
:101FA000B4EEFFFFF00000000000000023E9FFFF97
:101FB000850100008B7503000015F9FFFFF000009C
:101FC0000000000000BFE7FFFF820300008BEB066C
:101FD0000000B4EEFFFFF000000000000000EFE79B
:101FE000FFFFD80000008BEB060000B4EEFFFFF00F
:101FF00000000000000000D2E7FFFF850100008B19
:10200000EB06000015F9FFFFF000000000000000E3
:102010006EE6FFFF820300008B610A0000B4EEFF52
:10202000FFF0000000000000009EE6FFFFD8000067
:10203000008B610A0000B4EEFFFFF000000000001A
:10204000000081E6FFFF850100008B610A0000159A
:10205000F9FFFFF0000000000000001DE5FFFF8217
:102060000300008BD60D0000B4EEFFFFF00000006F
:10207000000000004DE5FFFFD80000008BD60D00EA
:1020800000B4EEFFFFF00000000000000030E5FFAC
:10209000FF850100008BD60D000015F9FFFFF00051
:1020A000000000000000CCE3FFFF820300008B4C27
:1020B000110000B4EEFFFFF000000000000000FC83
:1020C000E3FFFFD80000008B4C110000B4EEFFFFCF
:1020D000F000000000000000DFE3FFFF85010000CA
:1020E0008B4C11000015F9FFFFF00000000000000C
:1020F000007BE2FFFF820300008BC2140000B4EEFD
:10210000FFFFF000000000000000ABE2FFFFD8007E
:1021100000008BC2140000B4EEFFFFF000000000CE
:102120000000008EE2FFFF850100008BC21400005A
:1021300015F9FFFFF0000000000000002AE1FFFF9A
:10214000820300008B38180000B4EEFFFFF000009F
:1021500000000000005AE1FFFFD80000008B381893
:102160000000B4EEFFFFF0000000000000003DE1C1
:10217000FFFF850100008B3818000015F9FFFFF004
:1021800000000000000000D9DFFFFF820300008B89
:10219000AD1B0000B4EEFFFFF000000000000000E7
:1021A00009E0FFFFD80000008BAD1B0000B4EEFF7C
:1021B000FFF000000000000000ECDFFFFF850100E1
:1021C000008BAD1B000015F9FFFFF00000000000C0
:1021D000000088DEFFFF820300008B231F0000B495
:1021E000EEFFFFF000000000000000B8DEFFFFD8A7
:1021F0000000008B231F0000B4EEFFFFF000000082
:10220000000000009BDEFFFF850100008B231F0004
:102210000015F9FFFFF00000000000000037DDFFAF
:10222000FF820300008B231F000015F9FFFF30F22F
:1022300000000000000037DDFFFFC500000089003E
:1022400088000302000088010302000088001F02CA
:1022500000009502000000506C6561736520776195
:1022600069740084037D0100001400830488000069
:102270000014008C000000000000000030F8FFFF98
:1022800000000000000000008E00000000000000C0
:1022900000000000000000000000000000572904BA
:1022A00000188304DC05000014008C97340000F350
:1022B0001900000000000000000000000000009570
:1022C000000000005469676874656E20656163688A
:1022D000206F662074686520009501000000746816
:1022E000726565206B6E6F627320756E6465722017
:1022F0002020009501000000746865206275696CFB
:102300006420706C6174666F726D20200095070008
:10231000000061626F757420666F7572207475724B
:102320006E732E00950000000049276D20676F69CD
:102330006E6720746F206D6F7665206D7900950152
:1023400000000065787472756465722061726F7543
:102350006E6420746F20200095010000006469669F
:10236000666572656E7420706F696E747320736F2A
:1023700020009507000000796F752063616E20636F
:102380006865636B2E2E2E00950000000074686552
:10239000206865696768742E2041742065616368F0
:1023A00020009501000000706F696E742C206C6F26
:1023B0006F73656E20746865202020009501000011
:1023C00000737065636966696564206B6E6F622077
:1023D000756E74696C009507000000746865206E66
:1023E0006F7A7A6C6520616C6D6F73742E2E2E007F
:1023F0009500000000746F756368657320746865EC
:10240000206275696C642020200095010000007036
:102410006C6174652E20546865206E6F7A7A6C65E5
:1024200020697300950100000061742074686520C4
:102430007269676874206865696768742000950729
:102440000000007768656E2061207468696E2070F6
:10245000696563652E2E2E0095000000006F6620D2
:1024600070617065722077696C6C20736C6964654B
:10247000200095010000006265747765656E207428
:102480006865206E6F7A7A6C6520200095010000E7
:1024900000616E64206275696C6420706C617465A3
:1024A000207769746800950700000020736F6D65E0
:1024B000206672696374696F6E2E009502000000D9
:1024C000506C656173652077616974008E97340084
:1024D00000F2190000D0070000000000000000001A
:1024E000009AE90300188EB605000039180000D0E4
:1024F000070000000000000000000024612900180F
:102500008EB5050000381800000000000000000033
:102510000000000000E09304001895000000004156
:10252000646A757374207468652072656172206BCB
:102530006E6F62009501000000756E74696C20700A
:1025400061706572206A75737420202020009501E7
:10255000000000736C69646573206265747765655B
:102560006E2074686520200095070000006E6F7A69
:102570007A6C6520616E6420706C617465009502F0
:10258000000000506C656173652077616974008E8E
:10259000B505000038180000D0070000000000005A
:1025A00000000000E0930400188E51160000C8E7F8
:1025B000FFFFD00700000000000000000000802A9C
:1025C0002D00188E51160000C8E7FFFF0000000024
:1025D0000000000000000000E093040018950000D7
:1025E000000041646A7573742066726F6E742072A5
:1025F0006967687420200095010000006B6E6F62AF
:1026000020756E74696C20706170657220202020C6
:102610000095010000006A75737420736C6964652D
:1026200073206265747765656E2000950700000071
:102630006E6F7A7A6C6520616E6420706C6174656F
:10264000009502000000506C656173652077616938
:1026500074008E51160000C7E7FFFFD0070000008E
:1026600000000000000000E0930400188E69F4FFF1
:10267000FFC8E7FFFFD007000000000000000000D7
:10268000003FE81D00188E69F4FFFFC8E7FFFF0058
:102690000000000000000000000000E093040018AB
:1026A000950000000041646A7573742066726F6E55
:1026B00074206C6566742020200095010000006B7A
:1026C0006E6F6220756E74696C2070617065722027
:1026D0002020200095010000006A75737420736C3F
:1026E00069646573206265747765656E200095077F
:1026F0000000006E6F7A7A6C6520616E6420706CE9
:10270000617465009502000000506C65617365207E
:1027100077616974008E69F4FFFFC8E7FFFFD00797
:1027200000000000000000000000E0930400189585
:10273000000000004E6F772049276D20676F696E9B
:102740006720746F20202020009501000000736531
:102750006E64206D7920657874727564657220747A
:102760006F20009501000000616C6C207468726538
:102770006520706F696E747320202020009507001B
:102780000000616761696E20746F2072656368651F
:10279000636B2E009502000000506C65617365202C
:1027A00077616974008EB505000038180000D00705
:1027B0000000000000000000000078381B00188EA8
:1027C000B6050000381800000000000000000000FE
:1027D00000000000E0930400189500000000416430
:1027E0006A75737420746865207265617220202098
:1027F00020200095010000006B6E6F6220756E74E2
:10280000696C2070617065722020202000950100A5
:1028100000006A75737420736C6964657320626567
:10282000747765656E200095070000006E6F7A7AF8
:102830006C6520616E6420706C61746500950200A7
:102840000000506C656173652077616974008EB516
:1028500005000038180000D007000000000000004C
:10286000000000E0930400188E2C290000C8E7FF48
:10287000FFD007000000000000000000005AC51F44
:1028800000188E2D290000C8E7FFFF00000000009F
:1028900000000000000000E0930400189500000014
:1028A0000041646A7573742066726F6E7420726979
:1028B00067687420200095010000006B6E6F622035
:1028C000756E74696C207061706572202020200024
:1028D00095010000006A75737420736C69646573F8
:1028E000206265747765656E200095070000006EB4
:1028F0006F7A7A6C6520616E6420706C617465001B
:102900009502000000506C65617365207761697401
:10291000008E2C290000C8E7FFFFD0070000000050
:10292000000000000000E0930400188E12E2FFFF98
:10293000C8E7FFFFD0070000000000000000000013
:10294000D0A02500188E13E2FFFFC8E7FFFF0000AC
:1029500000000000000000000000E0930400189553
:102960000000000041646A7573742066726F6E74B3
:10297000206C6566742020200095010000006B6EBD
:102980006F6220756E74696C2070617065722020B2
:1029900020200095010000006A75737420736C6933
:1029A000646573206265747765656E200095070025
:1029B00000006E6F7A7A6C6520616E6420706C61C5
:1029C0007465009502000000506C656173652077A6
:1029D000616974008E12E2FFFFC8E7FFFFD00700B5
:1029E000000000000000000000E0930400188EB515
:1029F00005000000000000D00700000000000000FB
:102A000000000095CD1600188EB6050000000000ED
:102A100000000000000000000000000000E093043F
:102A2000001895000000004E6F77206C65742773C6
:102A300020747269706C65202020200095010000D0
:102A400000636865636B2D2D207061706572207363
:102A5000686F756C640095010000006A75737420DE
:102A6000736C696465206265747765656E2020000B
:102A700095070000006E6F7A7A6C6520616E6420A5
:102A8000706C61746500891F9502000000506C65D0
:102A900061736520776169740084037D010000140F
:102AA0000083048800000014008C00000000000077
:102AB000000030F8FFFF00000000000000008E0062
:102AC0000000000000000000000000000000000006
:102AD00000000057290400188304DC0500001400DE
:102AE0008C97340000F31900000000000000000083
:102AF00000000000009500000000546967687465DC
:102B00006E2065616368206F66207468652000959B
:102B1000010000007468726565206B6E6F6273203F
:102B2000756E6465722020200095010000007468B5
:102B300065206275696C6420706C6174666F726D7B
:102B4000202000950700000061626F757420666F99
:102B50007572207475726E732E0095000000004926
:102B6000276D20676F696E6720746F206D6F7665C3
:102B7000206D7900950100000065787472756465B8
:102B8000722061726F756E6420746F202000950151
:102B9000000000646966666572656E7420706F6916
:102BA0006E747320736F20009507000000796F75B5
:102BB0002063616E20636865636B2E2E2E00950086
:102BC000000000746865206865696768742E20419C
:102BD00074206561636820009501000000706F69D2
:102BE0006E742C206C6F6F73656E20746865202086
:102BF0002000950100000073706563696669656473
:102C0000206B6E6F6220756E74696C009507000012
:102C100000746865206E6F7A7A6C6520616C6D6FE8
:102C200073742E2E2E009500000000746F7563687B
:102C3000657320746865206275696C6420202000CB
:102C40009501000000706C6174652E205468652049
:102C50006E6F7A7A6C6520697300950100000061DF
:102C60007420746865207269676874206865696794
:102C70006874200095070000007768656E20612069
:102C80007468696E2070696563652E2E2E0095004C
:102C90000000006F662070617065722077696C6C4F
:102CA00020736C6964652000950100000062657402
:102CB0007765656E20746865206E6F7A7A6C652022
:102CC00020009501000000616E64206275696C64EB
:102CD00020706C6174652077697468009507000046
:102CE0000020736F6D65206672696374696F6E2E64
:102CF000009502000000506C656173652077616982
:102D000074008E97340000F3190000D00700000013
:102D1000000000000000009AE90300188E00000087
:102D20000038180000D0070000000000000000007C
:102D3000006C692E00188E0000000038180000009A
:102D40000000000000000000000000E093040018F4
:102D5000950000000041646A7573742074686520F2
:102D600072656172206B6E6F6200950100000075E4
:102D70006E74696C207061706572206A757374205E
:102D8000202020009501000000736C6964657320A9
:102D90006265747765656E2074686520200095070C
:102DA0000000006E6F7A7A6C6520616E6420706C32
:102DB000617465009502000000506C6561736520C8
:102DC00077616974008E0000000038180000D00799
:102DD00000000000000000000000E0930400188ED6
:102DE0009C100000C8E7FFFFD007000000000000B3
:102DF00000000000802A2D00188E9B100000C8E7FC
:102E0000FFFF000000000000000000000000E09351
:102E1000040018950000000041646A757374206610
:102E2000726F6E74207269676874202000950100CB
:102E300000006B6E6F6220756E74696C207061703B
:102E40006572202020200095010000006A757374CF
:102E500020736C69646573206265747765656E20A4
:102E60000095070000006E6F7A7A6C6520616E64D1
:102E700020706C617465009502000000506C656103
:102E800073652077616974008E9C100000C8E7FFAD
:102E9000FFD00700000000000000000000E09304E5
:102EA00000188E64EFFFFFC8E7FFFFD007000000A7
:102EB00000000000000000004C1D00188E65EFFFB0
:102EC000FFC8E7FFFF000000000000000000000056
:102ED00000E093040018950000000041646A7573D7
:102EE000742066726F6E74206C65667420202000FA
:102EF00095010000006B6E6F6220756E74696C2026
:102F00007061706572202020200095010000006A29
:102F100075737420736C696465732062657477657A
:102F2000656E200095070000006E6F7A7A6C652050
:102F3000616E6420706C6174650095020000005041
:102F40006C656173652077616974008E64EFFFFFC3
:102F5000C8E7FFFFD00700000000000000000000ED
:102F6000E09304001895000000004E6F7720492779
:102F70006D20676F696E6720746F20202020009598
:102F80000100000073656E64206D792065787472AD
:102F90007564657220746F20009501000000616CFB
:102FA0006C20746872656520706F696E7473202080
:102FB0002020009507000000616761696E20746F32
:102FC000207265636865636B2E00950200000050F7
:102FD0006C656173652077616974008E0000000084
:102FE00038180000D00700000000000000000000BA
:102FF00080191B00188E0000000038180000000027
:1030000000000000000000000000E093040018959C
:103010000000000041646A75737420746865207252
:1030200065617220202020200095010000006B6E59
:103030006F6220756E74696C2070617065722020FB
:1030400020200095010000006A75737420736C697C
:10305000646573206265747765656E20009507006E
:1030600000006E6F7A7A6C6520616E6420706C610E
:103070007465009502000000506C656173652077EF
:10308000616974008E0000000038180000D007004D
:10309000000000000000000000E0930400188E40D3
:1030A0002B0000C8E7FFFFD0070000000000000071
:1030B000000000A65D2200188E3F2B0000C8E7FF2D
:1030C000FF000000000000000000000000E093048A
:1030D0000018950000000041646A757374206672E0
:1030E0006F6E74207269676874202000950100007B
:1030F000006B6E6F6220756E74696C207061706514
:1031000072202020200095010000006A7573742051
:10311000736C69646573206265747765656E200001
:1031200095070000006E6F7A7A6C6520616E6420EE
:10313000706C617465009502000000506C656173ED
:10314000652077616974008E402B0000C8E7FFFF9F
:10315000D00700000000000000000000E093040021
:10316000188EC0D4FFFFC7E7FFFFD00700000000A4
:10317000000000000000C0C62D00188EC1D4FFFF63
:10318000C8E7FFFF00000000000000000000000092
:10319000E093040018950000000041646A757374A0
:1031A0002066726F6E74206C656674202020009516
:1031B000010000006B6E6F6220756E74696C207088
:1031C00061706572202020200095010000006A7562
:1031D000737420736C6964657320626574776565C8
:1031E0006E200095070000006E6F7A7A6C65206192
:1031F0006E6420706C617465009502000000506C74
:10320000656173652077616974008EC0D4FFFFC863
:10321000E7FFFFD00700000000000000000000E012
:10322000930400188E0000000000000000D007008A
:10323000000000000000000000913B1A00188E0002
:10324000000000000000000000000000000000007E
:10325000000000E09304001895000000004E6F7716
:10326000206C6574277320747269706C652020204F
:1032700020009501000000636865636B2D2D2070B0
:10328000617065722073686F756C64009501000051
:10329000006A75737420736C696465206265747765
:1032A00065656E20200095070000006E6F7A7A6CCD
:1032B0006520616E6420706C61746500891F9502E1
:1032C000000000506C6561736520776169742E2E73
:1032D0002E008403690100001400830488000000AC
:1032E00014008C000000000000000030F8FFFF0018
:1032F000000000000000008E000000000000000040
:103300000000000000000000000000005729040039
:10331000188304DC0500001400901F891F5F00362D
:10332000083608FF1046696C616D656E7420466151
:103330006E20202020202020004D792074656D70A3
:1033400065726174757265207761732020636861AE
:103350006E6765642065787465726E616C6C792E39
:1033600020526573656C6563742066696C616D6578
:103370006E742020206D656E7520746F20747279D4
:1033800020616761696E2E20200020534420636114
:1033900072642072656164206572726F72004927E1
:1033A0006D20616C7265616479206275696C646915
:1033B0006E67005761726E696E673A4275696C6438
:1033C00020737065656473666173746572207468D8
:1033D000616E2035306D6D2F7320207265717569B7
:1033E00072652078336720666F726D617420206685
:1033F0006F72206265737420726573756C74732EBE
:1034000020202000526573756D65204275696C64DB
:103410002020202020202000536C65657020284348
:103420006F6C642050617573652920004368616E7C
:1034300067652046696C616D656E742020202000F0
:1034400043616E63656C204275696C6420202020A6
:10345000202020002020205A2050617573652048CC
:103460006569676874202020005A20506175736573
:103470002048656967687420202020200042756913
:103480006C642053746174697374696373202020C1
:10349000004261636B20746F204D6F6E69746F72B0
:1034A0002020202000202020202020006820206DC7
:1034B000004275696C642046696E697368656421B1
:1034C00020202020202020202020202020202020FC
:1034D0002020202020202020204275696C64205468
:1034E000696D652020202020206820206D004C6917
:1034F0006E653A202020202020202020202020201F
:103500002020004275696C642054696D653A202062
:103510002020206820206D004C6173742042756962
:103520006C643A20202020206820206D00457374B0
:10353000696D61746564204275696C642054696DBD
:10354000654C69666574696D6520546F74616C3A89
:1035500020202020680057616974696E6720666FBB
:103560007220486F6D696E67200077616974696EBB
:1035700067200020204E4120202020006572726FBD
:103580007221004455414C20200053494E474C4580
:10359000004F464620202000435553544F4D0057BE
:1035A000484954452000505552504C4500424C5516
:1035B00045202000475245454E200050494E4B20A3
:1035C00020004F52414E47450052454420202000E4
:1035D00048656174656420506C61746500496E666D
:1035E0006F20616E642053657474696E6773202068
:1035F00000426F742053746174697374696373203B
:103600002020202000416363656C65726174652031
:1036100020202020202020200065786974206D65FE
:103620006E75202020202020202020200048656C5E
:103630007020546578742020202020202020202015
:10364000004865617420486F6C6420202020202091
:103650006D2020200048656174204C454473202073
:103660002020202020202020004C454420436F6C47
:103670006F7220202020202020202020005A20505F
:103680006F736974696F6E2020202020206D6D207B
:103690000050617573652041637469766520202050
:1036A0002020202000536F756E64202020202020D1
:1036B000202020202020202000546F6F6C20436F9A
:1036C000756E742020202020202020200043616C73
:1036D000696272617465204E6F7A7A6C657320201E
:1036E00000526573746F72652044656661756C7411
:1036F000732020200047656E6572616C20536574ED
:1037000074696E677320202000507265686561746B
:103710002053657474696E67732020200053746FA2
:103720007020426C696E6B696E672120202020201A
:1037300000426C696E6B204C454473202020202091
:1037400020202020004C6576656C204275696C64F1
:1037500020506C617465202000456E61626C6520AC
:103760005374657070657273202020200044697363
:1037700061626C65205374657070657273202020DF
:103780000056657273696F6E204E756D62657220AA
:10379000202020200052756E205374617274757061
:1037A0002053637269707420004368616E676520FE
:1037B00046696C616D656E742020202000486F6D35
:1037C00065204178657320202020202020202020A3
:1037D000004A6F67204D6F64652020202020202044
:1037E00020202020004D6F6E69746F72204D6F6431
:1037F0006520202020202020005574696C697469A0
:103800006573202020202020202020200050726579
:103810006865617420202020202020202020202086
:10382000004275696C642066726F6D2053442020DD
:103830002020202000492063616E2774207265617A
:103840006420534420202020206361726473207719
:103850006974682073746F7261676520206C61728F
:10386000676572207468616E203247422E202020E6
:103870002020202020202020202020202020202048
:10388000202020202000492063616E27742072656B
:10389000616420746869732020205344206361723E
:1038A0006420666F726D6174212020202020547284
:1038B00079207265666F726D617474696E6720201D
:1038C0002020746865206361726420746F20464113
:1038D0005431362E202000534420636172642072DC
:1038E000656164206572726F72004E6F20534420D0
:1038F0006361726420666F756E6400556E50617509
:10390000736520202020202020202020202000500F
:103910006175736520202020202020202020202079
:103920002020005175697420746869732070726F6B
:10393000636573733F0043616E63656C20746869EF
:1039400073206275696C643F002044656661756C24
:10395000742076616C7565733F00205265736574E1
:103960002053657474696E677320746F2020005053
:103970006C6174666F726D20202020202020200052
:103980004C65667420546F6F6C202020202020200E
:103990002020202000526967687420546F6F6C20CB
:1039A00020202020202020202000205072656865E3
:1039B00061742053657474696E677320202000451C
:1039C000787472756465723A2020202D2D2D2F2D6C
:1039D0002D2D4300506C6174666F726D3A2020206B
:1039E0002D2D2D2F2D2D2D43004C204578747275D3
:1039F0006465723A202D2D2D2F2D2D2D4300522040
:103A000045787472756465723A202D2D2D2F2D2DF9
:103A10002D4300202D2D250048656174696E673A9D
:103A20002020202020202020202020200048656108
:103A300074696E673A0047414D45204F5645522103
:103A40000020202020202020205A2B202020202051
:103A500020202020200020203C2D59202842616376
:103A60006B29202020202020202000202020202022
:103A70002020205A2D20202020202020202020001F
:103A80002020202020202020592D202020202020F0
:103A9000202020200020203C2D5820284261636BEC
:103AA0002920205A2D3E20202000202020202020C8
:103AB0002020592B202020202020202020200020E2
:103AC00020202020202020582D20202020202020B1
:103AD00020202000202020202020284261636B2904
:103AE000202020592D3E2020002020202020202092
:103AF00020582B20202020202020202020002020A3
:103B00002020204A6F67206D6F64652020202020D0
:103B1000202000556E6C6F6164206C6566740055E2
:103B20006E6C6F616420726967687400556E6C6FAB
:103B30006164004C6F6164004C6F6164206C656669
:103B400074004C6F61642072696768740066726FFC
:103B50006D20746865206E6F7A7A6C653F20202036
:103B6000200044696420706C617374696320657817
:103B7000747275646520004C6574277320747279C3
:103B800020616761696E2E004D79206865696768FC
:103B90007420697320676F6F642120200068656955
:103BA00067687420636865636B206F75743F2000DD
:103BB000446F6573206D79206E6F7A7A6C65200092
:103BC000746F206D616B6520736F6D657468696ECD
:103BD000673F202000486F77276420697420676F53
:103BE0003F2052656164792020004D79206D6F740B
:103BF0006F722074696D6564206F75742020616632
:103C00007465722035206D696E757465732E202081
:103C100020205072657373204D20746F2065786981
:103C2000742E202020202020202020202020202032
:103C30002020202020202020202000477265617451
:103C400021202049276C6C2073746F702020207213
:103C5000756E6E696E67206D792065787472756413
:103C600065722E5072657373204D20746F20636FE0
:103C70006E74696E75652E20202020202020202063
:103C80002020202020202020202020005765276C85
:103C90006C206B65657020676F696E672E20202031
:103CA000496620796F7527726520686176696E674D
:103CB0002020202074726F75626C652C206368650B
:103CC000636B206F757420206D616B6572626F7419
:103CD0002E636F6D2F68656C70202020004F4B2184
:103CE0002049276C6C206B656570206D7920202041
:103CF000206D6F746F722072756E6E696E672E2004
:103D0000596F7520206D6179206E65656420746F30
:103D10002070757368202020206861726465722E9F
:103D20002E2E202020202020202020202000666908
:103D30006C616D656E74206672656520616E6420CD
:103D40002020636C6F736520746865206C657665F0
:103D5000722E20202020507265737320274D27205B
:103D6000746F20657869742E202020202020202068
:103D7000202020202020202020202020202000572C
:103D800068656E206D792066696C616D656E742062
:103D900069732072656C65617365642C2020202036
:103DA00020202020202020507265737320274D276B
:103DB00020746F20657869742E2020202020202018
:103DC0002020202020202020202020202020200013
:103DD0005768656E2066696C616D656E74206973E5
:103DE000202020206265696E672065787472756492
:103DF00065642066726F6D20746865206E6F7A7AD4
:103E00006C652C20202020202020202050726573FB
:103E10007320274D2720746F20657869742E202029
:103E2000005768656E2066696C616D656E74206907
:103E300073202020206265696E6720657874727532
:103E40006465642066726F6D20746865206E6F7A99
:103E50007A6C652C205072657373204D20746F202E
:103E600073746F7020657874727564696E672E2044
:103E70002000756E74696C20796F75206665656CBD
:103E80002074686520206D6F746F722074756720D0
:103E9000697420696E2E202020205075736820667A
:103EA0006F72206120666577206D6F726520736583
:103EB000636F6E64732C207468656E20776169741B
:103EC0002E200049276D20726561647921204465A8
:103ED0007461636820202074686520677569646573
:103EE000207475626520616E6420206D6F76652098
:103EF000746865206C6576657220746F202020746C
:103F00006865206C6566742E202050756C6C2E2EB2
:103F10002E20200049276D2072656164792120449C
:103F20006574616368202020746865206775696422
:103F300065207475626520616E6420206D6F766502
:103F400020746865206C6576657220746F2020206F
:103F50007468652072696768742E202050756C6CD7
:103F60002E2E2E200049276D207265616479212054
:103F700050756C6C20746865206775696465207481
:103F8000756265206F666620616E64202070756CB6
:103F90006C207468652066696C616D656E742020A4
:103FA0002067656E746C792E2E2E20202020202014
:103FB00020202020200049276D207265616479212E
:103FC0002050756C6C207468652067756964652085
:103FD00074756265206F666620616E64202070755E
:103FE0007368207468652066696C616D656E742005
:103FF00020207468726F7567682E2E2E2020202076
:10400000202020202020004F4B2049276D20726562
:1040100061647921202020202020204E6F77207796
:1040200065276C6C206C6F61642074686520207259
:10403000696768742065787472756465722E2020D3
:10404000202020507573682066696C616D656E7400
:1040500020696E2E2E2E20004F4B2049276D207296
:10406000656164792120202020202020507573680C
:10407000207468652066696C616D656E742020200F
:104080007468726F7567682E2E2E202020202020E5
:104090002020202020202020202020202020202020
:1040A00020202020202020200048656174696E6750
:1040B0002050726F67726573733A20202020202091
:1040C00020202020202020202020202020202020F0
:1040D00020202020202020202020202020202020E0
:1040E00020202020202020202020202020202020D0
:1040F00020202020202020202000506C6561736546
:104100002077616974207768696C6520492068654B
:104110006174206D792065787472756465722120F0
:10412000202020202020202020202020202020208F
:10413000202020202020202020202020202020207F
:104140002020202020202020202000706F7073204D
:104150006F757420696E2066726F6E742E20205702
:1041600068656E207468652066696C616D656E7443
:1041700020697372656164792C2070726573732095
:10418000274D2720746F20636F6E74696E75652EDE
:1041900020202020202020202020200065787472FC
:1041A0007564657220626C6F636B2E204665656472
:1041B00066696C616D656E742066726F6D207468DF
:1041C0006520202073706F6F6C207468726F756744
:1041D00068207468652020207475626520756E748F
:1041E000696C2069742E2E2E20202020006E6F7A9C
:1041F0007A6C652077696C6C2067657420686F74D1
:10420000215768696C652049276D2068656174696C
:104210006E672C202072656D6F766520746865204E
:1042200066696C616D656E74207475626520667276
:104230006F6D207468652E2E2E20202020004927C7
:104240006D2068656174696E67207570206D7920D6
:104250002020657874727564657220736F207765AD
:104260002063616E20206C6F616420746865206635
:10427000696C616D656E742E2020426520636172E9
:104280006566756C2C207468652E2E2E2020006EBD
:104290006F7A7A6C652077696C6C2067657420682A
:1042A0006F74215768696C652049276D20686561C6
:1042B00074696E672C202072656D6F766520746856
:1042C000652066696C616D656E7420747562652029
:1042D00066726F6D207468652E2E2E2020202000BF
:1042E00049276D2068656174696E67207570206D5F
:1042F000792020207269676874206578747275640B
:10430000657220736F20776563616E206C6F6164E6
:104310002066696C616D656E742E20204265206395
:1043200061726566756C2C207468652E2E2E2020B7
:10433000004D7920657874727564657273206172BE
:1043400065202020206E6F742068656174696E6737
:104350002075702E2020202020436865636B206D1F
:1043600079202020202020202020202020636F6E14
:104370006E656374696F6E732120202020202020D9
:104380002000592041786973204C696E65005820DF
:1043900041786973204C696E65005965732020204F
:1043A000004E6F2020202000446F6E652100536571
:1043B0006C6563742062657374206C696E65732E1E
:1043C000004772656174212020492776652073615A
:1043D00076656420207468657365207365747469FC
:1043E0006E677320616E64202049276C6C207573A2
:1043F00065207468656D20746F202020206D616BCE
:1044000065206E696365206D6F64656C7321202083
:1044100020006C696E65206F6E6520697320657879
:104420007472612020206C6F6E672E2054686520A6
:10443000592061786973207365746973206C6566AF
:1044400074206F6E2074686520706C617465616E95
:1044500064205820617869732069732072696768E5
:10446000742E004C6F6F6B20666F7220746865202D
:10447000626573742020206D617463686564206CCC
:10448000696E6520696E2065616368617869732073
:104490007365742E204C696E657320617265206EA1
:1044A000756D626572656420312D313320616E64F3
:1044B0002E2E2E0049276D20676F696E6720746F5E
:1044C000206D616B652020206120736572696573C2
:1044D000206F66206C696E657320736F776520634B
:1044E000616E2066696E64206D7920202020202076
:1044F0006E6F7A7A6C6520616C69676E6D656E743B
:104500002E202020005765276C6C20676F20746F69
:1045100020746865206D61696E6D656E752E204929
:104520006620796F75206E65656420202068656C53
:104530007020676F20746F3A2020202020202020D8
:10454000206D616B6572626F742E636F6D2F68658D
:104550006C7020202000417765736F6D65212020ED
:10456000202020202020202020205765276C6C2030
:10457000676F20746F207468652053442020636146
:104580007264206D656E7520616E6420796F752090
:10459000202063616E2073656C6563742061206DFB
:1045A0006F64656C2120005765276C6C206B656516
:1045B0007020676F696E6720202020616E64206C18
:1045C0006F616420736F6D6520202020202020669D
:1045D000696C616D656E742C466F722068656C70D5
:1045E00020676F746F206D616B6572626F742E63EC
:1045F0006F6D2F68656C70005765276C6C20747246
:104600007920616761696E212020202020202020F0
:10461000202020202020202020202020202020209A
:10462000202020202020202020202020202020208A
:10463000202020202020202020202020202020207A
:10464000202020202020202000416161682C20743F
:10465000686174206665656C73202020206D756329
:1046600068206265747465722E202020202020202E
:10467000204C6574277320676F206F6E20616E6415
:10468000206C6F6164736F6D652066696C616D6528
:104690006E742120202020202000736F2069742751
:1046A00073206E69636520616E64202020206C6534
:1046B00076656C2E20497427732070726F62616278
:1046C0006C796120626974206F66662066726F6D16
:1046D0002020202020207368697070696E672E2E5C
:1046E0002E202020202020202020004F7572206EB8
:1046F0006578742073746570732077696C6C2067BB
:104700006574206D652073657420757021202020EC
:1047100020202046697273742C207765276C6C20EA
:10472000726573746F72656D79206275696C64204F
:10473000706C6174666F726D2E2E2E004120736F47
:104740006C696420274D27206D65616E73202020E1
:1047500049276D20776F726B696E6720616E6420E8
:1047600077696C6C757064617465206D7920737401
:1047700061747573202020207768656E2049276D4D
:104780002066696E69736865642E2E2E0041206272
:104790006C696E6B696E6720274D27206D65616EB1
:1047A0007349276D2077616974696E6720616E6453
:1047B0002077696C6C636F6E74696E7565207768BD
:1047C000656E20796F752020207072657373207478
:1047D000686520627574746F6E2E2E2E20005765EA
:1047E0006C636F6D65212049276D202020202020DB
:1047F0002020546865205265706C696361746F7223
:104800002032582E20205072657373207468652002
:10481000726564204D20746F202067657420737466
:104820006172746564212020202020202020004512
:104830007874727564657200506C6174666F726D25
:10484000004C65667420546F6F6C00526967687421
:1048500020546F6F6C00436F6F6C21005374617252
:1048600074205072656865617421004669726D77C5
:104870006172652056657273696F6E20372E200055
:104880002020202020202020202020202020202028
:10489000202020200020202D2D2D2D2D2D2D2D2DC3
:1048A0002D2D2D2D2D2020202000205468652052F4
:1048B00065706C696361746F72203258202000202B
:1048C00020202020202020202020202020202020E8
:1048D00020202000202020002D2D3E0043202020DD
:1048E00020002F20202043004E4120004F4646004C
:1048F0004F4E200020F9C9FFE0FCE7FFF8FF000061
:1049000000000000080000002003190040063200EB
:1049100060094B00000A5000800C64000010800009
:10492000D0FEC0FF18FFD0FF63FFE0FFB1FFF0FF34
:104930000000000051001000A4002000F80030002A
:1049400040014000A2015000F70160004B027000DE
:104950009F028000F20290004503A0009703B00080
:10496000E803C0003A04D0008C04E000DF04F0004B
:104970003205000186051001DB0520012F063001FC
:10498000DA0650013007600186077001DC078001FC
:104990006808900101009403360009016B00D800FB
:1049A000A000BD00D500AB000A019D003F018400BE
:1049B00074017C00A9017400DE016D001302660021
:1049C000480260007D025900B2025200E7024B002B
:1049D0001C03440051033A0086033000BB0322004D
:1049E000F0030200303457344838B141344215489E
:1049F000674ED2513053EC658D7691799984CA8592
:104A0000E986CA878C89BB89818B2797D397949B2A
:104A1000239C0C9DC39DEA9EF0A33CA420A8D4AB8C
:104A200044CCD7CD56CF9FD054D130D211241FBE05
:104A3000CFEFD1E2DEBFCDBF15E0A0E0B2E0E4ED04
:104A4000F2EB01E00BBF02C007900D92AE3BB10745
:104A5000D9F72DE1AEEBB5E001C01D92A137B20749
:104A6000E1F719E4CCE2DAE400E006C0229701099C
:104A7000FE010BBF0E9429D8C43ED10780E0080781
:104A8000A9F70E9401420C9468D90C9400006BBFF6
:104A9000FA01DC0102C007900D9221503040D8F796
:104AA0000895F89420910206309103068091000643
:104AB00090910106821B930B789408958093F905D9
:104AC000089581E08093F70508958091F905089590
:104AD0008091F8050895209102063091030681E047
:104AE000232B09F080E0089510920306109202062D
:104AF00010920506109204061092080610920906FC
:104B00001092FB051092FC051092FD051092FE0517
:104B10001092FA051092F9051092F8051092F2051C
:104B20001092F3051092F4051092F5051092DD0530
:104B30001092F1051092F0051092EF05089581E0B2
:104B40002091EF053091F0052630310509F080E025
:104B500008956091FB057091FC058091FD05909191
:104B6000FE0508951092FB051092FC051092FD05BC
:104B70001092FE0508954F925F926F927F928F92EE
:104B80009F92AF92BF92CF92DF92EF92FF920F93DC
:104B90001F93CF93DF93CDB7DEB7CC55D1090FB6B6
:104BA000F894DEBF0FBECDBFCE01CD960E94C37B71
:104BB00084E1FE01FD96A1ECB5E001900D928A958D
:104BC000E1F745E06DE97AE1CE0101960E94F4CE6D
:104BD000CE0101960E9436CF8093C00564E070E05C
:104BE00081EC95E00E94C64EDC016D917D918D9126
:104BF0009C910E94BBD42B013C0184E00E94197956
:104C00009B01AC0163E070E081EC95E06A962FAF08
:104C10006A976B963FAF6B976C964FAF6C976D969C
:104C20005FAF6D970E94C64EFC0180809180A2808C
:104C3000B38083E00E94197965966CAF7DAF8EAF2B
:104C40009FAF659762E070E081EC95E00E94C64EF0
:104C5000DC01CD90DD90ED90FC9061E070E081ECA6
:104C600095E00E94C64EDC018D919D910D90BC9106
:104C7000A02D69968CAF9DAFAEAFBFAF699760E0D6
:104C800070E081EC95E00E94C64E8C0165966CAD9B
:104C90007DAD8EAD9FAD65970E948DD4860E971E1B
:104CA000A81EB91ED8018D919D910D90BC91A02D8B
:104CB00065968CAF9DAFAEAFBFAF65976A962FADCF
:104CC0006A976B963FAD6B976C964FAD6C976D96F0
:104CD0005FAD6D97C301B2010E946BD30E9488D46F
:104CE0009F938F937F936F9369960CAD1DAD2EADFF
:104CF0003FAD699765964CAD5DAD6EAD7FAD659787
:104D0000CE0189960E948B4E48E052E060E070E050
:104D1000CE0189960E94547C8DE499E00E94E0A126
:104D20009093D8058093D7058CEE99E00E94E0A17E
:104D30009093DA058093D9058CE29CE00E94E0A173
:104D40009093D6058093D5050F900F900F900F90FC
:104D50008091F605882391F060E070E08DE499E0A1
:104D60000E940EA160E070E08CEE99E00E940EA11E
:104D700060E070E08CE29CE00E940EA184E1FE0104
:104D8000B996DE01559601900D928A95E1F762E0A1
:104D900070E0CE0145960E94C64E8C0182E00E94D2
:104DA00019790E9488D49B01AC01A6E9B0E00E9469
:104DB000C3D6F801608371838283938384E1FE010B
:104DC0007596DE01119601900D928A95E1F760E0EB
:104DD00070E0CE0101960E94C64E8C0180E00E94D8
:104DE000197920E030E04DED52EC0E94BFD50E94D1
:104DF00088D4D8016D937D938D939C93139761E034
:104E000070E0CE0101960E94C64E8C0181E00E94A6
:104E1000197920E030E044E952EC0E94BFD50E94AD
:104E200088D4F80160837183828393834CE850E0D7
:104E300060E070E0CE0145960E94547C42E850E06C
:104E400060E070E0CE0101960E94547C60E087ED46
:104E500098E00E94BB46C45ADF4F0FB6F894DEBFFD
:104E60000FBECDBFDF91CF911F910F91FF90EF90BB
:104E7000DF90CF90BF90AF909F908F907F906F907A
:104E80005F904F9008950F931F93CF93DF93CDB70B
:104E9000DEB764970FB6F894DEBF0FBECDBFCE016C
:104EA00001960E94C37B63E070E0CE0101960E94F0
:104EB000C64E8C0163E070E081EC95E00E94C64E26
:104EC000FC014081518162817381F80140835183EB
:104ED0006283738364E070E0CE0101960E94C64E47
:104EE0008C0164E070E081EC95E00E94C64EFC010C
:104EF0004081518162817381F801408351836283D3
:104F00007383CE0101960E944E7A62E070E0CE017A
:104F100001960E94C64E8C0162E070E081EC95E043
:104F20000E94C64EFC014081518162817381F8016B
:104F300040835183628373834CE850E060E070E00B
:104F4000CE0101960E94547C42E850E060E070E09F
:104F500081EC95E00E94547C6091C00587ED98E05B
:104F60000E94BB4664960FB6F894DEBF0FBECDBF5D
:104F7000DF91CF911F910F9108956091D7057091A6
:104F8000D8058DE499E00E940EA16091D905709139
:104F9000DA058CEE99E00E940EA16091D505709122
:104FA000D6058CE29CE00E940EA18CE29CE00E945F
:104FB000F3A1882319F18CE29CE00E940DA28111DB
:104FC0001DC08DE499E00E940DA2811108C061E02E
:104FD0008DE499E00E943EA281E08093FA058CEE78
:104FE00099E00E940DA2811109C061E08CEE99E068
:104FF0000E943EA281E08093FA0508950895CF9320
:10500000DF93EB0170930502609304029091F80521
:10501000981709F44BC0882329F1209781F481E087
:105020008093F60562E774E081EE9AE00E9458A54D
:1050300081E090E09093DC058093DB050FC0613048
:10504000710561F41092F6056DE375E081EE9AE06A
:105050000E9458A5D093DC05C093DB0581E08093C6
:10506000F80524C08091DB059091DC058130910525
:1050700029F41092DC051092DB0516C082309105F0
:1050800029F40E94BD2784E090E006C0039749F40C
:105090000E94BD2785E090E09093DC058093DB05BE
:1050A00005C06230710511F41092F805DF91CF91BF
:1050B0000895CF93FC01C62F828193816081718115
:1050C0008617970798F44281538184819581840FD4
:1050D000951F0E943ED6A681B781A80FB91FCC9319
:1050E0008281938101969383828302C081E08087CD
:1050F000CF910895682F80E096E00C945928CF93C3
:10510000DF93FC0182819381892B21F481E08187E7
:1051100080E019C08481958120813181B9010E948C
:105120003ED6C681D781C80FD91F8481958101964B
:10513000B9010E943ED69583848382819381019731
:10514000938382838881DF91CF91089580E096E0F8
:105150000C947F28CF9380E096E00E947F28C82F90
:1051600080E096E00E947F28982F8C2FCF910895A1
:105170001F93CF93DF9300D0CDB7DEB780E096E0EA
:105180000E947F28682F80E096E06A830E947F2833
:10519000782F80E096E079830E947F28182F80E0A6
:1051A00096E00E947F28982F6A817981812F0F9045
:1051B0000F90DF91CF911F910895CF93DF930E94BD
:1051C000A628C82F0E94A628D82F0E94A6284D2FB7
:1051D00050E0FA013397ED31F10508F0B1C0EE5817
:1051E000FF4F0C94A7D68091BF058823A1F08DE4D2
:1051F00099E00E941EA08CEE99E00E941EA0809172
:10520000BE05811104C08CE29CE00E941EA0109299
:10521000BE051092BF050E94AA28BC01C13019F436
:1052200084EE99E002C085E499E008960E940EA100
:105230008CE29CE00E94F3A1882309F48CC08CE2EC
:105240009CE00E940DA2811186C0C13019F484EE49
:1052500099E002C085E499E008960E940DA28111B0
:105260007AC070C09091F90581E089270E94403C86
:105270000DC00E94A628682F6170C13019F484EE19
:1052800099E002C085E499E00E945A87C1E090C08D
:105290000E94A628682F617087ED98E00E94BB46A7
:1052A000F5CF61E087ED98E00E94B6468091BF059A
:1052B000882319F081E08093BE050E94AA28BC01D2
:1052C0008CE29CE00E940EA18CE29CE00E940DA268
:1052D000C1E0C827C093FA056C2F8DE499E00E94C5
:1052E0003EA26C2F8CEE99E00E943EA240E061E06D
:1052F00070E087ED98E00E9479440E94EC36C82F58
:10530000811156C00E94CA3B059741F021E040E060
:1053100063EB72E087ED98E00E94574460E070E034
:105320008CE29CE00E940EA160E087ED98E00E9474
:10533000B646ACCF0E94B828A9CF0E94A628A6CF17
:10534000C0E036C081E08093FA05C13059F584EEA3
:1053500099E061E005C0C13041F584EE99E060E07C
:1053600008960E943EA240E061E070E087ED98E080
:105370000E947944C13009F089CF0E94FF35C82FBF
:10538000882309F483CF21E040E062E672E087EDF4
:1053900098E00E94574460E070E08CEE99E00E9433
:1053A0000EA106C085E499E0D4CF85E499E0D7CF7B
:1053B0008C2FDF91CF9108952F923F924F925F9261
:1053C0006F927F928F929F92AF92BF92CF92DF9215
:1053D000EF92FF920F931F93CF93DF93CDB7DEB77A
:1053E000A8970FB6F894DEBF0FBECDBF0E94455000
:1053F000882309F487C080910206909103062091CA
:105400000006309101062817390721F00E94B35099
:105410008111D9C50E94B3508111F0C5C090F20529
:10542000D090F305E090F405F090F5050E94F34F5D
:10543000C616D706E806F90608F0E0C58091DD0536
:105440008111DCC58091F1058F5F8093F105863075
:1054500008F458C081EE9AE00E948CA421E040E05C
:105460006AE775E087ED98E00E94574481E08093F9
:10547000DD050E94548410920306109202061092D9
:10548000050610920406109208061092090660E0C4
:1054900070E08DE499E00E940EA160E070E08CEE77
:1054A00099E00E940EA160E070E08CE29CE00E9416
:1054B0000EA1CE0101960E942F7B62E070E0CE012A
:1054C00001960E94C64E8C0182E00E94197920E06C
:1054D00030E046E153E40E94BFD50E9488D4F80131
:1054E00060837183828393831092F90546E950E0CB
:1054F00060E070E0CE0101960E94547C0E94C5508D
:105500001092F1050E944A858823D1F0809102060D
:105510009091030620910006309101062817390763
:1055200021F00E945385811188C50E945385811105
:1055300007C08091020690910306892B09F473C578
:105540008091FA05882391F08CE29CE00E94BEA134
:10555000882361F060E08DE499E00E943EA260E063
:105560008CEE99E00E943EA21092FA058091F90516
:1055700081110C9417348091F70581110C94173424
:105580008091EF059091F005039781F40E94AA792C
:10559000882341F080EE95E00E94CED0882331F040
:1055A0000E9454841092F0051092EF058091EF054F
:1055B0009091F005019741F40E94AA79811104C0ED
:1055C0001092F0051092EF058091EF059091F00593
:1055D000029751F480EE95E00E94CED0882321F00E
:1055E0001092F0051092EF058091EF059091F00573
:1055F0000497C1F580EE95E00E94CED0882349F053
:1056000021E040E064E073E087ED98E00E945744B9
:1056100032C58091FF05813019F484EE99E002C013
:1056200085E499E008960E94BEA12091FF05882399
:1056300071F0213019F484EE99E002C085E499E01C
:10564000FC01E258FF4F8081882309F411C5213005
:1056500009F40BC585E499E008960E94F3A188231C
:1056600009F4F3C48091EF059091F0050597F9F4E2
:1056700080EE95E00E94CED0882349F021E040E002
:1056800061E473E087ED98E00E9457440CC08CE21F
:105690009CE00E94F3A1882331F08CE29CE00E9400
:1056A000BEA1882321F01092F0051092EF058091A1
:1056B000EF059091F005069709F03FC080EE95E068
:1056C0000E94CED08823B1F08091DE0581FF06C014
:1056D00060E087ED98E00E9434472FC01092F005FB
:1056E0001092EF0540E060E170E087ED98E00E94E5
:1056F000794423C081EE9AE00E9418A88823E9F03B
:105700008091DE0582FF04C081EE9AE00E94E7A549
:1057100040E050E060E070E087ED98E00E945D4579
:1057200040E060E170E087ED98E00E9479440E94DB
:1057300031881092F0051092EF058091EF0590915D
:10574000F005892B09F024C48091F805882361F0C5
:105750008091DB059091DC05019709F091C40E94CE
:10576000BB64811198C48CC4809102069091030699
:10577000892B09F40DC487ED98E00E94DF448091E5
:1057800004069091050660910006709101060E9442
:105790003ED6E0910606F0910706E80FF91F10814A
:1057A0001B3809F46BC01E3809F420C61B3909F4F4
:1057B000ADC5193809F47AC6163909F4CAC01638C5
:1057C00011F40C94F3331C3809F045C080910206A3
:1057D00090910306459708F4DBC30E94A6280E9417
:1057E000B8282B013C010E94B828698F7A8F8B8FD3
:1057F0009C8F0E94B8286B017C010E94B8284B0145
:105800005C010E94B8289B014091FB055091FC056A
:105810006091FD057091FE054F5F5F4F6F4F7F4FA9
:105820004093FB055093FC056093FD057093FE05C6
:105830009F938F933F932F93098D1A8D2B8D3C8DC2
:10584000B301A201CE0101960E948B4ECE010196BA
:105850000E944E7A6DC01C3909F47BC0103909F4DE
:1058600078C08DE7810F823008F473C0183809F4CE
:1058700070C00E94BB64811160C0D9C780910206CC
:1058800090910306499708F483C387ED98E00E943E
:10589000DF440E94A62881E090E09093F005809379
:1058A000EF050E94B828698F7A8F8B8F9C8F0E949A
:1058B000B8286D8F7E8F8F8F98A30E94B8286B01B8
:1058C0007C010E94B8284B015C010E94B828162F69
:1058D000072F382E292E0E94B8282B013C018091D9
:1058E000FB059091FC05A091FD05B091FE05019688
:1058F000A11DB11D8093FB059093FC05A093FD05B0
:10590000B093FE052F923F920F931F930D8D1E8D26
:105910002F8D38A1498D5A8D6B8D7C8DCE010196CE
:105920000E948B4EB301A201CE0101960E94547CCD
:105930000F900F900F900F902BC31D3909F4F5C5F0
:10594000153809F43FC6143909F465C6153909F448
:10595000A9C68DE7810F823008F043C0809102060E
:1059600090910306089708F413C30E94A6280E948A
:10597000A628082F0E94B8286B017C010E94AA2843
:10598000DC014091FB055091FC056091FD05709193
:10599000FE054F5F5F4F6F4F7F4F4093FB05509366
:1059A000FC056093FD057093FE0583E090E0909305
:1059B000F0058093EF0520E432E44FE050E00E94D0
:1059C000C3D6AB01BC0180EE95E00E94AAD081E075
:1059D000143809F080E0A7019601602F0E94F77F3C
:1059E000D7C2173851F480910206909103060697AA
:1059F00008F4CEC284E090E00BC01D38C9F5809158
:105A0000020690910306069708F4C2C285E090E072
:105A10009093F0058093EF050E94A6280E94A62887
:105A20008093FF050E94AA280E94AA284091FB05A6
:105A30005091FC056091FD057091FE054F5F5F4F31
:105A40006F4F7F4F4093FB055093FC056093FD051E
:105A50007093FE05DC0120E432E44FE050E00E9448
:105A6000C3D6AB01BC0180EE95E00E94AAD090C2E3
:105A70001F3809F06EC080910206909103060297CC
:105A800008F486C20E94A6280E94A6284091FB0521
:105A90005091FC056091FD057091FE054F5F5F4FD1
:105AA0006F4F7F4F4093FB055093FC056093FD05BE
:105AB0007093FE0594E2E92E92E0F92E00E010E0EA
:105AC000C82ED12C28EE822E23E0922EA12CB12CB0
:105AD000C601002E02C0959587950A94E2F780FFD3
:105AE0002EC0CE0101960E94C37BB801CE01019663
:105AF0000E94BF4EFC0160817181828193816D8B18
:105B00007E8B8F8B988F402F0E94247920E030E08D
:105B10004AE754E40E94BFD50E9488D4A5019401AD
:105B20000E9488D62D8B3E8B4F8B588FF89444E083
:105B300050E0B701CE0145960E943BD978940F5FA3
:105B40001F4FF4E0EF0EF11C0530110509F0C0CF36
:105B50001FC2103909F068C08091020690910306B7
:105B6000029708F415C20E94A6280E94A628A82E13
:105B70004091FB055091FC056091FD057091FE057B
:105B80004F5F5F4F6F4F7F4F4093FB055093FC0576
:105B90006093FD057093FE05CE0101967C010E9485
:105BA000C37B84E2C82E82E0D82E00E010E0B12C46
:105BB0007E2C6F2CC501002E02C0959587950A9406
:105BC000E2F780FF25C0F894B801C7010E94C64ED5
:105BD00044E050E0B6010E9425D97894B801872DA1
:105BE000962D0E94C64E4C01B801872D962D0E941D
:105BF000C64EFC0160817181828193810E94BBD479
:105C0000402F0E943D79F4016083718382839383E6
:105C10000F5F1F4FF4E0CF0ED11C0530110551F678
:105C2000C7010E94D27AB4C1113939F580910206B8
:105C300090910306039708F4ABC10E94A6280E9426
:105C4000A628182F0E94A6284091FB055091FC051C
:105C50006091FD057091FE054F5F5F4F6F4F7F4F65
:105C60004093FB055093FC056093FD057093FE0582
:105C7000682F812F0E94A2808BC11239A9F58091D3
:105C8000020690910306069708F482C10E94A62896
:105C90000E94A628182F0E94A62888A70E94A6283E
:105CA0008FA30E94A628082F0E94A628C090FB055B
:105CB000D090FC05E090FD05F090FE052FEFC21A94
:105CC000D20AE20AF20AC092FB05D092FC05E092E9
:105CD000FD05F092FE05802F0E94D8884FA168A58F
:105CE000812F0E947B8954C1133951F5809102069E
:105CF00090910306069708F44BC10E94A6280E94C3
:105D0000AA288C010E94AA287C010E94A628409102
:105D1000FB055091FC056091FD057091FE054F5FFC
:105D20005F4F6F4F7F4F4093FB055093FC0560938F
:105D3000FD057093FE05B701C8010E94CB4D28C137
:105D40001838D9F58091020690910306049708F45B
:105D50001FC18091040690910506209102063091A2
:105D60000306039660910006709101060E943ED6DC
:105D7000E0910606F0910706E80FF91F808190E098
:105D800004962817390708F403C10E94A6288091B9
:105D9000FB059091FC05A091FD05B091FE050196D3
:105DA000A11DB11D8093FB059093FC05A093FD05FB
:105DB000B093FE050E94DD28EBC0163931F58091C5
:105DC000020690910306039708F4E2C00E94A628F9
:105DD0000E94A628182F0E94A6284091FB055091EA
:105DE000FC056091FD057091FE054F5F5F4F6F4FA1
:105DF0007F4F4093FB055093FC056093FD05709326
:105E0000FE05812F0E941CA4C3C0173911F5809193
:105E1000020690910306029708F4BAC00E94A628D1
:105E20000E94A6284091FB055091FC056091FD055C
:105E30007091FE054F5F5F4F6F4F7F4F4093FB05A3
:105E40005093FC056093FD057093FE050E942C4E57
:105E50009FC0183931F58091020690910306029790
:105E600008F496C00E94A6280E94A6288091FB05EF
:105E70009091FC05A091FD05B091FE050196A11D34
:105E8000B11D8093FB059093FC05A093FD05B09395
:105E9000FE050E94473660E087ED98E00E94344797
:105EA00077C0193951F58091020690910306059744
:105EB00008F46EC00E94A6280E94B8288091FB05B5
:105EC0009091FC05A091FD05B091FE050196A11DE4
:105ED000B11D8093FB059093FC05A093FD05B09345
:105EE000FE0580E096E00E943D4181E08093BF0581
:105EF00087ED98E00E94F0444BC01A3911F580916B
:105F0000020690910306029708F442C00E94A62858
:105F10000E94A6284091FB055091FC056091FD056B
:105F20007091FE054F5F5F4F6F4F7F4F4093FB05B2
:105F30005093FC056093FD057093FE050E944E3D55
:105F400027C01C3929F5809102069091030602971B
:105F5000F8F00E94A6280E94A6284091FB055091C7
:105F6000FC056091FD057091FE054F5F5F4F6F4F1F
:105F70007F4F4093FB055093FC056093FD057093A4
:105F8000FE0591E0813009F090E0892F0E94AD80FC
:105F90008091FB059091FC05A091FD05B091FE0557
:105FA00081309A4CAA49BB4308F441C481E09AEC81
:105FB000AAE9BBE38093FB059093FC05A093FD0544
:105FC000B093FE0534C48091F2059091F305A09141
:105FD000F405B091F5050196A11DB11D8093F20560
:105FE0009093F305A093F405B093F5050E94B65085
:105FF000682F80E096E00E945928FDC90E94B350A6
:10600000811180CA8091020690910306892B09F0C4
:1060100079CA8091EF059091F005892B09F072CA39
:106020000E94C5506FCA8091EF059091F005892BB1
:1060300009F086CA0E94C48583CA0E946185682FC0
:1060400080E096E00E94592861CA8091FF05813066
:1060500019F484EE99E002C085E499E0FC01E2586D
:10606000FF4F8081882339F0FDCA84EE99E0F4CA9D
:1060700087E00E942C4E1092F0051092EF05F2CAB4
:106080008091DB059091DC050297D9F40E94BB64F6
:10609000811195C016C0809104029091050200976D
:1060A00019F461E274E004C0019731F460E075E036
:1060B00081EE9AE00E9458A50E94BB2582E090E004
:1060C00028C08091DB059091DC058330910531F18A
:1060D000049709F46FC08091DB059091DC05853051
:1060E000910509F4D3C08630910509F099C010924A
:1060F000FF0584E090E09093F0058093EF0540E089
:1061000052ED69E47BE680EE95E00E94AAD087E03C
:1061100090E09093DC058093DB0589C380910402B5
:1061200090910502019709F082C380EE95E00E94EC
:10613000CED0882309F47BC3CE0101960E94A6D05D
:106140008FE0FE013196A0EEB5E001900D928A95A8
:10615000E1F710920502109204020E942FA421E0A0
:1061600040E06FEA74E087ED98E00E94574464E1F4
:1061700080E00E94A28064E181E00E94A28064E14C
:1061800083E00E94A28064E184E00E94A28060E03B
:1061900070E08DE499E00E940EA160E070E08CEE6A
:1061A00099E00E940EA160E070E08CE29CE00E9409
:1061B0000EA13DC30E94BB64811168C08CCF0E94B8
:1061C0002FA483E090E09093DC058093DB05809121
:1061D000040290910502019759F440E059EE64EAF7
:1061E00075E380EE95E00E94AAD086E00E942C4ED6
:1061F0008091040290910502892B09F018C364E193
:1062000080E00E94A28064E181E00E94A28064E1BB
:1062100083E00E94A28064E184E00E94A28007C320
:1062200087309105A1F481E08093FF0584E090E040
:106230009093F0058093EF0540E052ED69E47BE632
:1062400080EE95E00E94AAD088E090E062CF88308E
:10625000910549F487ED98E00E94B0440E944327DD
:1062600089E090E056CF099709F0E1C20E94BB6433
:10627000882309F4DCC281EE9AE00E946BA610929A
:10628000DC051092DB051092F805D1C28091040262
:1062900090910502019741F06FE780E00E94A28093
:1062A0006FE781E00E94A280809104029091050234
:1062B000892B41F46FE783E00E94A2806FE784E0BE
:1062C0000E94A2806CE074E081EE9AE00E9458A5E2
:1062D0001092FF0585E090E09093F0058093EF0524
:1062E00040E052ED69E47BE680EE95E00E94AAD0A2
:1062F00086E090E09093DC058093DB0524E140E0AC
:1063000063E087ED98E00E94A24491C2809102066A
:1063100090910306809708F43BCE87ED98E00E94A9
:10632000DF440E94A62881E090E09093F0058093DE
:10633000EF050E94B828698F7A8F8B8F9C8F0E94FF
:10634000B8286D8F7E8F8F8F98A30E94B8286B011D
:106350007C010E94B8284B015C010E94B828162FCE
:10636000072F282E9FA30E94B8282B013C010E94D2
:10637000A628382E0E94B82869A37AA38BA39CA3D1
:106380000E94AA289EA38DA38091FB059091FC05F5
:10639000A091FD05B091FE050196A11DB11D809350
:1063A000FB059093FC05A093FD05B093FE052FA17E
:1063B0002F932F920F931F930D8D1E8D2F8D38A12C
:1063C000498D5A8D6B8D7C8DCE0101960E948B4E2E
:1063D000CDA0DEA0E9A0FAA00BA11CA1232DB30142
:1063E000A201CE0101960E94547EA2CA80910206AB
:1063F000909103064A9708F4CBCD87ED98E00E9470
:10640000DF440E94A62881E090E09093F0058093FD
:10641000EF050E94B828698F7A8F8B8F9C8F0E941E
:10642000B8286D8F7E8F8F8F98A30E94B8286B013C
:106430007C010E94B8284B015C010E94B828162FED
:10644000072F282E9FA30E94B8282B013C010E94F1
:10645000A628382E8091FB059091FC05A091FD05A2
:10646000B091FE050196A11DB11D8093FB0590938F
:10647000FC05A093FD05B093FE052FA12F932F924D
:106480000F931F930D8D1E8D2F8D38A1498D5A8D21
:106490006B8D7C8DCE0101960E948B4E232DB30116
:1064A000A201CE0101960E94447D42CA809102065B
:1064B00090910306029708F46BCD0E94A6280E94D3
:1064C000A628E82E4091FB055091FC056091FD0542
:1064D0007091FE054F5F5F4F6F4F7F4F4093FB05FD
:1064E0005093FC056093FD057093FE050E94BB640C
:1064F000882309F44DCDDE2CDD1CDD24DD1C00E0FD
:1065000010E0F12CC701002E02C0959587950A94E2
:10651000E2F780FF04C06D2D802F0E9489800F5FFD
:106520001F4F0530110571F733CD80910206909110
:1065300003060B9708F42CCD0E94A6280E94A628DB
:10654000182F0E94A628282F30E0F4E61F9F200D68
:10655000311D11242436310541F021E040E06BEB80
:1065600073E087ED98E00E9457440E94A6280E949D
:10657000B8280E94AA288531904B41F020E040E0E5
:106580006EE773E087ED98E00E9457440E94AA28C6
:106590000E94B8280E94B8280E94A6288091FB0576
:1065A0009091FC05A091FD05B091FE050196A11DFD
:1065B000B11D8093FB059093FC05A093FD05B0935E
:1065C000FE05E6CC8091020690910306059708F43B
:1065D000DFCC82E090E09093F0058093EF050E947D
:1065E000A6280E94B8289B01AC018091FB059091E0
:1065F000FC05A091FD05B091FE050196A11DB11D00
:106600008093FB059093FC05A093FD05B093FE05D8
:10661000A8EEB3E024CA8091020690910306059784
:1066200008F4B6CC0E94A6280E94A6288093DF0515
:106630000E94AA288C010E94A6288093DE05409122
:10664000FB055091FC056091FD057091FE054F5FC3
:106650005F4F6F4F7F4F4093FB055093FC05609356
:10666000FD057093FE050115110571F0D80120E4B8
:1066700032E44FE050E00E94C3D6AB01BC0180EE93
:1066800095E00E94AAD093C0CE0101960E94A6D0A8
:106690008FE0FE013196A0EEB5E001900D928A9553
:1066A000E1F785C081EE9AE00E94ADA48C01809153
:1066B000020690910306069708F46ACC0E94A62869
:1066C0000E94A628E82E0E94A628C82E0E94A6286E
:1066D000D82E0E94A628F82E4091FB055091FC056B
:1066E0006091FD057091FE054F5F5F4F6F4F7F4FCB
:1066F0004093FB055093FC056093FD057093FE05E8
:10670000E0FC03C0C8010E9448C8F801C282D382DD
:1067100060E076E0C8010E940BCCE1FE39CCE0914C
:10672000100CEE0FFF0BEE5FF34F2081318120172D
:10673000310731F0B80181EE9AE00E94C6A403C08F
:10674000C8010E948DC88E2D8470FF2039F0811100
:1067500005C06F2DC8010E947DC81ACC882309F49A
:1067600017CCFF2079F0AF2DB0E020E432E44FE009
:1067700050E00E94C3D6AB01BC0180EE95E00E94C0
:10678000AAD00DC0CE0101960E94A6D08FE0FE01D6
:106790003196A0EEB5E001900D928A95E1F784E084
:1067A0008093DF058091DE0584708093DE054FE0E5
:1067B00050E069E170E087ED98E00E945D456091EE
:1067C000DF0581EE9AE00E9413A841E060E170E0ED
:1067D00087ED98E00E94794486E090E09093F00580
:1067E0008093EF05D5CB8091020690910306029726
:1067F00008F4CECB0E94A6280E94A6288093FF050D
:106800004091FB055091FC056091FD057091FE05DE
:106810004F5F5F4F6F4F7F4F4093FB055093FC05D9
:106820006093FD057093FE050E94B080B1CBA896E1
:106830000FB6F894DEBF0FBECDBFDF91CF911F9191
:106840000F91FF90EF90DF90CF90BF90AF909F900F
:106850008F907F906F905F904F903F902F90089512
:1068600040E063E97AE18AE098E00E94F4CE80E0BB
:1068700092E0909301068093000610920306109216
:10688000020610920506109204068AE096E09093A4
:10689000070680930606109208061092090680EEFD
:1068A00095E00E94A6D081EC95E00C948A4E40E0E1
:1068B00063E97AE186E398E00E94F4CE80E198E013
:1068C0000C9472CECF93DF9300D0CDB7DEB721E02A
:1068D000298322E32A8342E050E0BC01CE010196E5
:1068E0000E943BD90F900F90DF91CF910895CF93E5
:1068F000DF93EC0140E050E060E171E40E94AE9E65
:1069000040E050E060E87EE3CE0102960E94AE9E39
:1069100040E050E060E271E4CE010496DF91CF9157
:106920000C94AE9E0F931F93CF93DF93EB018B01DB
:10693000085E1F4F892B31F467E0CE010E9445D9D4
:106940006CE005C068E3CE010E9445D960E2C80151
:106950000E9445D9CE010A960E947734CE01409616
:106960000E947734CE014A960E94623464EF71E04F
:10697000CE0106960E945BD965E070E0CE010296DA
:106980000E945BD964EF71E0CE0104960E945BD94E
:106990006CE271E0CE010896DF91CF911F910F91CB
:1069A0000C945BD90F931F93CF93DF9300D01F926A
:1069B000CDB7DEB78C0160E00E9445D961E0C80127
:1069C00002960E9445D98FEF89831B821A82B801F3
:1069D0006C5F7F4F43E050E0CE0101960E943BD9AF
:1069E0000F900F900F90DF91CF911F910F9108950D
:1069F000FF920F931F93CF93DF9300D000D0CDB7BA
:106A0000DEB7F82E062F1FB7F89468E080E491E017
:106A10004C830E9445D9F9820A834C814B8343E021
:106A200050E064E471E0CE0101960E943BD91FBFA3
:106A30000F900F900F900F90DF91CF911F910F91BA
:106A4000FF90089561E00C9445D9CF93DF93EC015A
:106A500066EE70E00E945BD966EE70E0CE010296B1
:106A60000E945BD96EE670E0CE0104960E945BD96D
:106A700065E0CE010696DF91CF910C9445D961E097
:106A80008EE691E00E9445D968EE73E082E791E0DE
:106A90000E945BD968EE73E084E791E00E945BD9C5
:106AA00066E970E086E791E00E945BD960EA7FE0EA
:106AB00088E791E00E945BD960EA7FE08AE791E095
:106AC0000E945BD960ED77E080E791E00E945BD99E
:106AD00060EA7FE086E891E00E945BD96AE070E0BE
:106AE0008CE791E00E945BD96AE070E08EE791E06C
:106AF0000E945BD96AE070E080E891E00E945BD977
:106B00006EE170E082E891E00E945BD96EE170E096
:106B100084E891E00E945BD942E553E060E070E0D8
:106B200088ED91E00E9453D944E853E060E070E0C2
:106B30008CED91E00E9453D960E070E080EE91E02E
:106B40000E945BD960E070E082EE91E00E945BD928
:106B500061E084EE91E00E9445D960E888E891E028
:106B60000C9445D9CF93CFB7F89440E150E062E25E
:106B700070E089EF92E00E943BD9CFBFCF9108959A
:106B8000EF92FF920F931F93CF93DF93CDB7DEB7B2
:106B90002D970FB6F894DEBF0FBECDBF8DE0E7E0B6
:106BA000F3E0DE01119601900D928A95E1F7CE0196
:106BB00001967C0102E210E060E0C8010E94009EA4
:106BC000F70121917F0190E0332727FD309582174F
:106BD000930739F40F5F1F4F0E32110569F781E0FB
:106BE00001C080E02D960FB6F894DEBF0FBECDBF7A
:106BF000DF91CF911F910F91FF90EF90089561E089
:106C000082E490E00E94009E91E0813009F090E0E3
:106C1000892F08951F93CF93DF93CDB7DEB7649785
:106C20000FB6F894DEBF0FBECDBF84E1EBEBF2E010
:106C3000DE01119601900D928A95E1F70E94FF35D1
:106C4000882381F088E990E0A0E0B0E089839A830E
:106C5000AB83BC8388E490E0A0E0B0E08D839E83AA
:106C6000AF83B8871FB7F89444E150E064E272E064
:106C7000CE0101960E943BD91FBF64960FB6F894CF
:106C8000DEBF0FBECDBFDF91CF911F9108951F933F
:106C9000CF93DF93CDB7DEB729970FB6F894DEBF59
:106CA0000FBECDBF85E0EFECF2E0DE011196019062
:106CB0000D928A95E1F70E94B2351FB7F89481ECE6
:106CC00093E29F838E8385E190EB9987888745E0E7
:106CD00050E066E070E0CE0101960E943BD96FE97A
:106CE00084E090E00E9445D96BE18CE090E00E9446
:106CF00045D960E084E492E00E9445D90E940A36BA
:106D000060E080E592E00E9445D944E150E060E116
:106D100072E084E193E00E943BD944E150E064EAF0
:106D200071E082E393E00E943BD94AE050E066E4E0
:106D300072E088E293E00E943BD90E943F3560E018
:106D400070E080EA91E00E945BD960E082EA91E025
:106D50000E9445D961E080E691E00E9445D988E52E
:106D600091E00E94253544E050E064E470E0CE01FB
:106D700006960E943BD960E071E080E090E00E94BE
:106D800092346CE171E081E090E00E94923480E402
:106D900091E00E94D2348AE491E00E94223560E0C2
:106DA00086E591E00E9445D91FBF29960FB6F89459
:106DB000DEBF0FBECDBFDF91CF911F910895CF935E
:106DC000CFB7F894682F82E490E00E9445D90E94E2
:106DD0000A36CFBFCF91089561E08CE490E00E9425
:106DE000009E91E0813009F090E0892F0895CF93C3
:106DF000CFB7F89480E491E00E94D2348AE491E025
:106E00000E94223588E591E00E94253561E080E608
:106E100091E00E9445D961E08EE691E00E9445D95B
:106E200081E00E94DF3660E084E492E00E9445D970
:106E300060E080E592E00E9445D960E08CE490E05B
:106E40000E9445D9CFBFCF9108951F93CF93DF9371
:106E5000CDB7DEB72C970FB6F894DEBF0FBECDBF0F
:106E60001FB7F89488EB98E8A0E0B0E089839A8394
:106E7000AB83BC831D821E821F82188619861A86E8
:106E80001B861C864CE050E068E372E0CE01019660
:106E90000E943BD91FBF2C960FB6F894DEBF0FBEE1
:106EA000CDBFDF91CF911F910895FF920F931F9354
:106EB000CF93DF93F82E162F60E070E080EA91E028
:106EC0000E941D9EEC0160E082EA91E00E94009E1B
:106ED000282F210F822F6CE30E9432D6092F2D33E9
:106EE00008F021961FB7F894BE016F0D711D80EA5E
:106EF00091E00E945BD9602F82EA91E00E9445D91F
:106F00001FBFDF91CF911F910F91FF9008951F93A5
:106F1000CF93DF9300D01F92CDB7DEB70E944736E4
:106F200019821A821B821FB7F89467E182E090E011
:106F30000E9445D961E082E490E00E9445D90E9418
:106F4000253760E08CE490E00E9445D961E088E05C
:106F500092E00E9445D943E050E06AE072E0CE0141
:106F600001960E943BD961E78EE092E00E9445D9EC
:106F70001FBF0F900F900F90DF91CF911F91089539
:106F80001F93CF93DF93CDB7DEB727970FB6F89453
:106F9000DEBF0FBECDBF1D821E821F821FB7F894B9
:106FA00044E150E060E172E084E193E00E943BD96B
:106FB00044E150E064EA71E082E393E00E943BD94F
:106FC0004AE050E066E472E088E293E00E943BD938
:106FD0000E943F350E940A3661E088E092E00E94FC
:106FE00045D943E050E06AE072E0CE0105960E9488
:106FF0003BD961E78EE092E00E9445D91FBF40E097
:1070000050E0BA0182E691E00E94409E6C3326E98E
:10701000720721E682072EE99207A8F4A4E6B0E001
:107020009B01AC010E94C3D622E035E847E455E05D
:107030000E9466D628513F474F4F5F4F29833A83BE
:107040004B835C830EC022E035E847E455E00E94A4
:1070500066D6A4E6B0E00E94C3D669837A838B83A8
:107060009C830E9425371FB7F89444E050E068E302
:1070700072E0CE0101960E943BD91FBF27960FB642
:10708000F894DEBF0FBECDBFDF91CF911F91089561
:1070900040E063E97AE18CE398E00C94F4CECF927F
:1070A000DF92EF92FF920F931F93CF93DF93EC0148
:1070B0008B018881811102C080E042C060E0CE0176
:1070C0000E9456CE87FFF8CF0E944850882329F0AF
:1070D000CE010E944B5061E80FC00E9445508111C3
:1070E0000AC00E944A85811106C080915D08909176
:1070F0005E08049731F46AE8C8010E94A9CE81E0D5
:107100001FC0F894C8800E945125D12C8C159D0574
:1071100030F462E8C8010E94A9CE7894F0CFE12C47
:10712000F12CEC14FD0454F46E2DCE010E9456CEC9
:107130000E947A288FEFE81AF80AF3CF61E8EACFC5
:10714000DF91CF911F910F91FF90EF90DF90CF9043
:10715000089586E090E090935E0880935D0881E05A
:10716000809342080895CF93DF93EB0161E00E9482
:107170005BCE61E84A9730F4CE010E94A9CE60E070
:1071800070E005C0CE010E94A9CE62EC72E0CE0193
:10719000DF91CF910C94ABCECF93DF93EB0161E005
:1071A0000E945BCE61E8CE010E94A9CE62EC72E043
:1071B000CE010E94ABCE60E070E0CE010E94ABCE6B
:1071C00061E0CE010E94A9CE60E0CE010E94A9CE6E
:1071D00060E070E0CE01DF91CF910C94ABCEEF92E6
:1071E000FF920F931F93CF93DF938B0161E8C80148
:1071F0000E94A9CECFE5D8E07E016991C8010E9426
:10720000A9CEF7018081882321F0F8E0CE37DF078F
:1072100099F7DF91CF911F910F91FF90EF90089513
:10722000CF93DF93EB0161E8CE010E94A9CE0E94CB
:107230005125AC0160E070E0CE01DF91CF910C945C
:10724000C0CE0F931F93CF93DF93CDB7DEB7649774
:107250000FB6F894DEBF0FBECDBF8B01F894CE0100
:1072600001960E94C37B61E8C8010E94A9CE60E03C
:1072700070E0CE0101960E94BF4EFC014081518119
:1072800062817381C8010E94C0CE61E070E0CE01CE
:1072900001960E94BF4EFC01408151816281738141
:1072A000C8010E94C0CE62E070E0CE0101960E944B
:1072B000BF4EFC014081518162817381C8010E94EF
:1072C000C0CE0E94BF80682FC8010E94A9CE7894CA
:1072D00064960FB6F894DEBF0FBECDBFDF91CF919D
:1072E0001F910F9108950F931F93CF93DF93CDB705
:1072F000DEB764970FB6F894DEBF0FBECDBF8B012B
:10730000F894CE0101960E94C37B61E8C8010E94F7
:10731000A9CE60E070E0CE0101960E94BF4EFC0154
:107320004081518162817381C8010E94C0CE61E0B9
:1073300070E0CE0101960E94BF4EFC014081518158
:1073400062817381C8010E94C0CE62E070E0CE010C
:1073500001960E94BF4EFC01408151816281738180
:10736000C8010E94C0CE63E070E0CE0101960E9489
:10737000BF4EFC014081518162817381C8010E942E
:10738000C0CE64E070E0CE0101960E94BF4EFC01C9
:107390004081518162817381C8010E94C0CE0E94E8
:1073A000BF80682F70E0C8010E94ABCE78946496CD
:1073B0000FB6F894DEBF0FBECDBFDF91CF911F9106
:1073C0000F9108950F931F93CF93DF938C01EB01DF
:1073D00061E8CE010E94A9CEC80103960E945F51C8
:1073E000682FCE01DF91CF911F910F910C94A9CE00
:1073F000CF93DF93EB0161E8CE010E94A9CE0E94FA
:107400007350AB01BC01CE010E94C0CEDF91CF9181
:107410000C94D650BF92CF92DF92EF92FF920F93CF
:107420001F93CF93DF93CDB7DEB77C018B01CDB631
:10743000DEB661E8C8010E94A9CE61E0C7010E94E2
:1074400056CE882369F00E944D51009749F0682F6D
:10745000C8010E94A9CE60E0C8010E94A9CE34C034
:107460008DB79EB74F970FB6F8949EBF0FBE8DBFD6
:10747000EDB7FEB731967F0140E050E06FE1C70104
:107480000E944A4FF7012081222321F0009711F436
:107490002E3291F3682FC8010E94A9CEB12CF701BA
:1074A00061917F01662339F0C8010E94A9CEB3948F
:1074B000FFE1BF12F4CF60E0C8010E94A9CE0FB671
:1074C000F894DEBE0FBECDBE0FB6F894DEBE0FBE82
:1074D000CDBEDF91CF911F910F91FF90EF90DF9084
:1074E000CF90BF900895CF93DF93EB0161E8CE0179
:1074F0000E94A9CEF8940E94BB64882361F00E9488
:107500006B25882341F061E0CE010E94A9CE7894DA
:10751000DF91CF91089560E0F7CF7F928F929F9295
:10752000AF92BF92CF92DF92EF92FF920F931F9391
:10753000CF93DF93CDB7DEB78C015B018DB69EB6DE
:1075400061E00E945BCE7C0163E0C8010E9456CEE0
:10755000C82ED12C2DB73EB72C193D090FB6F89483
:107560003EBF0FBE2DBF0DB71EB70F5F1F4F7FB6BB
:10757000F894482F50E0B701C8010E9425D97FBE7A
:1075800061E8C5010E94A9CE7801C701801B910B5B
:107590008C159D053CF4F70161917F01C5010E94A6
:1075A000A9CEF3CF0FB6F8949EBE0FBE8DBEDF916D
:1075B000CF911F910F91FF90EF90DF90CF90BF90F0
:1075C000AF909F908F907F9008953F924F925F92DF
:1075D0006F927F928F929F92AF92BF92CF92DF92E3
:1075E000EF92FF920F931F93CF93DF9300D000D0C1
:1075F000CDB7DEB77C016B012DB73EB73C832B8343
:1076000061E00E945BCE5C0163E0C7010E9456CE40
:10761000382E282F30E03A8329838DB79EB7821BFE
:10762000930B0FB6F8949EBF0FBE8DBF0DB71EB75C
:107630000F5F1F4F7FB6F894832C912CA401B501E6
:10764000C8010E9425D97FBE3801412C512C2981C7
:107650003A814216530664F464E0640DC7010E9447
:1076600056CEF30181933F01FFEF4F1A5F0AEFCF30
:10767000FFB6F894A401B501C8010E943BD9FFBE32
:1076800061E8C6010E94A9CE632DC6010E94A9CE61
:107690002B813C810FB6F8943EBF0FBE2DBF0F90DB
:1076A0000F900F900F90DF91CF911F910F91FF904E
:1076B000EF90DF90CF90BF90AF909F908F907F9092
:1076C0006F905F904F903F9008950F931F93CF93CB
:1076D000DF931F92CDB7DEB78B0161E00E9456CEDB
:1076E00080FF04C089830E945484898181FD0E94A7
:1076F000742561E8C8010E94A9CE60E0C8010F901E
:10770000DF91CF911F910F910C94A9CECF93DF936E
:10771000EC0161E80E94A9CE6091AD0CCE01DF9131
:10772000CF910C94A9CE10927E0808950F931F93C9
:10773000CF93DF9380917E08882349F080917E0863
:1077400081111EC0EBECF5E0AEE7B8E010C00EE72B
:1077500018E0C2E2D0E060E0CE010E94009EF80195
:1077600081938F012196C233D105A9F7E7CF849188
:107770008D93319685E0E93DF807C9F710928C08A2
:107780008EE798E0DF91CF911F910F9108958FE5DB
:1077900098E0089580915D0890915E080895CF93D8
:1077A000DF9381EE9AE00E94B8A48FE598E00E94F2
:1077B0009751EC01009789F40E9474250E9454842B
:1077C0000E94848160E087ED98E00E94EB4682E0B1
:1077D00090E090935E0880935D08CE01DF91CF9199
:1077E0000895CF92DF92EF92FF920F931F93CF9362
:1077F000DF938C017B0161E8C7010E94A9CE8FE570
:10780000C82E88E0D82EC1E0D0E0F801808190E059
:10781000C817D9074CF46C2FC8010E9456CEF60148
:1078200081936F012196F1CF10927D080E94CF3B8A
:10783000682FC701DF91CF911F910F91FF90EF90BB
:10784000DF90CF900C94A9CE0E9480858823B9F058
:1078500085E090E090935E0880935D0881EE9AE069
:107860000E94AFA441E064E070E087ED98E00E94E0
:1078700079440E9474250E9454840C948481089554
:10788000CF93C82F0E946525C817C9F08C2F0E947E
:107890005E25CC2341F083E090E090935C088093D8
:1078A0005B0861E007C081E090E090935C08809302
:1078B0005B0860E085E498E0CF910C9400D1CF9113
:1078C0000895CF93DF93EB010E94652591E089270E
:1078D0000E94403C61E8CE01DF91CF910C94A9CE8B
:1078E0001F93CF93DF93182FEB010E946825181781
:1078F000E1F0112341F025E030E030935C08209363
:107900005B0861E007C021E030E030935C08209321
:107910005B0860E085E498E00E9400D1BE01812F01
:10792000DF91CF911F910C94FF27DF91CF911F9191
:10793000089540E054EA63E976ED85E498E00E941A
:10794000AAD010925408089585E498E00E94CED001
:10795000882369F040E054EA63E976ED85E498E035
:107960000E94AAD0809154088F5F80935408089594
:10797000CF93DF93EB0120914508211108C020919E
:107980005A08FC0120838091590888830FC02091F8
:107990005408FC01208385E498E00E942FD120E068
:1079A00037E843E953E00E9466D62883DF91CF9100
:1079B00008950F931F93CF93DF9300D0CDB7DEB719
:1079C0008C0161E80E94A9CEBE016F5F7F4FCE019E
:1079D00002960E94B83C60915B08C8010E94A9CE43
:1079E0006A81C8010E94A9CE6981C8010E94A9CEFE
:1079F00080915B0890915C089C012D7F21303105BE
:107A000011F0059729F40E94A925AB01BC0108C01B
:107A10004091550850915608609157087091580848
:107A2000C8010E94C0CE40E050E0BA01C8010E94E7
:107A3000C0CE0F900F90DF91CF911F910F910895BD
:107A4000CF93DF93CDB7DEB72F970FB6F894DEBF95
:107A50000FBECDBF69E578E08AE598E00E94B83CAA
:107A60006091590880915A080E945537CE010196BD
:107A70000E94A6D08FE0FE013196A5E4B8E0019007
:107A80000D928A95E1F7109254082F960FB6F8944C
:107A9000DEBF0FBECDBFDF91CF910895CF93DF93AF
:107AA00000D000D000D0CDB7DEB761E070E081EE4D
:107AB0009AE00E94A8A50E94203D0E94A9256093FB
:107AC000550870935608809357089093580882E0A1
:107AD00090E090935C0880935B0810925E0810928F
:107AE0005D0860E083E00E94898060E084E00E949D
:107AF000898045E06DE97AE1CE0101960E94F4CEDD
:107B000060E0CE0101960E9443CF26960FB6F8940E
:107B1000DEBF0FBECDBFDF91CF9108950F931F93AE
:107B2000CF93DF93CDB7DEB766970FB6F894DEBF7D
:107B30000FBECDBF80915D0890915E0801970297BE
:107B400008F077C00E94548460E083E00E9489803E
:107B500060E084E00E94898041E060E270E087EDAF
:107B600098E00E9479440E94A9256093550870937B
:107B7000560880935708909358080E94203D62E071
:107B800070E081E00E94FF27BE016B5E7F4FCE0157
:107B900046960E94B83C0E949684182F882309F4C8
:107BA00044C0CE0101960E942F7B62E070E0CE01BE
:107BB0000196113059F40E94C64E8C0182E00E9459
:107BC000197920E030E041E153E40AC00E94C64E3A
:107BD0008C0182E00E94197920E030E046E153E414
:107BE0000E94BFD50E9488D4F8016083718382838C
:107BF000938380E00E945E2546E950E060E070E0FB
:107C0000CE0101960E94547C6AED75E081EE9AE007
:107C10000E9458A581E08093150C40E856E968E978
:107C200070E08EE898E00E94AAD087ED98E00E946C
:107C3000E64480915D0890915E080197B9F48091C7
:107C40005B0890915C08049789F084E090E0909341
:107C50005E0880935D0881E08093420840E452E42E
:107C60006FE070E08DE998E00E94AAD08091C3098E
:107C7000811122C08091620A81111EC080E00E94A1
:107C80002C7640E064E070E087ED98E00E94794453
:107C900081E08093440884E090E090935C088093B6
:107CA0005B0866960FB6F894DEBF0FBECDBFDF91BE
:107CB000CF911F910F91089560E08DE499E00E94AB
:107CC0003EA260E08CEE99E00E943EA2D7CFEF92F8
:107CD000FF920F931F93CF93DF937C01EB01FC0185
:107CE0008081882309F4EEC061E0C7010E9456CE6E
:107CF000082F62E0C7010E9456CE803209F449C0C5
:107D0000C0F4823049F148F48111DCC061E8CE0151
:107D10000E94A9CE62EC72E0D0C0863151F18E3162
:107D200009F0D0C061E8CE010E94A9CE8CE29CE0AF
:107D30002DC08332E9F150F4813209F0C3C061E80B
:107D4000CE010E94A9CE8CE29CE02FC08432D1F1FA
:107D5000853209F46FC0B6C061E8CE010E94A9CE99
:107D6000013019F484EE99E002C085E499E00896A8
:107D70000DC061E8CE010E94A9CE013019F484EE55
:107D800099E002C085E499E0089618C00E94E6A137
:107D900093C061E8CE010E94A9CE013019F484EEAF
:107DA00099E002C085E499E008960E94E0A184C0B1
:107DB00061E8CE010E94A9CE8CE29CE00E94BEA1A7
:107DC000682F34C061E8CE010E94A9CE013019F4B9
:107DD00084EE99E002C085E499E008960E94E6A34B
:107DE000882311F010E801C010E08CE29CE00E94B2
:107DF000E6A3882311F080E401C080E0182B013055
:107E000019F484EE99E002C085E499E008960E9496
:107E1000EBA3182B013019F484EE99E002C085E43D
:107E200099E008960E94BEA1612F682BCE010E94A6
:107E3000A9CE46C061E8CE010E94A9CE013019F456
:107E400084EE99E002C085E499E008960E94EAA1D8
:107E5000BC01CE010E94ABCE013019F484EE99E052
:107E600002C085E499E008960E94EDA1BC01CE0114
:107E70000E94ABCE013019F484EE99E002C085E493
:107E800099E008960E94F0A1BC01CE010E94ABCE01
:107E90008CE29CE00E94EAA1BC01CE010E94ABCE24
:107EA0008CE29CE00E94EDA1BC01CE010E94ABCE11
:107EB0008CE29CE00E94F0A1BC01CE010E94ABCEFE
:107EC00081E001C080E0DF91CF911F910F91FF9081
:107ED000EF9008950F931F93CF93DF938C01EB01E5
:107EE000FC018081882309F490C060E0C8010E94F1
:107EF00056CE87FD8AC0482F50E04C31510508F01E
:107F000084C0FA01E157FF4F0C94A7D6BE01C80107
:107F10000E94B33878C0BE01C8010E94EF3873C018
:107F200080915D0890915E089C01215031092230BA
:107F3000310510F0059779F484E090E090935C08A7
:107F400080935B080E948E3D64E070E087ED98E0CE
:107F50000E94264503C081E08093440861E8CE0179
:107F60000E94A9CE50C0BE01C8010E9410394BC06A
:107F7000BE01C8010E94213946C0BE01C8010E944D
:107F8000733941C0BE01C8010E94E2393CC0BE0144
:107F9000C8010E94F83937C0BE01C8010E94F13BF8
:107FA00032C0BE01C8010E940A3A2DC0BE01C801FC
:107FB0000E94613C28C0BE01C801DF91CF911F9192
:107FC0000F910C94673EBE01C8010E94733A1BC01A
:107FD000BE01C8010E948D3A16C0BE01C8010E94B0
:107FE000E53A11C0BE01C8010E94653B0CC0CE013C
:107FF0000E94863B08C0CE010E94D93C04C0BE014D
:10800000C8010E94CC3881E001C080E0DF91CF91AF
:108010001F910F910895CF93DF93CDB7DEB72F97C0
:108020000FB6F894DEBF0FBECDBF80915B1D90915F
:108030005C1D892B39F080915B1D90915C1D04972C
:1080400009F012C180914408882309F468C0809126
:108050004208811105C080918E08882399F007C0DD
:108060008DE998E00E94CED08111F5CF58C08EE8FE
:1080700098E00E94CED0811105C00E94BB64882385
:1080800009F44DC080915B0890915C089C012D7FA4
:108090002130310511F0059741F484E090E0909390
:1080A0005C0880935B080E948E3D109244081092F9
:1080B0004208CE0101960E94A6D08FE0FE013196C3
:1080C000ADE9B8E001900D928A95E1F7CE010196F5
:1080D0000E94A6D08FE0FE013196AEE8B8E0019094
:1080E0000D928A95E1F7809143080E94C841109251
:1080F0004308CE0101960E94A6D08FE0FE01319682
:10810000ACEAB8E001900D928A95E1F710927E08F2
:1081100010925F0810925E0810925D08A5C08091D1
:10812000351D9091361D892B91F08091351D9091D0
:10813000361D049761F08091AC08811186C040E43F
:108140005DE063E070E08CEA98E00E94AAD0809144
:10815000341D882321F082E19DE10E9404CE8091AC
:10816000351D9091361D049709F049C08CEA98E0BE
:108170000E94FAD088E39DE10E946ACE80915D085A
:1081800090915E0820914208069761F4222341F005
:1081900069E888E39DE10E94A9CE1092420827C0B9
:1081A0006BE821C0222371F069E888E39DE10E9419
:1081B000A9CE1092420866E070E087ED98E00E9438
:1081C000264515C068E37DE182E19DE10E944F38BC
:1081D00081110DC068E37DE182E19DE10E946A3F6B
:1081E000811105C065E888E39DE10E94A9CE82E186
:1081F0009DE10E9404CE8EE09DE10E9481D180919C
:108200005D0890915E08029741F40E9445508111EB
:1082100004C010925E0810925D0880915D089091F4
:108220005E08059779F40E944A85811104C0109276
:108230005E0810925D0840E064E070E087ED98E031
:108240000E9479440E94A43C0FC08CEA98E00E94EE
:10825000CED0882309F47BCF82E19DE10E94F6CD48
:1082600084E08093341D73CF2F960FB6F894DEBF51
:108270000FBECDBFDF91CF910895AF92BF92CF9245
:10828000DF92EF92FF920F931F93CF93DF93CDB7BF
:10829000DEB76F970FB6F894DEBF0FBECDBF7C017F
:1082A00020915D0830915E082130310589F14CF450
:1082B000232BE1F581E090E090935E0880935D08C8
:1082C00027C02230310521F02530310509F12EC0BB
:1082D0008E010F5F1F4F6E0180E2C80ED11C580146
:1082E000C7010E947F28F80181938F01882319F02C
:1082F000EC15FD05A9F766E473E0C5010E94EDD811
:10830000892BA1F0B5018FE598E00E94F6D80EC048
:108310000FE518E0C7010E947F28F80181938F01C3
:10832000882321F0F8E00E371F07A1F70E94993C3F
:108330000E94B22581E090E090935C0880935B08F6
:108340006F960FB6F894DEBF0FBECDBFDF91CF9111
:108350001F910F91FF90EF90DF90CF90BF90AF9063
:10836000089540E063E97AE18BEB98E00E94F4CE57
:108370008CEA98E00E94A6D08DE998E00E94A6D0F1
:108380008EE898E00E94A6D085E498E00C94A6D0F0
:10839000CF93DF931F92CDB7DEB7F89494B78823BD
:1083A000A1F098E10FB6F8949093600010926000ED
:1083B0000FBE14BE99E228E130E00FB6F894A895FC
:1083C000209360000FBE9093600089830E94D65076
:1083D0000E94D24C0E944D850E9474250E94CA9D25
:1083E0000E94367A0E9454840E9484818981682F79
:1083F00087ED98E00E94344778940F90DF91CF91F9
:108400000895CF93DF9300D000D000D0CDB7DEB772
:1084100047E069EA7AE1CE0101960E94F4CE61E07C
:10842000CE0101960E9423CF47E069EA7AE1CE01AE
:1084300001960E94F4CE60E0CE0101960E9443CFE7
:1084400087ED98E00E94204881E00E94C84178941E
:108450000E940B400E94DC2987ED98E00E94B74AF9
:108460000E941C4EA895F4CF40E063E97AE181ECCC
:1084700098E00C94F4CE0F931F93CF93DF9300D02A
:1084800000D000D0CDB7DEB7062F1FB7F89445E077
:108490006BE97AE1CE0101960E94F4CE61E0011110
:1084A00001C060E0CE0101960E9443CF1FBF269617
:1084B0000FB6F894DEBF0FBECDBFDF91CF911F91F5
:1084C0000F910895CF93DF9300D000D000D0CDB7A7
:1084D000DEB71092CF081092CE0842E065EA7AE14A
:1084E000CE0101960E94F4CE60E0CE0101960E947A
:1084F00043CF42E065EA7AE1CE0101960E94F4CED4
:1085000060E0CE0101960E9443CF26960FB6F89404
:10851000DEBF0FBECDBFDF91CF9108956F927F92E6
:108520008F929F92AF92CF92EF92FF920F931F93F1
:10853000CF93DF93CDB7DEB768970FB6F894DEBF61
:108540000FBECDBF4C0104960E94A6D0C401439635
:108550000E94A6D0C40182960E94A6D0C401C196F2
:108560000E94A6D046E061EA7AE1CE0101960E941F
:10857000F4CE47E061EA7AE1CE0107960E94F4CE9C
:1085800042E061EA7AE1CE010D960E94F4CE42E02B
:108590006BE97AE1CE0143960E94F4CE8E010F5F23
:1085A0001F4F9E01295F3F4FAE01435F5F4FBE01EA
:1085B0006D5E7F4FC401805C9F4F0E94C28944E082
:1085C0006BE97AE1C8010E94F4CE45E061EA7AE104
:1085D000CE0107960E94F4CEE12CFF24F39400E034
:1085E0009E012F5F3F4FAE01495F5F4F60E0C401C6
:1085F00082599F4F0E94F08644E061EA7AE1CE0101
:1086000001960E94F4CE43E061EA7AE1CE0107963A
:108610000E94F4CE9CE1E92EFF24F39401E09E0138
:108620002F5F3F4FAE01495F5F4F61E0C401835F41
:108630009E4F0E94F086C40184559E4F0E94A6D092
:10864000C40185549E4F0E94A6D0840106531E4F3C
:10865000C80102960E94A6D0C80141960E94A6D0E9
:1086600041E065EA7AE1CE0101960E94F4CE40E055
:1086700065EA7AE1CE0107960E94F4CE43E065EA0E
:108680007AE1CE010D960E94F4CE340182E1681A9F
:108690008EEF780A9E012F5F3F4FAE01495F5F4F1B
:1086A000BE01635F7F4FC3010E9455A8A301B801BB
:1086B000C401865F9D4F0E9444A43401EFEB6E1A03
:1086C000ECEF7E0A40E063E0C3010E948DD0A4017C
:1086D0004D5A5C4F87E593E0FA019183808322E055
:1086E000A22EC12C30E1E32EFF24F39400E211EA24
:1086F00027E030E0B301C4018B5A9C4F0E94DB9FFE
:1087000061E08CE490E00E94009EF401E153FC4F94
:1087100091E0811101C090E0908368960FB6F894C3
:10872000DEBF0FBECDBFDF91CF911F910F91FF90A4
:10873000EF90CF90AF909F908F907F906F90089523
:108740000E94174D109220018AE08093210110921F
:10875000220180E090E2909329018093280182E039
:10876000809373008093B00094E09093B10099E1FE
:108770009093B3001092B4008093700081E08093D6
:1087800090008BE0809391001092990010929800D5
:1087900010929D0010929C001092710008952FB7C6
:1087A000F894FC0160817181828193812FBF0895CB
:1087B0000E94652581112DC0809170008D7F80936E
:1087C0007000809173008D7F8093730078940E9475
:1087D0006484F8948091700082608093700080912E
:1087E00073008260809373002091240130912501F1
:1087F00080912801909129012817390750F081E0D4
:1088000090E0909329018093280110922501109205
:1088100024010895CF93DF93EC01FC01EC52FC4F4F
:108820007183608362307105F9F48B5A9C4F0E940A
:10883000E6A3811112C00E94FF35882371F0CE019A
:108840008A589F4F0E94E6A3882391F0CE018B5E49
:108850009E4F0E94E6A3882359F08091D60881118B
:1088600007C081E08093D608C053DC4F81E0888345
:10887000DF91CF910895CF93DF93EC0189E180934D
:10888000D3088FE08093D20881E090E09093CF08E6
:108890008093CE086FEFCE01865F9D4F0E9413A894
:1088A000CF52DC4F81E08883DF91CF9108950F9301
:1088B0001F93CF93DF931F92CDB7DEB78C01FC01DE
:1088C000EE52FC4F2083865F9D4F49830E9458A53E
:1088D000C8010E943B4480E00E942C4EF801ED52FA
:1088E000FC4F498140830F90DF91CF911F910F91F1
:1088F0000895FC01EA52FC4F442321F08081862B2D
:108900008083089560958081682360830895CF9364
:10891000DF93EC018A589F4F0E94F3A181110EC092
:10892000CE018B5E9E4F0E94F3A1811107C0CE0144
:108930008B5A9C4FDF91CF910C94F3A181E0DF9192
:10894000CF910895FC01E152FC4F31E03083319624
:10895000608331964083319620833196108208954A
:10896000EF92FF920F931F93CF93DF93EC01FC01E3
:10897000E152FC4F10828C0102511E4F31967C0156
:108980008FE1E81A8CEFF80A4081F7016081C80195
:108990000E948FAAF701F080CE51DC4F8881F81633
:1089A00038F461E573E0C8010E94B5A9F394F6CFED
:1089B000DF91CF911F910F91FF90EF90089540E0CC
:1089C00052ED69E47BE643960C94AAD0FC01EC518D
:1089D000FC4F408151816281738182960C94AAD0B0
:1089E000CF93DF93EC01A296CE010E94FDD0CE0181
:1089F000DF91CF910C94FAD01F920F920FB60F9285
:108A000011240BB60F922F933F934F935F936F9365
:108A10007F938F939F93AF93BF93EF93FF9387EDD4
:108A200098E00E94D843FF91EF91BF91AF919F9141
:108A30008F917F916F915F914F913F912F910F9007
:108A40000BBE0F900FBE0F901F9018950F931F93A2
:108A5000CF93DF9300D000D000D0CDB7DEB78B012D
:108A60006115710589F41092D1081092D00847E081
:108A700067EA7AE1CE0101960E94F4CE60E0CE0171
:108A800001960E9443CF0CC08091D40890E08617D5
:108A9000970731F082E090E09093D1088093D0085E
:108AA0000093D40826960FB6F894DEBF0FBECDBF54
:108AB000DF91CF911F910F910895CF93DF9300D055
:108AC00000D000D0CDB7DEB741155105E9F41092C2
:108AD000CF081092CE0842E065EA7AE1CE01019615
:108AE0000E94F4CE61E0CE0101960E9443CF42E0A5
:108AF00065EA7AE1CE0101960E94F4CE61E0CE01F2
:108B000001960E9443CF10C06115710519F40E94AF
:108B100062420AC06093D3084093D20881E090E09B
:108B20009093CF088093CE0826960FB6F894DEBFB8
:108B30000FBECDBFDF91CF9108951F920F920FB658
:108B40000F9211240BB60F922F933F934F935F9385
:108B50006F937F938F939F93AF93BF93EF93FF9305
:108B6000CF93DF93CDB7DEB72697DEBFCDBF809121
:108B7000D7089091D808A091D908B091DA088C59FB
:108B80009F4FAF4FBF4F8093D7089093D808A093C3
:108B9000D908B093DA080E9494848091C70891E0C4
:108BA000980F9093C708853A08F4C5C01092C7087B
:108BB0008091CC089091CD081816190614F40197ED
:108BC0003AC08091D0089091D10881309105F1F49C
:108BD0008091CA089091CB0801969093CB0880931E
:108BE000CA0882E090E09093D1088093D00882E197
:108BF00090E09093CD088093CC0847E067EA7AE153
:108C0000CE0101960E94F4CE60E034C0823091051E
:108C1000B9F48091D40890E02091CA083091CB0833
:108C2000281739079CF083E090E09093D108809357
:108C3000D00880E590E09093CD088093CC081EC0CA
:108C40000397E1F41092CB081092CA0881E090E0FB
:108C50009093D1088093D00882E190E09093CD0862
:108C60008093CC0847E067EA7AE1CE0101960E9442
:108C7000F4CE61E0CE0101960E9443CF8091C808F6
:108C80009091C9081816190634F401979093C908F1
:108C90008093C80850C08091CE089091CF08813051
:108CA000910511F582E090E09093CF088093CE0873
:108CB0008091D30890E09093C9088093C80842E05F
:108CC00065EA7AE1CE0101960E94F4CE61E0CE0120
:108CD00001960E9443CF42E065EA7AE1CE01019617
:108CE0000E94F4CE61E023C0029729F581E090E074
:108CF0009093CF088093CE088091D20890E0909313
:108D0000C9088093C80842E065EA7AE1CE0101967D
:108D10000E94F4CE60E0CE0101960E9443CF42E073
:108D200065EA7AE1CE0101960E94F4CE60E0CE01C0
:108D300001960E9443CF26960FB6F894DEBF0FBE71
:108D4000CDBFDF91CF91FF91EF91BF91AF919F91F7
:108D50008F917F916F915F914F913F912F910F90E4
:108D60000BBE0F900FBE0F901F90189581539C4F14
:108D7000FC01608308950F931F93CF93DF9300D07E
:108D800000D000D0CDB7DEB7062F1FB7F89445E06E
:108D90006DE97AE1CE0101960E94F4CE61E0CE0148
:108DA00001960E9423CF45E06DE97AE1CE0101965C
:108DB0000E94F4CE602FCE0101960E9443CF1FBFC8
:108DC00026960FB6F894DEBF0FBECDBFDF91CF91D0
:108DD0001F910F9108950F931F93CF93DF93EC0191
:108DE000062FFC01EA52FC4F11E0108360E00E9464
:108DF000BB460E94FF35682FCE018B5E9E4F0E94BE
:108E000002A10E94EC36682F6127CE018B5A9C4F3D
:108E10000E9402A1CE010E94DF44011103C0CE01D5
:108E20000E94E6440E943188FE01EF52FC4F1082FE
:108E3000319681E0808336961182108232961182BB
:108E400010823296118210823597108238961082E5
:108E50003196108231961082CE51DC4F1882DF910C
:108E6000CF911F910F910895BF92CF92DF92EF9211
:108E7000FF920F931F93CF93DF9300D000D000D0C9
:108E8000CDB7DEB78C01B62E60E070E00E942645BB
:108E900060E082E090E00E94009E8095881F882715
:108EA000881F0E94517C61E08EE09DE10E94A3D169
:108EB00082E19DE10E9404CEF801108211821282AB
:108EC000138260E084E492E00E94009EF801EC517D
:108ED000FC4FA82FB0E020E037E843E953E00E94C0
:108EE000C3D6605C7D4B804F9F4F608371838283CC
:108EF00093836801FDE6CF0ED11CF60180818823A3
:108F000009F45EC07801F6EFEF1AFDEFFF0AC70122
:108F10000E9422A542E065EA7AE1CE0101960E9414
:108F2000F4CE61E0CE0101960E9423CF42E065EAD3
:108F30007AE1CE0101960E94F4CE61E0CE01019665
:108F40000E9423CF42E065EA7AE1CE0101960E94B9
:108F5000F4CE61E0CE0101960E9443CF42E065EA83
:108F60007AE1CE0101960E94F4CE61E0CE01019635
:108F70000E9443CF60E086E591E00E94009E81114F
:108F800003C065E070E002C064E070E0C7010E94C9
:108F9000A8A5BB2049F02FEF8BE792E92150804034
:108FA0009040E1F700C00000C7010E9423A4C70160
:108FB0000E9499A4AB01BC01C80104960E94AAD0EA
:108FC00040E050E060E070E0C8010E945D45BB20D9
:108FD00061F00E94928883E00E942C4EF801E053D9
:108FE000FC4F10823496118210826B2DC8010E94B2
:108FF000EB46F6018081882341F060E086E591E050
:109000000E94009E81110E942FA426960FB6F8940C
:10901000DEBF0FBECDBFDF91CF911F910F91FF90AB
:10902000EF90DF90CF90BF90089540E063E97AE140
:109030008FEB9CE00E94F4CE87ED98E00C948E427A
:109040000F931F93CF93DF9300D000D000D0CDB704
:10905000DEB78C0181E59DE00E945C520E94F7A37F
:10906000F801E359FF4F8083F801108211821282C8
:109070001382C8010E94A04347E067EA7AE1CE016B
:1090800001960E94F4CE61E0CE0101960E9423CFAA
:1090900044E06DE97AE1CE0101960E94F4CE61E0F0
:1090A000CE0101960E9423CF43E06DE97AE1CE0123
:1090B00001960E94F4CE61E0CE0101960E9423CF7A
:1090C00047E06BE97AE1CE0101960E94F4CE61E0BF
:1090D000CE0101960E9423CF40E06FE97AE1CE01F4
:1090E00001960E94F4CE61E0CE0101960E9423CF4A
:1090F00041E06FE97AE1CE0101960E94F4CE61E091
:10910000CE0101960E9423CF42E06FE97AE1CE01C1
:1091100001960E94F4CE61E0CE0101960E9423CF19
:10912000C801805C9F4F0E94498A40E950ED63E08E
:1091300070E0C801C1960E94AAD0C80182599F4F11
:109140000E94D187C801835F9E4F0E94D18745E06E
:109150006BE97AE1CE0101960E94F4CE61E0CE0186
:1091600001960E9423CFC8018F5B9C4F0E943BD089
:10917000C8018B5A9C4F0E94F19E40E251EA67E081
:1091800070E0C80185549E4F0E94AAD026960FB663
:10919000F894DEBF0FBECDBFDF91CF911F910F912D
:1091A00008959F92AF92BF92CF92DF92EF92FF927B
:1091B0000F931F93CF93DF937C01D62E142FC22ED3
:1091C000241708F471C0A22FB0E0A41BB109802FAE
:1091D00090E0A817B9070CF467C0F701E452FC4F00
:1091E0006081718116161706DCF432970190F081C8
:1091F000E02DE701C852DC4F88819981E81BF90B0B
:10920000F7FF03C0F195E195F109EA9FC001EB9FDB
:10921000900DFA9F900D11240E9452D6962E01C0F7
:10922000912CE701C251DE4F901680F44D2D612F35
:10923000CE010E948FAA012F0C1539F061E573E071
:10924000CE010E94B5A90F5FF7CF00E0602F610F3C
:109250004D2DCE010E948FAAC12CD12C10E0A92C3B
:10926000B12C9601200F311F2A153B0544F46FEFF6
:10927000CE010E9401AB8FEFC81AD80AF2CFF701D6
:10928000E252FC4F808191E089278083882331F06E
:1092900061EC77E0CE010E94CDA904C06FEFCE0152
:1092A0000E9401AB892D01C080E0DF91CF911F9119
:1092B0000F91FF90EF90DF90CF90BF90AF909F9075
:1092C00008956F927F928F929F92AF92BF92CF92AA
:1092D000DF92EF92FF920F931F93CF93DF93EC01F6
:1092E0008C0106521C4FF801118210826C01F4E2CD
:1092F000CF1AFCEFDF0AF601118210827C01F8E23E
:10930000EF1AFCEFFF0AF701118210820E948744D6
:10931000882309F48BC03E01FBEA6F1AFCEF7F0A39
:10932000C3010E94F3A19E0122593F4F4901FE0152
:10933000E35FFE4F5F018823E1F0C3010E9429A291
:10934000880F991FF70120813181280F391F318340
:109350002083C3010E94E0A1880F991FF80120819A
:109360003181280F391F3183208366EE662E712CE0
:1093700018C0FE01E451FF4F8081882329F060E08E
:10938000C90108960E943EA2FE01E557FE4F80816A
:10939000882329F060E0C50108960E943EA2612C56
:1093A000712CF8E08F0E911CC4010E94F3A1882358
:1093B00039F0FE01E451FF4F8081882309F463C036
:1093C00028E0A20EB11CC5010E94F3A1882339F048
:1093D000FE01E557FE4F8081882309F46CC0F80137
:1093E00080819181F701208131818217930734F4C4
:1093F000681A790AF6017182608203C0F6019183CE
:109400008083F60180819181892BD9F061E082E42B
:1094100091E00E94009E8823A1F067E080E491E043
:109420000E94009E873009F05EC00BC08E01095279
:109430001C4FF8018081882321F00E943188F801B7
:109440001082FE01E152FC4F8081882309F480C024
:109450007E01FDE1EF1AFCEFFF0ACE018E519C4F19
:10946000DE01AF51BC4FBE0160527C4FF70100815D
:10947000FC0120814C91FB016081CE010E94D1480A
:10948000F701808365C0C4010E9429A2F7012081F1
:109490003181280F391F31832083C4010E94E0A14C
:1094A000F80120813181280F391F31832083F6EEA6
:1094B0006F0E711C85CFC5010E9429A2F701208182
:1094C0003181280F391F31832083C5010E94E0A11B
:1094D000F80120813181280F391F31832083FEE676
:1094E0006F0E711C7CCFFE01E952FC4F808181110F
:1094F00002C081E08083F701A081B181F601C080C4
:10950000D180EE24D7FCE094FE2CF801008111817B
:109510000A1B1B0B17FF03C01195019511092FEFB3
:1095200030E00E94BCD6A70196010E9488D6B22ED8
:109530002FEF30E0D8010E94BCD6A70196010E940F
:1095400088D6822F20E04B2D60E00E94F18779CFF2
:10955000DF91CF911F910F91FF90EF90DF90CF900F
:10956000BF90AF909F908F907F906F9008955F9283
:109570006F927F928F929F92AF92BF92CF92DF9223
:10958000EF92FF920F931F93CF93DF93EC01FC01B7
:10959000E359FF4F8081811102C0512C1CC08E0104
:1095A000065F1D4FC8010E9494A47E0124E0E20ED4
:1095B000F11CC7010E94CED0882379F3C8010E9414
:1095C000A2A6C8010E9499A4AB01BC01C7010E94D8
:1095D000AAD055245394FE01E153FC4F8081882387
:1095E00041F08E0105541E4FC8010E94CED081115A
:1095F000F2C07E013FE2E31A3CEFF30AF7018081FB
:10960000882339F18E01065F1D4FC8010E9418A8FA
:109610008823F9F040E050E060E070E0CE010E9465
:109620005D450E943188F70110827E01FEE2EF1A4B
:10963000FCEFFF0AF7016081C8010E942CA681E0BF
:10964000F70180833196808181110E948E3D1092B6
:10965000D5087E01F2E2EF0EF11CC7010E94CED0C8
:10966000882321F08091AD0C83FDC2C0C7010E9408
:10967000CED08E0100531C4F882329F0F801808141
:10968000811159C007C0CE0143960E94CED08111EE
:10969000F5CF51C00E94CA3B029709F44CC00E940A
:1096A000CA3B019709F447C0FE01EA52FC4F808192
:1096B0008E7F806480836E01F6E7CF0ED11CC601D9
:1096C0000E94E0A19E012D5E3F4F5901FE01E35F24
:1096D000FE4F3F012E5B3C4F4901181619060CF452
:1096E0008BC0C30108960E94E0A1181619060CF45D
:1096F00083C0C4010E94E0A1181619060CF47CC0B6
:1097000060E070E0C6010E940EA160E070E0C3015D
:1097100008960E940EA160E070E0C4010E940EA1B4
:10972000C5010E94FDD0C7010E94CED0882319F048
:10973000CE010E94F044F8018081882309F43FC0E3
:109740008091D50881113BC00E94194E811137C00C
:1097500079C0293031050CF0C7C02230310509F439
:1097600095C02430310539F467E477E0CE01865F97
:109770009D4F0E9458A560E070E0C50108960E94C8
:109780000EA160E070E0C60108960E940EA160E0A4
:1097900070E0C7010E940EA180E00E942C4E0E9442
:1097A00072890E94A9380E9461250E94548410E0A9
:1097B00060E0812F0E9489801F5F1530C9F78E01FC
:1097C0000F5C1F4FC8010E94CED0882309F4DAC075
:1097D0005110D8C096C0CE018B5A9C4F0E94C4A293
:1097E00040E251EA67E070E0C8010E94AAD001CFD0
:1097F000CE010E94F0443ACFFE01EC51FC4F808133
:109800009181A281B38180349244AF40B10549F483
:10981000C5010E942FD16115724D89449B4608F401
:109820006FCF68E977E0CE01865F9D4F0E9458A513
:10983000CE010E943B4421E04FEF60E080E00E94B7
:10984000F1875ECF81E08093D5088AE08093D308CA
:109850008093D20881E090E09093CF088093CE0867
:10986000FE01EC52FC4F20813181CE01835F9E4F7F
:109870006C01EF57F1097F018F5991095C01283084
:10988000310509F066CF66EF76E070CF21E040E069
:1098900064E576E0CE010E945744F8E0AF0EB11CBB
:1098A000C5010E94E6A3882329F060E070E0C501AD
:1098B0000E940EA128E0C20ED11CC6010E94E6A3A0
:1098C000882329F060E070E0C6010E940EA1C70164
:1098D0000E94E6A3882329F060E070E0C7010E949F
:1098E0000EA1F80110824EC02031310519F465EA4D
:1098F00076E03CCF2032310509F03DCF63E076E0E1
:1099000035CFCE01805C9F4F0E94958A8823D1F18C
:1099100040E950ED63E070E0C8010E94AAD0FE016A
:10992000E759FF4F80818823B1F0813059F5CE018E
:10993000835F9E4FDF91CF911F910F91FF90EF902A
:10994000DF90CF90BF90AF909F908F907F906F905F
:109950005F900C944D87CE0182599F4F0E944D8796
:10996000CE01DF91CF911F910F91FF90EF90DF908B
:10997000CF90BF90AF909F908F907F906F905F90AF
:109980000C946149DF91CF911F910F91FF90EF905F
:10999000DF90CF90BF90AF909F908F907F906F900F
:1099A0005F900895CF93DF9300D000D000D0CDB763
:1099B000DEB761E08AE491E00E94009E91E08111AF
:1099C00001C090E09093D50C1092D90C1092D80C55
:1099D0001092DB0C1092DA0C1092DE0C1092DF0C5D
:1099E00085EC9CE00E94FDD01092D40C43E06BE922
:1099F0007AE1CE0101960E94F4CE61E0CE0101969B
:109A00000E9423CF43E06BE97AE1CE0101960E94E8
:109A1000F4CE60E0CE0101960E9443CF26960FB6A9
:109A2000F894DEBF0FBECDBFDF91CF9108951092A5
:109A3000A0001092A1001092A9001092A80010920C
:109A4000AB001092AA001092A5001092A4001092F0
:109A500072000895CF92DF92EF92FF92CF938091A0
:109A6000D80C9091D90C892B39F485EC9CE00E949C
:109A7000FDD01092D40C4BC021E02093D40C8091E7
:109A8000D80C9091D90C892B31F42093DF0CC12C88
:109A9000D12C76012EC08091DA0C9091DB0C2091B4
:109AA000D60C3091D70CB9010E943ED6880F991F71
:109AB000880F991FE091DC0CF091DD0CE80FF91F85
:109AC0008091DA0C9091DB0C0196B9010E943ED690
:109AD0009093DB0C8093DA0C8091D80C9091D90C88
:109AE00001979093D90C8093D80CC080D180E280EC
:109AF000F3809701A8EEB3E00E94ADD6AB01BC01A4
:109B000085EC9CE00E94AAD0C114D10439F4CF9115
:109B1000FF90EF90DF90CF900C94174DE12CF12C3B
:109B200084EFC81681E0D806E104F10418F0C2E021
:109B300083E002C0C3E086E0A7019601220F331F35
:109B4000441F551F04C0220F331F441F551F8A9501
:109B5000D2F760E074E284EF90E00E9466D6215074
:109B6000310980E48093A000C860C093A1003093C5
:109B7000A9002093A8001092AB001092AA001092A6
:109B8000A5001092A40010927200CF91FF90EF9068
:109B9000DF90CF9008950F931F932091D50C22232F
:109BA00009F444C04091D60C5091D70C2091D80CA8
:109BB0003091D90C4217530789F18C019B01809198
:109BC000D80C9091D90C8417950728F56091D80C82
:109BD0007091D90C8091DA0C9091DB0C860F971F55
:109BE000BA010E943ED6880F991F880F991FE091F5
:109BF000DC0CF091DD0CE80FF91F00831183228348
:109C000033838091D80C9091D90C01969093D90C04
:109C10008093D80C03C081E08093DE0C8091D40C3B
:109C2000811104C01F910F910C942A4D1F910F9127
:109C300008958091D40C08958091D50C882359F013
:109C40008091D40C882339F085EC9CE00E94CED022
:109C500081110C942A4D0895FF920F931F93CF9377
:109C6000DF93883048F5E82FF0E0EE0FFF1FE75A4A
:109C7000FC4F0081118101151105F1F0F12C84E0F8
:109C8000F89E90011124F801E20FF31F8591949141
:109C9000F9013296E00FF11FC591D491209719F088
:109CA000BE010E94CB4DF394CD2B49F7DF91CF91AC
:109CB0001F910F91FF90089564EF71E08BE790E0A2
:109CC000DF91CF911F910F91FF900C94CB4D40E00D
:109CD00063E97AE180E39DE00E94F4CE84E190E0C4
:109CE0009093D70C8093D60C1092D90C1092D80C6C
:109CF0001092DB0C1092DA0C80EE9CE09093DD0C5D
:109D00008093DC0C1092DE0C1092DF0C85EC9CE052
:109D10000C94A6D008958F929F92AF92BF92CF924B
:109D2000DF92EF92FF920F931F93CF93DF93CDB704
:109D3000DEB7FC0140835183628373830483158300
:109D400026833783C086D186E286F386848695860D
:109D5000A686B7864F85588969897A89408B518B49
:109D6000628B738BDF91CF911F910F91FF90EF90DA
:109D7000DF90CF90BF90AF909F908F900895660F27
:109D8000771F660F771F860F971F0895660F771F3F
:109D9000660F771F860F971F08950F9300E02EE33D
:109DA0003BE94BE75AE966E27AE98DED98E90E94D2
:109DB0002E9790934A0D8093490D892B79F40FEFDC
:109DC0002EE33BE94BE75AE966E27AE98DED98E943
:109DD0000E942E9790934A0D8093490D81E0209127
:109DE000490D30914A0D232B09F480E00F9108951D
:109DF0008091490D90914A0D0E94AA909093480D30
:109E00008093470D21E0892B09F420E0822F0895EB
:109E1000CF93DF93CDB7DEB7AB970FB6F894DEBF25
:109E20000FBECDBFAE014F5F5F4F69E673E080911B
:109E3000470D9091480D0E94B495BE016F5F7F4F12
:109E40008091470D9091480D0E94AA949093460DE1
:109E50008093450D21E0892B09F420E0822FAB96F9
:109E60000FB6F894DEBF0FBECDBFDF91CF9108953E
:109E70008091470D9091480D0E940F9760957095C5
:109E800080959095662797FD639577278827992772
:109E9000862F0895BF92CF92DF92EF92FF920F9399
:109EA0001F93CF93DF93CDB7DEB7AB970FB6F89480
:109EB000DEBF0FBECDBF8C016A0135E0B32EE62EAA
:109EC000F12C81E0E81AF108BE016F5F7F4F8091AD
:109ED000450D9091460D0E94F194882301F1D8011F
:109EE000FE01319620E030E02E153F0544F0F801E8
:109EF000E20FF31F10822115310571F007C0819127
:109F00008823A9F38D932F5F3F4FEECFC114D10467
:109F100041F0F601208305C0BA94B1F602C0F80101
:109F2000108280E090E0AB960FB6F894DEBF0FBED3
:109F3000CDBFDF91CF911F910F91FF90EF90DF90F8
:109F4000CF90BF9008950F931F93CF93DF938C0111
:109F5000EB01BE018091450D9091460D0E94F19458
:109F6000882369F0B801CE010E94EDD8892B89F7CA
:109F70008091450D9091460D0E94E49481E0DF911F
:109F8000CF911F910F910895FF920F931F93CF933D
:109F9000DF93CDB7DEB7AB970FB6F894DEBF0FBE39
:109FA000CDBF8B01BE016F5F7F4F0E94A34FF82E84
:109FB000882361F0BE016F5F7F4F8091470D9091C4
:109FC000480D0E942A92F801918380838F2DAB96D1
:109FD0000FB6F894DEBF0FBECDBFDF91CF911F91BA
:109FE0000F91FF90089560913F0D7091400D809109
:109FF000410D9091420D08951F93CF93DF93CDB7FC
:10A00000DEB7AB970FB6F894DEBF0FBECDBFBE0173
:10A010006F5F7F4F0E94A34F182F882349F0BE0126
:10A020006F5F7F4F8091470D9091480D0E949396EE
:10A03000812FAB960FB6F894DEBF0FBECDBFDF9178
:10A04000CF911F910895CF93DF93CDB7DEB7AB9734
:10A050000FB6F894DEBF0FBECDBFAE014F5F5F4FAE
:10A06000BC018091450D9091460D0E943E9691E075
:10A07000811101C090E0892FAB960FB6F894DEBF36
:10A080000FBECDBFDF91CF91089580913D0D089512
:10A0900080913E0D0895CF93DF93EC018091430DA5
:10A0A0009091440D0097E1F0488150E0BE016E5F51
:10A0B0007F4F0E947B9328818091390D90913A0DBA
:10A0C000A0913B0DB0913C0D820F911DA11DB11DC2
:10A0D0008093390D90933A0DA0933B0DB0933C0DB6
:10A0E000DF91CF91089580913E0D882381F080917A
:10A0F000430D9091440D009721F00E945C920E94C4
:10A1000071981092440D1092430D10923E0D609183
:10A11000390D70913A0D80913B0D90913C0D089551
:10A120000E943998882391F041E050E068E37DE097
:10A130008091430D9091440D0E94709221E0181679
:10A1400019060CF020E02093370D089521E041E03E
:10A150006FE379E087ED98E00E9457441092370D45
:10A160001092360D08958091370D0895CF93DF93A7
:10A170001F92CDB7DEB78091380D89830E94905031
:10A1800089810F90DF91CF91089510923D0D8091BC
:10A19000430D9091440D009721F00E945C920E9423
:10A1A00071981092440D1092430D089580913D0DC9
:10A1B00081110E94C55080913E0D81110E94735003
:10A1C0008091450D9091460D009731F00E94DE94EC
:10A1D0001092460D1092450D8091470D9091480DBB
:10A1E000009731F00E9424921092480D1092470D72
:10A1F0008091490D90914A0D009731F00E94CB97C4
:10A2000010924A0D1092490D10923F0D1092400D80
:10A210001092410D1092420D08950E947099811183
:10A220000EC00E943998811105C00E94D65081E06D
:10A2300090E008950E94D65082E090E008950E9438
:10A24000CD4E811105C00E94D65083E090E0089564
:10A250000E94F84E811105C00E94D65084E090E023
:10A2600008950E94084F811105C00E94D65085E0D4
:10A2700090E008950E94384F811105C00E94D65089
:10A280008AE090E008950E945698882319F086E0AD
:10A2900090E0089580E090E008950E94D6500E94DA
:10A2A0000D51009719F08630910541F48091450DCC
:10A2B0009091460D0E94E49480E090E00895CF9341
:10A2C000DF93EC010E94D6500E940D51009761F57A
:10A2D0001092390D10923A0D10923B0D10923C0DD8
:10A2E0001092440D1092430DCE010E94FC4FCE01FE
:10A2F0000E942350882391F063E47DE0CE010E9408
:10A30000C44F882369F08091430D9091440D892BAF
:10A3100049F081E080933E0D80E005C087E003C0F6
:10A3200083E001C088E090E0DF91CF910895CF9362
:10A33000DF93EC010E94D6500E940D51009719F056
:10A340008630910561F51092390D10923A0D1092F8
:10A350003B0D10923C0D1092440D1092430D63E49E
:10A360007DE0CE010E94C44F882331F08091430DDF
:10A370009091440D009711F487E010C00E94099756
:10A3800060933F0D7093400D8093410D9093420D6B
:10A3900081E080933D0D0E94905080E090E0DF913D
:10A3A000CF91089540E063E97AE18BE49DE00C945D
:10A3B000F4CECF92DF92EF92FF920F931F93CF9341
:10A3C000DF9300D000D000D0CDB7DEB78C017C0188
:10A3D0006C018EE1C80ED11CC7010E94E6CEE6E0FA
:10A3E000EE0EF11CEC14FD04B9F746E069EA7AE1DF
:10A3F000C7010E94F4CE85E0F80184A345E063EA3A
:10A400007AE1CE0101960E94F4CE86E0FE013196FB
:10A41000D80101900D928A95E1F746E065E97AE16D
:10A42000CE0101960E94F4CE86E0FE013196D8015D
:10A43000169601900D928A95E1F743E065E97AE17D
:10A44000CE0101960E94F4CE86E0FE013196D8013D
:10A450001C9601900D928A95E1F744E069EA7AE151
:10A46000CE0101960E94F4CE86E0FE013196D8011D
:10A47000529601900D928A95E1F747E069E97AE1F9
:10A48000CE0101960E94F4CE86E0FE013196D801FD
:10A49000589601900D928A95E1F726960FB6F8949A
:10A4A000DEBF0FBECDBFDF91CF911F910F91FF9007
:10A4B000EF90DF90CF900895EF92FF920F931F934C
:10A4C000CF93DF93EC01F12C86E0E82E8CA1F816F7
:10A4D00078F48E01EF9C000D111D112461E0C8017C
:10A4E0000E9423CF61E0C8010E9443CFF394EECFD6
:10A4F0006E9661E0CE010E9423CF61E0CE01DF9134
:10A50000CF911F910F91FF90EF900C9443CF0F9339
:10A510001F93CF93DF93EC0185E18A95F1F700005B
:10A5200061E0CE014E960E9443CF85E18A95F1F716
:10A53000000010E006E08CA1181750F461E0CE0195
:10A54000019F800D911D11240E9443CF1F5FF3CF07
:10A5500085E18A95F1F70000DF91CF911F910F916E
:10A560000895CF92DF92EF92FF920F931F93CF93B4
:10A57000DF93C62EEA0128E0E22EF12C30E8D32E3C
:10A580008C01025E1F4F61E09D2D9C2109F460E06B
:10A59000CE010E9443CF61E0C8010E9443CF85E114
:10A5A0008A95F1F7000060E0C8010E9443CFD6947D
:10A5B00081E0E81AF108E114F10429F761E0CE0125
:10A5C0000E9443CF60E0CE010E9423CF61E0C8012A
:10A5D0000E9443CFCE010E9436CFF82E60E0C80122
:10A5E0000E9443CF61E0CE010E9423CF81E08F25FE
:10A5F000DF91CF911F910F91FF90EF90DF90CF905F
:10A600000895DF92EF92FF920F931F93CF93DF9302
:10A61000EC01E62E8A01F12C46E0D42E8CA1F8162E
:10A6200050F460E0CE01DF9C800D911D11240E944A
:10A6300043CFF394F3CF85E18A95F1F7000060E012
:10A64000CE014E960E9443CFA8016E2DCE01DF9120
:10A65000CF911F910F91FF90EF90DF900C94B1522A
:10A6600040E063E97AE186E79DE00E94F4CE81E56F
:10A670009DE00C94D9514F925F926F927F928F928E
:10A680009F92AF92BF92CF92DF92EF92FF920F9381
:10A690001F93CF93DF938091AF0D9091B00D892BD5
:10A6A00009F0B6C39091B80D8091B70D981771F06D
:10A6B000C091B70D17E7C19FE0011124C754D24FD5
:10A6C000FE01EC58FF4F81E0808302C0C0E0D0E083
:10A6D000D093B00DC093AF0D209709F466C3FE016F
:10A6E00020E030E0C08CD18CE28CF38CA901440FC7
:10A6F000551F440F551F445E594EDA01CD92DD922D
:10A70000ED92FC9213972F5F3F4F34962530310521
:10A7100049F78AAD80937C0D80917D0D811111C028
:10A720001092880D1092890D10928A0D10928B0D47
:10A73000FE01E25AFF4F808191819F3408F042C0B0
:10A740004DC04EE75DE0EBEAFDE0BE0120E030E009
:10A75000DB011C96CD90DD90ED90FC901F97CD28ED
:10A76000CE28CF2819F1DA018C918823F9F0D9018C
:10A77000A755B24F8C91D901AA0FBB1FAD5EB94E40
:10A78000882341F08D919C91119700811181801B4C
:10A79000910B07C08D919C91119700811181800FC1
:10A7A000911F11969C938E93DA011C922F5F3F4F5D
:10A7B0006C5F7F4F4F5F5F4F32962230310509F457
:10A7C000AFCFC6CF9D3930F463E0969587956A95F3
:10A7D000E1F702C088E893E128E014C0983230F035
:10A7E000969587959695879524E00CC0943120F036
:10A7F0009695879522E006C08032910510F480E29C
:10A8000090E021E02093830D80978115B8E09B07AD
:10A81000B8F0E92FFF27EE0FFF1FEE0FFF1FED5AD5
:10A82000F24F4591559165917491AA27879F9001A8
:10A83000869F210D3A1F06942A1F3A1F112418C023
:10A84000FC01F695E795EC7FED5AF64F4591559151
:10A850006591749187709927869F9001879F300D2D
:10A86000969F300D112403E0369527950A95E1F760
:10A87000421B530B5093810D4093800D8091830DAB
:10A880008093820DFE01EE58FF4F8081882309F4EA
:10A890006DC0CA59DF4F888199819093870D80934D
:10A8A000860D9F3460F09D3930F4D3E096958795FE
:10A8B000DA95E1F702C088E893E128E014C0983205
:10A8C00030F0969587959695879524E00CC0943145
:10A8D00020F09695879522E006C08032910510F40D
:10A8E00080E290E021E02093830D80978115C8E0FD
:10A8F0009C07B8F0E92FFF27EE0FFF1FEE0FFF1F99
:10A90000ED5AF24F4591559165917491AA27879F11
:10A910009001869F210D3A1F06942A1F3A1F112489
:10A9200018C0FC01F695E795EC7FED5AF64F45917E
:10A9300055916591749187709927869F9001879FA3
:10A94000300D969F300D112463E0369527956A955A
:10A95000E1F7421B530BCA01A0E0B0E080938C0DDD
:10A9600090938D0DA0938E0DB0938F0D5093290170
:10A9700040932801E091AF0DF091B00D20AD2093F0
:10A98000940DEA58FF4F3081809113169091141660
:10A99000892B09F033608091151690911616892B3A
:10A9A00009F034608091111638131BC0C091AF0DAF
:10A9B000D091B00D88819981AA81BB814C895D8934
:10A9C0006E897F89FE01EB58FF4F308111E00097BF
:10A9D000A105B10509F410E010934C16111144C003
:10A9E00083C0A5E1B2E0E9E1F2E080E090E061E05F
:10A9F00070E0AB01082E01C0440F0A94EAF7C09141
:10AA00001116C327C42349F1C32FC4235091111633
:10AA1000CC2391F0542B50931116CD91DC911197CA
:10AA20001881AB01008002C0440F551F0A94E2F761
:10AA300040954123488311C040954523409311160A
:10AA4000CD91DC9111971881AB01008002C0440FB9
:10AA5000551F0A94E2F7142B188301969396B39628
:10AA60008530910531F6A2CF122F11706A017B015A
:10AA7000F594E794D794C794F094E094D094C0945C
:10AA8000C11CD11CE11CF11CC0924D16D0924E1677
:10AA9000E0924F16F092501601E0311100E0009361
:10AAA000441640934516509346166093471670938C
:10AAB00048168093551690935616A0935716B09348
:10AAC0005816112311F08FEF01C081E080934A16D0
:10AAD00081E0812780934B161092511610925216E6
:10AAE00010925316109254168C819D81AE81BF81B5
:10AAF0004C895D896E897F8911E00097A105B105B8
:10AB000009F410E010937516112309F442C021FBDB
:10AB1000112710F96A017B01F594E794D794C79443
:10AB2000F094E094D094C094C11CD11CE11CF11CA1
:10AB3000C0927616D0927716E0927816F092791637
:10AB400001E0313009F000E000936D1640936E167D
:10AB500050936F16609370167093711680937E16E3
:10AB600090937F16A0938016B0938116112311F055
:10AB70008FEF01C081E08093731681E0812780937D
:10AB8000741610927A1610927B1610927C16109200
:10AB90007D1688859985AA85BB854C895D896E89D6
:10ABA0007F8911E00097A105B10509F410E0109329
:10ABB0009E16112309F442C022FB112710F96A01E5
:10ABC0007B01F594E794D794C794F094E094D094E3
:10ABD000C094C11CD11CE11CF11CC0929F16D092E4
:10ABE000A016E092A116F092A21601E0323009F010
:10ABF00000E0009396164093971650939816609332
:10AC0000991670939A168093A7169093A816A093FE
:10AC1000A916B093AA16112311F08FEF01C081E09D
:10AC200080939C1681E0812780939D161092A31635
:10AC30001092A4161092A5161092A6168C859D85CA
:10AC4000AE85BF854C895D896E897F8911E000974B
:10AC5000A105B10509F410E01093C716112309F4FA
:10AC600042C023FB112710F96A017B01F594E79498
:10AC7000D794C794F094E094D094C094C11CD11C94
:10AC8000E11CF11CC092C816D092C916E092CA16F7
:10AC9000F092CB1601E0333009F000E00093BF16CC
:10ACA0004093C0165093C1166093C2167093C3169A
:10ACB0008093D0169093D116A093D216B093D3164A
:10ACC000112311F08FEF01C081E08093C51681E060
:10ACD00081278093C6161092CC161092CD16109232
:10ACE000CE161092CF1688899989AA89BB894C897A
:10ACF0005D896E897F89F08131E00097A105B105FA
:10AD000009F430E03093F016332309F441C024FBFA
:10AD1000EE27E0F98A019B01359527951795079550
:10AD200030952095109501951F4F2F4F3F4F009361
:10AD3000F1161093F2162093F3163093F41621E0D7
:10AD4000F43009F020E02093E8164093E916509380
:10AD5000EA166093EB167093EC168093F9169093B5
:10AD6000FA16A093FB16B093FC16EE2311F08FEFAA
:10AD700001C081E08093EE1681E08E278093EF166C
:10AD80001092F5161092F6161092F7161092F81609
:10AD90001092A00D10929F0D1092900D1092910D97
:10ADA0001092920D1092930D33C080ED97E0909326
:10ADB0002901809328018091131690911416892BF4
:10ADC00039F58091151690911616892B09F5709119
:10ADD0001216809111167817D9F0A5E1B2E0E9E1D9
:10ADE000F2E080E090E041E050E09A01082E01C0DE
:10ADF000220F0A94EAF7609111166727622311F077
:10AE00000C94916201969396B3968530910569F7FB
:10AE100080917D0D2091AF0D3091B00D811104C056
:10AE2000232B09F044C069C1EEE7FDE0ABEABDE0C9
:10AE300080E090E0FF24F394B9016A587F4F211518
:10AE4000310569F0EB01488150E0EC0123960C2EAE
:10AE500002C0559547950A94E2F740FD20C0408115
:10AE600041111DC0EC01C755D24F4881EC01CC0FF8
:10AE7000DD1FCD5ED94E442341F0488159810D91AB
:10AE80001C911197400F511F07C0488159810D91A6
:10AE90001C911197401B510B59834883F0820196F6
:10AEA000319612968230910509F4BACFC8CFE0915D
:10AEB000830D40919F0D5091A00DC0909B0DD0909F
:10AEC0009C0DE0909D0DF0909E0DF094E094D09438
:10AED000C094C11CD11CE11CF11CCD2CDE2CEF2C2C
:10AEE000FF24E7FCFA9470E021E030E061E07E1797
:10AEF0000CF049C0C091AF0DD091B00DDE01AE583D
:10AF0000BF4F8C918111FCC080914C16811170C192
:10AF10008091751681115EC280919E1681114CC37D
:10AF20008091C716811139C48091F016811126C510
:10AF30008091900D9091910DA091920DB091930DF3
:10AF40000196A11DB11D8093900D9093910DA0933A
:10AF5000920DB093930D8090900D9090910DA090D4
:10AF6000920DB090930DA091AF0DB091B00D54968D
:10AF70008D919D910D90BC91A02D88169906AA06E1
:10AF8000BB0608F4E2C50091900D1091910D20913F
:10AF9000920D3091930DE091AF0DF091B00D84A51D
:10AFA00095A5A6A5B7A580179107A207B30708F432
:10AFB000FFC540918C0D50918D0D60918E0D70915B
:10AFC0008F0D04A915A926A937A9AA27419FB12D3C
:10AFD000529FC001629F900D619F800D911D429F05
:10AFE000B00D811D9A1F519FB00D811D9A1F609F4A
:10AFF000B00D811D9A1F509FB10D8A1F9A1FB695E3
:10B000008A1F9A1F1124DF01AA59BF4F4D915C91ED
:10B01000480F591F5093870D4093860DE25AFF4FFA
:10B0200080819181A281B38160E070E084179507EF
:10B03000A607B70720F49093870D8093860D809123
:10B04000860D9091870D9F3408F484C59D3908F0D2
:10B050007EC563E0969587956A95E1F728E0209391
:10B06000830D80978115D8E09D0708F488C5E92FE6
:10B07000FF27EE0FFF1FEE0FFF1FED5AF24F459116
:10B08000559165917491AA27879F9001869F210D04
:10B090003A1F06942A1F3A1F1124421B530B509348
:10B0A00029014093280180918C0D90918D0DA091E4
:10B0B0008E0DB0918F0D840F951FA11DB11D809332
:10B0C0008C0D90938D0DA0938E0DB0938F0D4091AC
:10B0D000900D5091910D6091920D7091930DE091B2
:10B0E000AF0DF091B00D84899589A689B78948176D
:10B0F00059076A077B0708F081C680E00C94DB6281
:10B100004115510509F43FC04230510509F0FCCE0C
:10B110008EAD9FAD919581959109AA2797FDA09538
:10B12000BA2F8090C8169090C916A090CA16B090F9
:10B13000CB16880D991DAA1DBB1D8C0D9D1DAE1D26
:10B14000BF1D8093C8169093C916A093CA16B093DA
:10B15000CB168EAD9FAD919581959109AA2797FD4C
:10B16000A095BA2F8090F1169090F216A090F31649
:10B17000B090F416880D991DAA1DBB1D8C0D9D1D48
:10B18000AE1DBF1D2CC08CAC9DACAA2497FCA09416
:10B19000BA2C8091C8169091C916A091CA16B09188
:10B1A000CB16880D991DAA1DBB1D8093C8169093C0
:10B1B000C916A093CA16B093CB168CAC9DACAA242A
:10B1C00097FCA094BA2C8091F1169091F216A09160
:10B1D000F316B091F416880D991DAA1DBB1D80931E
:10B1E000F1169093F216A093F316B093F4168CCE4A
:10B1F0008090551690905616A0905716B0905816FD
:10B2000080914D1690914E16A0914F16B091501608
:10B21000880D991DAA1DBB1D80934D1690934E1647
:10B22000A0934F16B0935016181619061A061B064F
:10B230000CF06ECE409051165090521660905316FE
:10B2400070905416481459046A047B040CF060CEC4
:10B250008090451690904616A0904716B0904816DC
:10B2600088199909AA09BB0980934D1690934E1627
:10B27000A0934F16B093501680914916882379F009
:10B2800080910D1690910E16F0914A168F0F911D18
:10B29000F7FD9A9590930E1680930D166CC09091C1
:10B2A0004B168091311681119627A0910E02B09114
:10B2B0000F0280911202FC91E90102C0CC0FDD1F48
:10B2C0008A95E2F7992319F0FC2BFC9304C0CE0178
:10B2D00080958F238C9380914B168823A1F08091C9
:10B2E000230290912402892B39F1A0912502B0917B
:10B2F00026028C9190E00090270202C095958795D8
:10B300000A94E2F713C080911C0290911D02892BD0
:10B3100099F0A0911E02B0911F028C9190E00090D4
:10B32000200202C0959587950A94E2F7817090916A
:10B33000301689130C94BD62A0910702B0910802E7
:10B34000FC91C90100900B0202C0880F991F0A945A
:10B35000E2F7F82BFC93A0910702B0910802FC9150
:10B36000C90100900B0202C0880F991F0A94E2F7EE
:10B3700080958F238C9380911C1690911D16A0911F
:10B380001E16B0911F1680904A16992487FC90943F
:10B39000A92CB92C880D991DAA1DBB1D80931C16C4
:10B3A00090931D16A0931E16B0931F1680915116F0
:10B3B00090915216A0915316B09154160196A11D6A
:10B3C000B11D8093511690935216A0935316B093CB
:10B3D00054169ECD80907E1690907F16A090801679
:10B3E000B09081168091761690917716A09178167C
:10B3F000B0917916880D991DAA1DBB1D80937616F4
:10B4000090937716A0937816B093791618161906AC
:10B410001A061B060CF080CD40907A1650907B16D1
:10B4200060907C1670907D16481459046A047B0461
:10B430000CF072CD80906E1690906F16A0907016E2
:10B44000B090711688199909AA09BB0980937616DC
:10B4500090937716A0937816B09379168091721610
:10B46000882379F080910F1690911016F091731641
:10B470008F0F911DF7FD9A959093101680930F16DC
:10B480006CC09091741680915A1681119627A091E4
:10B490003102B091320280913502FC91E90102C083
:10B4A000CC0FDD1F8A95E2F7992319F0FC2BFC9352
:10B4B00004C0CE0180958F238C93809174168823CD
:10B4C000A1F08091460290914702892B39F1A09119
:10B4D0004802B09149028C9190E000904A0202C06B
:10B4E000959587950A94E2F713C080913F02909159
:10B4F0004002892B99F0A0914102B09142028C91B7
:10B5000090E00090430202C0959587950A94E2F777
:10B5100081709091591689130C94C162A0912A02EE
:10B52000B0912B02FC91C90100902E0202C0880F3D
:10B53000991F0A94E2F7F82BFC93A0912A02B0918C
:10B540002B02FC91C90100902E0202C0880F991FA6
:10B550000A94E2F780958F238C9380912016909126
:10B560002116A0912216B09123168090731699246B
:10B5700087FC9094A92CB92C880D991DAA1DBB1D80
:10B580008093201690932116A0932216B093231631
:10B5900080917A1690917B16A0917C16B0917D16C1
:10B5A0000196A11DB11D80937A1690937B16A093EE
:10B5B0007C16B0937D16B0CC8090A7169090A816FC
:10B5C000A090A916B090AA1680919F169091A016EF
:10B5D000A091A116B091A216880D991DAA1DBB1DA0
:10B5E00080939F169093A016A093A116B093A216D5
:10B5F000181619061A061B060CF092CC4090A316DA
:10B600005090A4166090A5167090A6164814590480
:10B610006A047B040CF084CC809097169090981666
:10B62000A0909916B0909A1688199909AA09BB0991
:10B6300080939F169093A016A093A116B093A21684
:10B6400080919B16882379F08091111690911216A3
:10B65000F0919C168F0F911DF7FD9A9590931216FD
:10B66000809311166BC090919D1680918316811165
:10B670009627A0915402B091550280915802FC91F6
:10B68000E90102C0CC0FDD1F8A95E2F7992319F07A
:10B69000FC2BFC9304C0CE0180958F238C9380916A
:10B6A0009D168823A1F08091690290916A02892BEE
:10B6B00031F1A0916B02B0916C028C9190E00090FE
:10B6C0006D0202C0959587950A94E2F713C08091A8
:10B6D000620290916302892B91F0A0916402B09173
:10B6E00065028C9190E00090660202C09595879566
:10B6F0000A94E2F7817090918216891346C7A0914F
:10B700004D02B0914E02FC91C9010090510202C05D
:10B71000880F991F0A94E2F7F82BFC93A0914D0231
:10B72000B0914E02FC91C9010090510202C0880FF5
:10B73000991F0A94E2F780958F238C9380912416A9
:10B7400090912516A0912616B091271680909C16F0
:10B75000992487FC9094A92CB92C880D991DAA1DB9
:10B76000BB1D8093241690932516A0932616B093A4
:10B7700027168091A3169091A416A091A516B091BA
:10B78000A6160196A11DB11D8093A3169093A41631
:10B79000A093A516B093A616C3CB8090D016909018
:10B7A000D116A090D216B090D3168091C816909161
:10B7B000C916A091CA16B091CB16880D991DAA1D65
:10B7C000BB1D8093C8169093C916A093CA16B09358
:10B7D000CB16181619061A061B060CF0A5CB4090BE
:10B7E000CC165090CD166090CE167090CF1648149F
:10B7F00059046A047B040CF097CB8090C01690909B
:10B80000C116A090C216B090C31688199909AA094A
:10B81000BB098093C8169093C916A093CA16B0931B
:10B82000CB168091C416882379F0809113169091DD
:10B830001416F091C5168F0F911DF7FD9A959093F0
:10B840001416809313166BC09091C6168091AC1697
:10B8500081119627A0917702B091780280917B02A6
:10B86000FC91E90102C0CC0FDD1F8A95E2F7992314
:10B8700019F0FC2BFC9304C0CE0180958F238C9390
:10B880008091C6168823A1F080918C0290918D0240
:10B89000892B31F1A0918E02B0918F028C9190E0B2
:10B8A0000090900202C0959587950A94E2F713C024
:10B8B0008091850290918602892B91F0A091870258
:10B8C000B09188028C9190E00090890202C0959519
:10B8D00087950A94E2F781709091AB16891358C648
:10B8E000A0917002B0917102FC91C90100907402A4
:10B8F00002C0880F991F0A94E2F7F82BFC93A091DD
:10B900007002B0917102FC91C9010090740202C0F2
:10B91000880F991F0A94E2F780958F238C9380916A
:10B92000281690912916A0912A16B0912B16809076
:10B93000C516992487FC9094A92CB92C880D991DC3
:10B94000AA1DBB1D8093281690932916A0932A1632
:10B95000B0932B168091CC169091CD16A091CE1657
:10B96000B091CF160196A11DB11D8093CC16909376
:10B97000CD16A093CE16B093CF16D6CA8090F916E6
:10B980009090FA16A090FB16B090FC168091F116DC
:10B990009091F216A091F316B091F416880D991DAE
:10B9A000AA1DBB1D8093F1169093F216A093F31677
:10B9B000B093F416181619061A061B060CF0B8CA2E
:10B9C0004090F5165090F6166090F7167090F816A5
:10B9D000481459046A047B040CF0AACA8090E91642
:10B9E0009090EA16A090EB16B090EC168819990981
:10B9F000AA09BB098093F1169093F216A093F3164F
:10BA0000B093F4168091ED16882379F08091151685
:10BA100090911616F091EE168F0F911DF7FD9A95E5
:10BA2000909316168093151661C09091EF16809131
:10BA3000D51681119627A0919A02B0919B02809110
:10BA40009E02FC91E90102C0CC0FDD1F8A95E2F74E
:10BA5000992319F0FC2BFC9304C0CE0180958F2311
:10BA60008C938091EF168823A9F08091AF0290917A
:10BA7000B002892B09F48FC5A091B102B091B20236
:10BA80008C9190E00090B30202C0959587950A943E
:10BA9000E2F714C08091A8029091A902892B09F4C1
:10BAA0007AC5A091AA02B091AB028C9190E000906F
:10BAB000AC0202C0959587950A94E2F78170909147
:10BAC000D416891709F467C510921B16A09193022A
:10BAD000B0919402FC91C9010090970202C0880FB6
:10BAE000991F0A94E2F780958F238C9380912C16EE
:10BAF00090912D16A0912E16B0912F168090EE16D3
:10BB0000992487FC9094A92CB92C880D991DAA1D05
:10BB1000BB1D80932C1690932D16A0932E16B093D8
:10BB20002F168091F5169091F616A091F716B09108
:10BB3000F8160196A11DB11D8093F5169093F61687
:10BB4000A093F716B093F816F3C97F5FD0C988E8C1
:10BB500093E184CA983230F09695879596958795AB
:10BB600024E07DCA943120F09695879522E077CA2B
:10BB70008032910510F480E290E021E070CAFC016F
:10BB8000F695E795EC7FED5AF64F45915591659105
:10BB9000749187709927869F9001879F300D969F9B
:10BBA000300D112403E0369527950A95E1F775CA03
:10BBB0000091900D1091910D2091920D3091930D67
:10BBC00080A991A9A2A9B3A980179107A207B307D9
:10BBD00008F0FFC0452B31F481E090E09093A00D78
:10BBE00080939F0D80919F0D9091A00D019771F40E
:10BBF00082E090E09093A00D80939F0D10929B0D9A
:10BC000010929C0D10929D0D10929E0D80919B0D97
:10BC100090919C0DA0919D0DB0919E0DEF01C05C87
:10BC2000DF4F488159816A817B81840F951FA61F50
:10BC3000B71F80939B0D90939C0DA0939D0DB09387
:10BC40009E0D4091880D5091890D60918A0D7091E3
:10BC50008B0D04A915A926A937A9AA27419FB12DA3
:10BC6000529FC001629F900D619F800D911D429F68
:10BC7000B00D811D9A1F519FB00D811D9A1F609FAD
:10BC8000B00D811D9A1F509FB10D8A1F9A1FB69546
:10BC90008A1F9A1F11249093850D8093840D4091E3
:10BCA000860D5091870D4817590728F4E659FF4F24
:10BCB0008081918113C0481B590B5093850D40938F
:10BCC000840DE659FF4F80819181A281B38160E0AC
:10BCD00070E0481759076A077B0720F49093850D99
:10BCE0008093840D8091840D9091850D9F3460F038
:10BCF0009D3930F4D3E096958795DA95E1F702C047
:10BD000088E893E128E014C0983230F09695879542
:10BD10009695879524E00CC0943120F096958795F0
:10BD200022E006C08032910510F480E290E021E02C
:10BD30002093830D8097811518E09107B8F0E92FC3
:10BD4000FF27EE0FFF1FEE0FFF1FED5AF24F459139
:10BD5000559165917491AA27879F9001869F210D27
:10BD60003A1F06942A1F3A1F112418C0FC01F695A9
:10BD7000E795EC7FED5AF64F459155916591749199
:10BD800087709927869F9001879F300D969F300D71
:10BD9000112463E0369527956A95E1F7421B530B12
:10BDA00050932901409328018091880D9091890D2D
:10BDB000A0918A0DB0918B0D840F951FA11DB11D0F
:10BDC0008093880D9093890DA0938A0DB0938B0D6D
:10BDD0007EC9452B31F481E090E09093A00D8093D3
:10BDE0009F0D8091800D9091810D909329018093FA
:10BDF00028018091820D8093830D69C91092B00D46
:10BE00001092AF0D9091B80D8091B70D981731F049
:10BE10008091B70D8F5F8F708093B70D9091B80DA3
:10BE20008091B70D981771F0C091B70D27E7C29FA9
:10BE3000E0011124C754D24FFE01EC58FF4F81E0BE
:10BE4000808302C0C0E0D0E0D093B00DC093AF0DAE
:10BE5000209709F464C3FE0120E030E0C08CD18C4F
:10BE6000E28CF38CA901440F551F440F551F445E0B
:10BE7000594EDA01CD92DD92ED92FC9213972F5F2D
:10BE80003F4F34962530310549F78AAD80937C0DBC
:10BE900080917D0D811111C01092880D1092890D35
:10BEA00010928A0D10928B0DFE01E25AFF4F808195
:10BEB00091819F3408F041C04CC04EE75DE0EBEA51
:10BEC000FDE0BE0120E030E0DB011C96CD90DD906E
:10BED000ED90FC901F97CD28CE28CF2819F1DA01DC
:10BEE0008C918823F9F0D901A755B24F8C91D901D3
:10BEF000AA0FBB1FAD5EB94E882341F08D919C9176
:10BF0000119700811181801B910B07C08D919C912D
:10BF1000119700811181800F911F11969C938E9330
:10BF2000DA011C922F5F3F4F6C5F7F4F4F5F5F4F77
:10BF300032962230310541F6AFCF9D3930F463E0BF
:10BF4000969587956A95E1F702C088E893E128E025
:10BF500014C0983230F0969587959695879524E091
:10BF60000CC0943120F09695879522E006C080326F
:10BF7000910510F480E290E021E02093830D8097FA
:10BF80008115B8E09B07B8F0E92FFF27EE0FFF1FE0
:10BF9000EE0FFF1FED5AF24F459155916591749147
:10BFA000AA27879F9001869F210D3A1F06942A1F7A
:10BFB0003A1F112418C0FC01F695E795EC7FED5A65
:10BFC000F64F459155916591749187709927869F99
:10BFD0009001879F300D969F300D112403E0369518
:10BFE00027950A95E1F7421B530B5093810D40931F
:10BFF000800D8091830D8093820DFE01EE58FF4FDE
:10C000008081882309F46DC0CA59DF4F88819981E6
:10C010009093870D8093860D9F3460F09D3930F4A6
:10C02000D3E096958795DA95E1F702C088E893E129
:10C0300028E014C0983230F09695879596958795AC
:10C0400024E00CC0943120F09695879522E006C03C
:10C050008032910510F480E290E021E02093830D7E
:10C0600080978115C8E09C07B8F0E92FFF27EE0FF5
:10C07000FF1FEE0FFF1FED5AF24F4591559165914D
:10C080007491AA27879F9001869F210D3A1F0694DD
:10C090002A1F3A1F112418C0FC01F695E795EC7F82
:10C0A000ED5AF64F45915591659174918770992796
:10C0B000869F9001879F300D969F300D112463E07D
:10C0C000369527956A95E1F7421B530BCA01A0E00C
:10C0D000B0E080938C0D90938D0DA0938E0DB09356
:10C0E0008F0D5093290140932801E091AF0DF091FD
:10C0F000B00D20AD2093940DEA58FF4F3081809110
:10C10000131690911416892B09F03360809115163F
:10C1100090911616892B09F034608091111638130E
:10C120001BC0C091AF0DD091B00D88819981AA81BB
:10C13000BB814C895D896E897F89FE01EB58FF4F79
:10C14000308111E00097A105B10509F410E01093CA
:10C150004C16111144C083C0A5E1B2E0E9E1F2E060
:10C1600080E090E061E070E0AB01082E01C0440F78
:10C170000A94EAF7C0911116C327C42349F1C32FCB
:10C18000C42350911116CC2391F0542B50931116C7
:10C19000CD91DC9111971881AB01008002C0440F52
:10C1A000551F0A94E2F740954123488311C04095FA
:10C1B000452340931116CD91DC9111971881AB0165
:10C1C000008002C0440F551F0A94E2F7142B188315
:10C1D00001969396B3968530910531F6A2CF122F32
:10C1E00011706A017B01F594E794D794C794F09499
:10C1F000E094D094C094C11CD11CE11CF11CC092ED
:10C200004D16D0924E16E0924F16F092501601E065
:10C21000311100E0009344164093451650934616A2
:10C220006093471670934816809355169093561650
:10C23000A0935716B0935816112311F08FEF01C039
:10C2400081E080934A1681E0812780934B161092FB
:10C2500051161092521610925316109254168C8149
:10C260009D81AE81BF814C895D896E897F8911E096
:10C270000097A105B10509F410E01093751611237C
:10C2800009F442C021FB112710F96A017B01F594E2
:10C29000E794D794C794F094E094D094C094C11CD0
:10C2A000D11CE11CF11CC0927616D0927716E09258
:10C2B0007816F092791601E0313009F000E0009331
:10C2C0006D1640936E1650936F16609370167093B0
:10C2D000711680937E1690937F16A0938016B0936C
:10C2E0008116112311F08FEF01C081E08093731646
:10C2F00081E081278093741610927A1610927B1633
:10C3000010927C1610927D1688859985AA85BB852A
:10C310004C895D896E897F8911E00097A105B1057F
:10C3200009F410E010939E16112309F442C022FB79
:10C33000112710F96A017B01F594E794D794C7940B
:10C34000F094E094D094C094C11CD11CE11CF11C69
:10C35000C0929F16D092A016E092A116F092A2165B
:10C3600001E0323009F000E00093961640939716F2
:10C37000509398166093991670939A168093A71607
:10C380009093A816A093A916B093AA16112311F0A2
:10C390008FEF01C081E080939C1681E0812780931C
:10C3A0009D161092A3161092A4161092A516109224
:10C3B000A6168C859D85AE85BF854C895D896E8965
:10C3C0007F8911E00097A105B10509F410E01093F1
:10C3D000C716112309F442C023FB112710F96A0183
:10C3E0007B01F594E794D794C794F094E094D094AB
:10C3F000C094C11CD11CE11CF11CC092C816D09283
:10C40000C916E092CA16F092CB1601E0333009F05B
:10C4100000E00093BF164093C0165093C11660937E
:10C42000C2167093C3168093D0169093D116A09322
:10C43000D216B093D316112311F08FEF01C081E013
:10C440008093C51681E081278093C6161092CC1682
:10C450001092CD161092CE161092CF168889998917
:10C46000AA89BB894C895D896E897F89F08131E019
:10C470000097A105B10509F430E03093F01633239D
:10C4800009F441C024FBEE27E0F98A019B013595B0
:10C4900027951795079530952095109501951F4F75
:10C4A0002F4F3F4F0093F1161093F2162093F3167F
:10C4B0003093F41621E0F43009F020E02093E816E0
:10C4C0004093E9165093EA166093EB167093EC16BE
:10C4D0008093F9169093FA16A093FB16B093FC166E
:10C4E000EE2311F08FEF01C081E08093EE1681E022
:10C4F0008E278093EF161092F5161092F616109272
:10C50000F7161092F8161092A00D10929F0D10922F
:10C51000900D1092910D1092920D1092930D81E05A
:10C520004AC0672F622330911116662399F0322B8F
:10C5300030931116CD91DC91119768819A0100809A
:10C5400002C0220F331F0A94E2F720952623288386
:10C550000C9402572095232320931116CD91DC9142
:10C56000119768819A01008002C0220F331F0A943C
:10C57000E2F7622B68830C940257109217160C9402
:10C58000AB59109218160C949D5A10921916C6C8E1
:10C5900010921A16B4C9A0919302B0919402FC9122
:10C5A000C9010090970202C0880F991F0A94E2F710
:10C5B000F82BFC938BCADF91CF911F910F91FF90C5
:10C5C000EF90DF90CF90BF90AF909F908F907F9033
:10C5D0006F905F904F9008957091950D7F5F70936D
:10C5E000950D8091960D8F5F8093960D5091990DCA
:10C5F0006091970D40E081E090E02091131630911A
:10C600001416232B61F47093950D50919A0D60913F
:10C61000980D7091960D40E081E090E02BC0751769
:10C6200090F346132EC0EFCF751708F4A9C0461734
:10C6300009F4A6C0E0919302F091940270819C01EC
:10C640000090970202C0220F331F0A94E2F7209550
:10C6500027232083209115163091161637FD93C09D
:10C660002091151630911616121613060CF4A7C059
:10C670004F5F70E02091151630911616232BA1F60E
:10C680007FC0E0917002F091710270819C01009076
:10C69000740202C0220F331F0A94E2F72095272369
:10C6A0002083209113163091141637FF1BC0309150
:10C6B000AC16E0917702F091780220917B0233234F
:10C6C00009F446C07081DC0102C0AA0FBB1F2A9585
:10C6D000E2F77A2B708320911316309114162F5F96
:10C6E0003F4F20C0209113163091141612161306D6
:10C6F00064F53091AC16E0917702F09178022091C8
:10C700007B02311131C07081DC0102C0AA0FBB1F56
:10C710002A95E2F77A2B7083209113163091141624
:10C72000215031093093141620931316E0917002B2
:10C73000F091710270819C010090740202C0220F7E
:10C74000331F0A94E2F7722B70834F5F70E055CF6E
:10C750007081DC0102C0AA0FBB1F2A95E2F79D0180
:10C76000209527232083B7CF7081DC0102C0AA0F58
:10C77000BB1F2A95E2F79D01209527232083CCCF6C
:10C780007093960D08953091D516E0919A02F0912C
:10C790009B0220919E02311141C07081DC0102C0D8
:10C7A000AA0FBB1F2A95E2F79D012095272320831E
:10C7B00020911516309116162F5F3F4F1BC03091F8
:10C7C000D516E0919A02F0919B0220919E023323AC
:10C7D00079F17081DC0102C0AA0FBB1F2A95E2F734
:10C7E0009D01209527232083209115163091161640
:10C7F000215031093093161620931516E0919302BB
:10C80000F091940270819C010090970202C0220F67
:10C81000331F0A94E2F7722B70832ACF7081DC01F8
:10C8200002C0AA0FBB1F2A95E2F77A2B7083C0CFF4
:10C830007081DC0102C0AA0FBB1F2A95E2F77A2B98
:10C840007083D2CF4F925F926F927F928F929F921E
:10C85000AF92BF92CF92DF92EF92FF920F931F930E
:10C86000CF93DF9310927C0D91EAC92E9DE0D92ED3
:10C8700025E9E22E2DE0F22EC7E9DDE039E9A32E0D
:10C880003DE0B32E00E010E099249394F60141902E
:10C890005190619071906F0183E0800F0E9419792F
:10C8A0009B01AC01C301B2010E94BFD59B01AC0149
:10C8B00060E070E48CE196E40E94E6D32B013C0139
:10C8C00020E030E040E85FE30E94BBD518163CF45E
:10C8D000C301B2010E94CFD32B013C010DC020E067
:10C8E00030E040E85FE3C301B2010E94E2D387FF7A
:10C8F00003C0412C512C3201C301B2010E948DD4DE
:10C90000862EF50161935F01662311F018820DC038
:10C91000A301920160E070E080E89FE30E94E6D30B
:10C920000E94CFD30E948DD468838881811101C079
:10C930009882F801EE0FFF1FED5EF94E1182108212
:10C94000F70181927F010F5F1F4F21960230110581
:10C9500009F09CCFDF91CF911F910F91FF90EF9045
:10C96000DF90CF90BF90AF909F908F907F906F900F
:10C970005F904F9008952091B80D9091B70D81E090
:10C98000291380E008950F931F93CF93DF93FB014A
:10C990007FB7F894EC0188819981AA81BB8180934B
:10C9A0001C1690931D16A0931E16B0931F1680811F
:10C9B0009181A281B3818093201690932116A09338
:10C9C0002216B0932316FA0180819181A281B3814E
:10C9D0008093241690932516A0932616B0932716BD
:10C9E000E90188819981AA81BB818093281690935F
:10C9F0002916A0932A16B0932B16F80180819181F5
:10CA0000A281B38180932C1690932D16A0932E169D
:10CA1000B0932F167FBFDF91CF911F910F91089593
:10CA20008F929F92AF92BF92EF92FF920F931F93BC
:10CA3000CF93DF93EFB7F89480901C1690901D165B
:10CA4000A0901E16B0901F16DC018D929D92AD92A3
:10CA5000BC9213978091201690912116A0912216D6
:10CA6000B0912316EB0188839983AA83BB838091BD
:10CA7000241690912516A0912616B0912716EA014A
:10CA800088839983AA83BB83809128169091291665
:10CA9000A0912A16B0912B16E90188839983AA8365
:10CAA000BB8380912C1690912D16A0912E16B091DB
:10CAB0002F16E80188839983AA83BB8380917C0D1C
:10CAC000D7018C93EFBFDF91CF911F910F91FF9012
:10CAD000EF90BF90AF909F908F90089580917300DA
:10CAE0008D7F809373009091B80D8091B70D98134E
:10CAF0005DC01092B00D1092AF0D2FB7F8948091D9
:10CB00001C1690911D16A0911E16B0911F168093B1
:10CB1000521590935315A0935415B09355158091C9
:10CB2000201690912116A0912216B0912316809381
:10CB3000561590935715A0935815B0935915809199
:10CB4000241690912516A0912616B0912716809351
:10CB50005A1590935B15A0935C15B0935D15809169
:10CB6000281690912916A0912A16B0912B16809321
:10CB70005E1590935F15A0936015B0936115809139
:10CB80002C1690912D16A0912E16B0912F168093F1
:10CB9000621590936315A0936415B09365152FBF2C
:10CBA0008091730082608093730008959091B80D16
:10CBB0008091B70D981709F496CF8091B70D8F5FCC
:10CBC0008F708093B70D8FCF80937D0D81E0809320
:10CBD0007E0D80937F0D089540E063E97AE181EB5B
:10CBE0009DE00C94F4CE9C0190EC80E4889410F0CD
:10CBF000381710F0381B892B9695220F331F892781
:10CC00009E7FA9F710F0220F8307891F08952F92A6
:10CC10003F924F925F926F927F928F929F92AF92CC
:10CC2000BF92CF92DF92EF92FF920F931F93CF9319
:10CC3000DF93CDB7DEB768970FB6F894DEBF0FBEAF
:10CC4000CDBF1C01F901310122E7620E711CD30135
:10CC50002C912223A9F09A01AB0121303105B1E0DA
:10CC60004B07510524F020E030E041E050E048015E
:10CC70005F01E1E08E169104AE06B1044CF004C0F1
:10CC800020E030E041E050E0812C912C5401A3944D
:10CC90007101FEE5EF0EF11CF70180819181A28107
:10CCA000B381772766270E944CD270588F4F9F4FD1
:10CCB0008C01332717FD3095232F0D831E832F837F
:10CCC0003887F70180819181A281B3817727662718
:10CCD000A50194010E944CD270588F4F9F4F7C0148
:10CCE0001127F7FC1095012FE986FA860B871C8720
:10CCF0000D811E812F8138850837110521053105E9
:10CD000048F418E7E12EF12C00E010E0ED82FE82FD
:10CD10000F83188709851A852B853C8508371105EF
:10CD20002105310548F418E7E12EF12C00E010E070
:10CD3000E986FA860B871C872D813E814F815885B5
:10CD4000CA01B9010E9422D669837A838B839C83AE
:10CD500029853A854B855C85CA01B9010E9422D696
:10CD60006D877E878F87988B910122593F4FD9011C
:10CD7000ED90FD900D911C91ED8AFE8A0F8B188F1E
:10CD800067017801CC0CDD1CEE1CFF1CF3018081D7
:10CD90008823B9F1F101EE59FF4F80809180A28084
:10CDA000B380C114D104E104F10489F0C501B401D8
:10CDB00009811A812B813C81601B710B820B930BC3
:10CDC000A70196010E9488D629013A0103C0412C8F
:10CDD000512C320122273327A9012C193D094E0974
:10CDE0005F09B9F06D857E858F8598896819790905
:10CDF0008A099B090E9488D6298B3A8B4B8B5C8BC6
:10CE00000CC0198A1A8A1B8A1C8A412C512C3201A7
:10CE100004C0198A1A8A1B8A1C8AD10154968D90E3
:10CE20009D90AD90BC905797D501C4018419950988
:10CE3000A609B70909891A892B893C89801B910B9E
:10CE4000A20BB30BB7FF3BC0C114D104E104F10442
:10CE5000F9F0A7019601C501B4010E9422D609810B
:10CE60001A812B813C81601B710B820B930B0D850A
:10CE70001E852F853889600F711F821F931FA701A0
:10CE80009601220F331F441F551F0E9488D604C0ED
:10CE900020E030E040E050E0C901DA01B7FF03C014
:10CEA00080E090E0DC012C013D0188169906AA067D
:10CEB000BB0614F42401350180E090E0DC0183011D
:10CEC0007201E80EF91E0A1F1B1FED86FE860F87F2
:10CED000188BF10123AD222309F41EC1892B8A2B63
:10CEE0008B2B09F079C0A30192012F5F3F4F4F4F69
:10CEF0005F4F57FF22C050954095309521953F4F89
:10CF00004F4F5F4F6D897E898F89988D0E9422D601
:10CF1000660F771F881F991FE980FA800B811C819B
:10CF20006E157F058007910708F04DC0E61AF70AD5
:10CF3000080B190BD801C70114C06D897E898F8930
:10CF4000988D0E9422D6DC01CB01880F991FAA1F61
:10CF5000BB1F09811A812B813C81800F911FA21F69
:10CF6000B31F811510E89107A105B10558F40E947F
:10CF7000F3656C01EE24D7FCE094FE2C7601DD24F1
:10CF8000CC2424C010E022E0B695A795979587950C
:10CF90002A95D1F71F5F811520E89207A105B105F9
:10CFA00090F70E94F3656C01EE24D7FCE094FE2C10
:10CFB0007601DD24CC2404C0CC0CDD1CEE1CFF1C4F
:10CFC0001A95D2F703C0C12CD12C76016701FF243A
:10CFD000D7FCF094EF2C07C0F101E25AFF4FC0805C
:10CFE000D180E280F3801414150416041704D4F4DD
:10CFF000D701C6010D811E812F813885801B910BC1
:10D00000A20BB30BAC01332722276091B9157091A5
:10D01000BA158091BB159091BC150E944CD25C0151
:10D0200097FF02C0A12CB12CF10184899589A689B2
:10D03000B7894D855E856F8578894F5F5F4F6F4FEC
:10D040007F4F481759076A077B070CF06DC00985A9
:10D050001A852B853C85C01AD10AE20AF30AA6017B
:10D06000332722276091B9157091BA158091BB15AD
:10D070009091BC150E944CD27C011127F7FC1095B1
:10D08000012FE982FA820B831C838091B515909160
:10D09000B615A091B715B091B815892B8A2B8B2B9B
:10D0A00099F1E988FA880B891C89A701332722277F
:10D0B000F101E259FF4F80819181A281B38165E046
:10D0C000B595A795979587956A95D1F777276627A0
:10D0D0000E94BBD26B017C016091B5157091B615B1
:10D0E0008091B7159091B81520E030E044E650E00B
:10D0F0000E944CD2A70196010E944CD2BB2797FDFB
:10D10000B095AB2FB7FF03C080E090E0DC01498110
:10D110005A8157FF0EC00BC080E090E0DC0140E078
:10D1200050E0A12CB12C05C080E090E0DC0140E093
:10D1300050E02FB7F894F101EC58FF4F30813111D6
:10D1400039C032973081332369F0F10144A655A6E6
:10D1500066A677A6ED84FE840F851889E0AAF1AA59
:10D1600002AB13ABB1016A597F4FED80FE800F8196
:10D170001885FB01E082F182028313836C5F7F4F8D
:10D18000E984FA840B851C85FB01E082F18202832D
:10D190001383F101B5AEA4AE57AF46AFEC5BFF4FC2
:10D1A0001182108232961182108236978083918389
:10D1B000A283B3832FBF68960FB6F894DEBF0FBE6D
:10D1C000CDBFDF91CF911F910F91FF90EF90DF9036
:10D1D000CF90BF90AF909F908F907F906F905F9017
:10D1E0004F903F902F9008952F923F924F925F92D1
:10D1F0006F927F928F929F92AF92BF92CF92DF9267
:10D20000EF92FF920F931F93CF93DF93CDB7DEB7CB
:10D210002C970FB6F894DEBF0FBECDBF9C878B87CF
:10D22000009709F49DC16115710509F499C11C01AC
:10D2300020E5220E311CD1018D919D910D90BC9164
:10D24000A02D89839A83AB83BC830B851C85045BEB
:10D250001F4FF80180819181A281B38129813A8198
:10D260004B815C8182179307A407B50709F478C145
:10D27000EB85FC85E35AFF4F808181115BC1FB0187
:10D28000ED58FF4F8081882309F454C1AB01445B02
:10D290005F4F5E834D83FA0180819181A281B381CA
:10D2A00029813A814B815C8182179307A407B507D6
:10D2B0000CF040C1BC01CD01ECE0959587957795C8
:10D2C0006795EA95D1F74B855C85485A5F4F58873B
:10D2D0004F83DA018D909D90AD90BC90B094A09456
:10D2E00090948094811C911CA11CB11CF6E0B59413
:10D2F000A79497948794FA95D1F7EB85FC85EC5A1F
:10D30000FF4FFA87E987C080D180E280F380A5E0F3
:10D31000F594E794D794C794AA95D1F79B01AC01F3
:10D320000E944CD22B013C01A5019401C701B6011A
:10D330000E944CD2461A570A680A790A20E0411422
:10D3400051046104710409F44AC0D301C201882761
:10D350009927AA27B07E892B8A2B8B2B49F472E060
:10D36000440C551C661C771C7A95D1F72F5FE7CFCC
:10D37000141415041604170494F5C301BB2797FD74
:10D38000B095AB2FE22EF12C2730A0F00E94F36570
:10D39000AA2797FDA095BA2FDC0199278827F6E0E8
:10D3A000EF1AF10804C0B595A79597958795EA946B
:10D3B000D2F718C00E94F365AA2797FDA095BA2F4F
:10D3C000DC019927882726E030E02E193F0904C0A8
:10D3D000880F991FAA1FBB1F2A95D2F703C080E0B0
:10D3E00090E0DC0129813A814B815C812817390763
:10D3F0004A075B0734F4F10180819181A281B381F6
:10D4000093C0AD81BE816D917D918D919C91BCE069
:10D410009595879577956795BA95D1F7EF81F885BA
:10D4200080809180A280B380B094A09490948094E6
:10D43000811C911CA11CB11C26E0B594A794979463
:10D4400087942A95D1F7A985BA85CD90DD90ED9086
:10D45000FC9035E0F594E794D794C7943A95D1F7CA
:10D460009B01AC010E944CD22B013C01A50194010F
:10D47000C701B6010E944CD2461A570A680A790AB7
:10D4800020E0411451046104710409F44AC0D3013D
:10D49000C20188279927AA27B07E892B8A2B8B2B3C
:10D4A00049F4A2E0440C551C661C771CAA95D1F7E0
:10D4B0002F5FE7CF141415041604170494F5C30165
:10D4C000BB2797FDB095AB2FE22EF12C2730A0F0B3
:10D4D0000E94F365AA2797FDA095BA2FDC01992732
:10D4E0008827E6E0EE1AF10804C0B595A795979550
:10D4F0008795EA94D2F718C00E94F365AA2797FD92
:10D50000A095BA2FDC019927882726E030E02E1954
:10D510003F0904C0880F991FAA1FBB1F2A95D2F785
:10D5200003C080E090E0DC01F80180839183A28356
:10D53000B38310C029813A814B815C81D8012D933E
:10D540003D934D935C93139781E0EB85FC85ED58FB
:10D55000FF4F8083EB85FC85E45AFF4F81E0808399
:10D560002C960FB6F894DEBF0FBECDBFDF91CF91E2
:10D570001F910F91FF90EF90DF90CF90BF90AF90F1
:10D580009F908F907F906F905F904F903F902F90E3
:10D590000895FF920F931F93CF93DF931091B80DCF
:10D5A0008FB7F8940091B70D8FBF60E070E0B7E7D8
:10D5B000FB2E101771F0111101C010E11150F19EF6
:10D5C000E0011124C754D24FCE010E94F468BE017D
:10D5D000F0CFDF91CF911F910F91FF9008952F927F
:10D5E0003F924F925F926F927F928F929F92AF92F3
:10D5F000BF92CF92DF92EF92FF920F931F93CF9340
:10D60000DF93CDB7DEB72A970FB6F894DEBF0FBE13
:10D61000CDBF9C017A876987009709F46BC1FB0134
:10D62000EE58FF4F8081882309F464C1F901E35A61
:10D63000FF4F808181115EC176968081882309F435
:10D6400059C119014CE4240E311CF10180819181F2
:10D65000A281B3818B01045B1F4FF8014080518090
:10D660006280738084159505A605B7050CF042C14C
:10D67000BC01CD01ECE09595879577956795EA9586
:10D68000D1F7A901485A5F4F5A834983FA01808034
:10D690009180A280B380F6E0B594A7949794879484
:10D6A000FA95D1F7445051095C834B83FA01C0804D
:10D6B000D180E280F380A5E0F594E794D794C794F5
:10D6C000AA95D1F79B01AC010E944CD26D837E8359
:10D6D0008F839887A5019401C701B6010E944CD29F
:10D6E0002D813E814F815885620F731F841F951FC6
:10D6F00020E0611571058105910509F44AC06B01AF
:10D700007C01CC24DD24EE2430EEF322CD28CE287B
:10D71000CF2849F452E0660F771F881F991F5A954A
:10D72000D1F72F5FE6CF16161706180619068CF5E7
:10D73000BB2797FDB095AB2FE22EF12C2730A0F040
:10D740000E94F365AA2797FDA095BA2FDC019927BF
:10D75000882746E0E41AF10804C0B595A795979587
:10D760008795EA94D2F718C00E94F365AA2797FD1F
:10D77000A095BA2FDC019927882726E030E02E19E2
:10D780003F0904C0880F991FAA1FBB1F2A95D2F713
:10D7900003C080E090E0DC01481659066A067B066B
:10D7A00034F4F80180819181A281B3818AC0F101B2
:10D7B0006081718182819381ECE095958795779561
:10D7C0006795EA95D1F7E981FA8180809180A280FE
:10D7D000B380F6E0B594A79497948794FA95D1F71F
:10D7E000EB81FC81C080D180E280F380A5E0F594DC
:10D7F000E794D794C794AA95D1F79B01AC010E94F6
:10D800004CD22B013C01A5019401C701B6010E9435
:10D810004CD2640D751D861D971D20E061157105A4
:10D820008105910509F44AC06B017C01CC24DD24FB
:10D83000EE24F0EEFF22CD28CE28CF2849F452E086
:10D84000660F771F881F991F5A95D1F72F5FE6CF74
:10D8500016161706180619068CF5BB2797FDB09506
:10D86000AB2FE22EF12C2730A0F00E94F365AA27FF
:10D8700097FDA095BA2FDC019927882726E0E21AA8
:10D88000F10804C0B595A79597958795EA94D2F7C6
:10D8900018C00E94F365AA2797FDA095BA2FDC0156
:10D8A0009927882726E030E02E193F0904C0880F09
:10D8B000991FAA1FBB1F2A95D2F703C080E090E0F2
:10D8C000DC01F80140815181628173814817590759
:10D8D0006A077B0779F080839183A283B383E9850C
:10D8E000FA85E45AFF4F81E08083E985FA85ED5897
:10D8F000FF4F80832A960FB6F894DEBF0FBECDBFD0
:10D90000DF91CF911F910F91FF90EF90DF90CF901B
:10D91000BF90AF909F908F907F906F905F904F904F
:10D920003F902F9008950F931F93CF93DF93109103
:10D93000B70D80E090E007E72091B80D121771F065
:10D94000019FE0011124C754D24FBE010E94EF6A2B
:10D950001F5F103109F410E0CE01EECFDF91CF91BF
:10D960001F910F9108954F925F926F927F928F92C5
:10D970009F92AF92BF92CF92DF92EF92FF920F935E
:10D980001F93CF93DF939090B70DC0E0D0E0B7E73F
:10D990008B2E8091B80D981609F454C0899C7001A3
:10D9A0001124C7018754924F7C01209709F443C08A
:10D9B000FE01EE58FF4F80818823E9F1F701EE5810
:10D9C000FF4F80818823B9F16E019CE5C90ED11CFF
:10D9D000F6018081811106C0F701E45AFF4F808172
:10D9E000882349F15E01F8E4AF0EB11CF5012081F6
:10D9F000318142815381F701E45BFF4F6081718186
:10DA0000828193810E94BBD22B013C01F5012081D0
:10DA10003181428153813496608171818281938109
:10DA20000E94BBD2AB01BC0193018201CE010E94D6
:10DA30000766F60110829394F0E19F1201C0912CC9
:10DA4000E701A7CF2097C1F0FE01E85BFF4F2081DF
:10DA500031814281538134966081718182819381C9
:10DA60000E94BBD2AB01BC018A019B01CE010E9486
:10DA70000766C45ADF4F1882DF91CF911F910F9133
:10DA8000FF90EF90DF90CF90BF90AF909F908F90DE
:10DA90007F906F905F904F9008950E94C96A0E9496
:10DAA000936C0C94B36C0F931092B80D1092B70D49
:10DAB000109252151092531510925415109255153C
:10DAC000109256151092571510925815109259151C
:10DAD00010925A1510925B1510925C1510925D15FC
:10DAE00010925E1510925F151092601510926115DC
:10DAF00010926215109263151092641510926515BC
:10DB00006093B9157093BA158093BB159093BC15AB
:10DB10002093B5153093B6154093B7155093B815AB
:10DB20000093291581E0809306020F9108952F92AA
:10DB30003F924F925F926F927F928F929F92AF929D
:10DB4000BF92CF92DF92EF92FF920F931F93CF93EA
:10DB5000DF93CDB7DEB7E8970FB6F894DEBF0FBE00
:10DB6000CDBF4B015C015CA34BA33EA32DA38091D1
:10DB7000D1159091D215892B41F09091B80D8091DB
:10DB8000B70D981711F40C94DB751091B80D1F5F49
:10DB90001AA7103109F41AA68091B80D27E7829FC1
:10DBA00010011124A1014754524F1A01FA01EC58F7
:10DBB000FF4F108232970083DA01DA96EC928FB72A
:10DBC000F894DA01E2E5F5E14191519161917191A9
:10DBD00058964D935D936D937C935B97149605E1F6
:10DBE000E636F00789F78FBF409084155090851571
:10DBF0006090861570908715D1014D925D926D925F
:10DC00007C921397009188151091891520918A159F
:10DC100030918B150F8B188F298F3A8F14960D9397
:10DC20001D932D933C93179700918C1510918D1592
:10DC300020918E1530918F150F8F18A329A33AA329
:10DC400018960D931D932D933C931B97409190151F
:10DC5000509191156091921570919315F10144873F
:10DC60005587668777878091941590919515A09137
:10DC70009615B0919715808B918BA28BB38B0091E9
:10DC8000991510919A1520919B1530919C15048B34
:10DC9000158B268B378B20919815EB58FF4F2083DF
:10DCA0004114510461047104D9F40F89188D298D30
:10DCB0003A8D012B022B032B99F40F8D18A129A16A
:10DCC0003AA1012B022B032B59F441155105610593
:10DCD000710541F411E019A70097A105B10521F4E0
:10DCE00019A602C021E029A7F10110AEC0903E158F
:10DCF000D0903F15E0904015F090411500915215DD
:10DD0000109153152091541530915515C016D10618
:10DD1000E206F30614F421E020AFC0904215D09043
:10DD20004315E0904415F09045150091561510915B
:10DD300057152091581530915915C016D106E20695
:10DD4000F30624F4F10120AD226020AFC090461507
:10DD5000D0904715E0904815F090491500915A155C
:10DD600010915B1520915C1530915D15C016D106A0
:10DD7000E206F30624F4F10120AD246020AFC09048
:10DD80004A15D0904B15E0904C15F0904D15009130
:10DD90005E1510915F152091601530916115C016C8
:10DDA000D106E206F30624F4F10120AD286020AF8D
:10DDB000C0904E15D0904F15E0905015F090511531
:10DDC00000916215109163152091641530916515CD
:10DDD000C016D106E206F30624F4F10120AD20615D
:10DDE00020AF411551056105710539F00097A10576
:10DDF000B10549F4F10111AE0BC00097A105B105C1
:10DE000011F021E003C0EDA1FEA12081F10121AFBD
:10DE100045284628472829F0209112162160209392
:10DE200012160F89188D298D3A8D012B022B032B89
:10DE300029F0209112162260209312160F8D18A13E
:10DE400029A13AA1012B022B032B29F020911216B4
:10DE5000246020931216452B462B472B29F0209146
:10DE60001216286020931216892B8A2B8B2B29F0EF
:10DE70008091121680618093121680911216F10122
:10DE8000EA58FF4F808390912915992311F08460FF
:10DE900080836091B80D8091B70D681B6F70262F3D
:10DEA00030E038A32F8F232B41F510922A151092C2
:10DEB0002B1510922C1510922D1510922E151092D4
:10DEC0002F151092301510923115109232151092B4
:10DED0003315109234151092351510923615109294
:10DEE0003715109238151092391510923A15109274
:10DEF0003B1510923C1510923D15EBA1FCA18081C1
:10DF00009181A281B3818101025A1F4F188F0F8B1B
:10DF1000F80180839183A283B3832091D11530913E
:10DF2000D2152115310509F444C0809106028823D9
:10DF300041F00F8D18A102171307DCF110920602B1
:10DF400038C04F8D58A1421753079CF542305105F8
:10DF500084F1C901AA2797FDA095BA2FAC013327F8
:10DF60002227862F90E0A0E0B0E0772766270E9466
:10DF7000BBD26B017C019B01AC01C501B4010E94C5
:10DF80004CD24B015C01EF89F88D80819181A28197
:10DF9000B38177276627A70196010E944CD2BB2741
:10DFA00097FDB095AB2FEF89F88D80839183A28385
:10DFB000B38381149104A104B10409F45CC0F1019C
:10DFC000EC5AFF4F09A50023C1F0D101D9969C91CD
:10DFD00004E0909FD0011124A355BA4E8D919D91DC
:10DFE0000D90BC91A02DB7FF10C0B095A095909555
:10DFF00081959F4FAF4FBF4F08C080919D15909165
:10E000009E15A0919F15B091A01580839183A28346
:10E01000B383208131814281538160E070E081E0EF
:10E0200090E00E94BBD26B017C019B01AC01C50159
:10E03000B4010E944CD22B013C0101EA15E19E0182
:10E040002F5F3F4F3EA32DA3D8016D917D918D9100
:10E050009D918D01A30192010E944CD2EDA1FEA1E0
:10E060006193719381939193FEA3EDA3F5E1053B39
:10E070001F0751F703C0C12CD12C7601F101EE58D6
:10E08000FF4F80818111D4C0EBA1FCA180819181DF
:10E09000A281B381EF89F88D80839183A283B383BA
:10E0A00089288A288B2809F485C08E010F5F1F4FAD
:10E0B000580107ED15E14E0125E1820E911C412C1E
:10E0C000512C32016394D501CD90DD90ED90FD90FF
:10E0D0005D01F7FE08C0F094E094D094C094C11C98
:10E0E000D11CE11CF11CF801608171818281938156
:10E0F0006C157D058E059F05A4F4A70196010E946D
:10E10000BBD246165706680679065CF0D8016D91B9
:10E110007D918D919C91A70196010E94BBD22B010C
:10E120003C010C5F1F4FA814B90469F6EBA1FCA1D8
:10E1300080819181A281B38181159048A105B105AB
:10E1400018F1EF89F88D80819181A281B38124E05B
:10E15000B695A795979587952A95D1F78083918352
:10E16000A283B38377276627A30192010E944CD232
:10E17000BB2797FDB095AB2F54E0880F991FAA1FBE
:10E18000BB1F5A95D1F710C0EF89F88D808191811E
:10E19000A281B38177276627A30192010E944CD206
:10E1A000BB2797FDB095AB2FEF89F88D80839183C6
:10E1B000A283B383D1019C961D921D921D921C9245
:10E1C0009F9754968D919D910D90BC91A02D019695
:10E1D000A11DB11DF10180AB91ABA2ABB3ABAF8977
:10E1E000B88D6D917D918D919C91EE59FF4F9B0162
:10E1F000AC010E9422D66083718382839383BAA587
:10E20000B093B80D4FB7F894EEE3F5E122E535E1B0
:10E21000C190D190E190F190D901CD92DD92ED9233
:10E22000FD929D01B5E1E235FB0791F74FBFEEC4CA
:10E23000E9A5E11135C00F8D18A1012B89F5809159
:10E24000661590916715A0916815B091691518161B
:10E2500019061A061B0624F581010C5A1F4FD80116
:10E260006D917D918D919C911616170618061906D1
:10E27000BCF4181419041A041B0494F4A5019401A5
:10E280000E94BBD2209166153091671540916815A8
:10E290005091691562177307840795070CF490C4B1
:10E2A000EF89F88D6081718182819381F101EE594E
:10E2B000FF4F9B01AC010E9422D660837183828351
:10E2C00093837A9780829182A282B382F1018489BA
:10E2D0009589A689B7898115F0E89F07A105B10541
:10E2E00068F0A7019601220F331F441F551FB595F3
:10E2F000A795979587957727662704C07727662780
:10E30000A70196010E944CD22B013C01F101E25978
:10E31000FF4F9C01552737FD5095452F09A5002338
:10E3200079F06091EF157091F0158091F115909151
:10E33000F2150E9422D66083718382839383CEC0BC
:10E340006091F3157091F4158091F5159091F61583
:10E350000E9422D660837183828393832DEB35E103
:10E360003CA32BA34CE655E15EA74DA738AE2FAAE0
:10E37000FCA7EBA7AFA9B8AD6D917D918D919D9153
:10E38000B8AFAFAB6F8B788F898F9A8F672B682B65
:10E39000692B09F494C0D10154960D911D912D91D2
:10E3A0003C9157970FA718AB29AB3AABEDA5FEA54B
:10E3B0004081518162817381ABA1BCA1401751079B
:10E3C0006207730728F1CD90DD90ED90FC90EBA5EE
:10E3D000FCA560817181828193812F89388D498D5F
:10E3E0005A8D0E9422D64B015C01A70196016FA5B0
:10E3F00078A989A99AA90E9422D6681579058A0563
:10E400009B0508F05CC0C082D182E282F38257C0D3
:10E410000D911D912D913C910BAB1CAB2DAB3EABE7
:10E420000F89188D298D3A8D330F000B102F98010D
:10E430000DA31EA32FA338A7ABA5BCA50D911D91BD
:10E440002D913C9158016901E12CF12C00E010E084
:10E450002F89388D498D5A8D6DA1762F862F962F55
:10E460000E94CED679018A016F8B7DA34C016BA9E6
:10E470007CA98DA99EA92FA538A949A95AA90E94AE
:10E4800027D759016A01B62FA72FF82FE92F970137
:10E49000A8016F897DA1C401EB2EFA2E0F2F1E2F2C
:10E4A0000E946DD861F058F00BA91CA92DA93EA9B6
:10E4B000ABA5BCA50D931D932D933C931397EBA196
:10E4C000FCA13496FCA3EBA30DA51EA50C5F1F4F6A
:10E4D0001EA70DA7E15DF54109F04CCF71012EE6B5
:10E4E000E20EF11CF70180819181A281B38181014B
:10E4F000085A1F4F8115F0E89F07A105B10528F4C0
:10E5000077276627A301920117C0A3019201009704
:10E51000E2E0AE07B105C8F4E2E0559547953795BE
:10E520002795EA95D1F7F2E0B595A7959795879548
:10E53000FA95D1F7772766270E94BBD2D8016D9351
:10E540007D938D939C9313972BC00097E8E0AE07C3
:10E55000B10578F4F4E05595479537952795FA95E8
:10E56000D1F764E0B595A795979587956A95D1F70A
:10E57000E1CF65E055954795379527956A95D1F791
:10E5800075E0B595A795979587957A95D1F77727F3
:10E5900066270E94BBD2F8016083718382839383D4
:10E5A000F70180819181A281B3818C019D0140E0BE
:10E5B00050E0BA018F8B188F298F3A8F4B8F5C8F69
:10E5C0006D8F7E8F9C01498D5A8D60E070E080E0F8
:10E5D00090E002E00E942DD8AF88B12EC98CDA8C71
:10E5E000E12CF12C00E010E00E9464D859016A018E
:10E5F0007B01E82F192F04E00E942DD80E2F0E94D6
:10E6000064D802E00E942DD8AF88B88CC98CDA8C0F
:10E61000E12CF12C00E010E00E9464D859016A015D
:10E620007B01E82F192F02E00E942DD80E2F0E94A7
:10E6300064D803E00E942DD8AF88B88CC98CDA8CDE
:10E64000E12CF12C00E010E00E9464D805E00E946B
:10E650002DD800E00E9464D80EE00E9446D8D10177
:10E66000D4962C93D497D5963C93D597D6964C9325
:10E67000D697D7965C938101085B1F4F188F0F8B3D
:10E680002F8D38A1232BD1F46091D3157091D4151F
:10E690008091D5159091D615609380157093811552
:10E6A0008093821590938315D8012D913D914D91C2
:10E6B0005C910E94BBD22B013C01D5C0EF89F88D43
:10E6C00080819181A281B3814091EB155091EC152D
:10E6D0006091ED157091EE15481759076A077B0791
:10E6E0006CF08093801590938115A0938215B09360
:10E6F0008315412C512C32016394B5C007ED15E10F
:10E7000018A30F8F8E010B5E1F4F1E8B0D8B0AE21D
:10E7100015E11CA30BA38E010F5F1F4F412C512C41
:10E7200032016394D8012D913D914D915D918D0100
:10E73000EBA1FCA181919191A191B191FCA3EBA3DB
:10E740002115310541055105D9F1EF8DF8A1C080A2
:10E75000D180E280F38049015A01881A990AAA0AF5
:10E76000BB0AB7FE08C0B094A09490948094811C1A
:10E77000911CA11CB11CC814D904EA04FB0404F5C3
:10E7800082179307A407B5073CF4BC01CD016C0DBB
:10E790007D1D8E1D9F1D06C0BC01CD016C197D091C
:10E7A0008E099F090E94BBD2161617061806190675
:10E7B000D4F4641575058605970514F42B013C0106
:10E7C0002F8D38A12C5F3F4F38A32F8F4D895E8945
:10E7D0000417150709F0A6CF4114510451E065064E
:10E7E000710499F103C0412C512C3201AF89B88DCD
:10E7F0006D917D918D919C91A30192010E944CD2CB
:10E800006093801570938115809382159093831582
:10E810001AE2E12E15E1F12E8E010F5F1F4FF80174
:10E8200061917191819191918F01A30192010E9457
:10E830004CD2D7016D937D938D939D937D01ED898E
:10E84000FE890E171F0759F71FC0EF89F88D8081C9
:10E850009181A281B3818093801590938115A093BB
:10E860008215B0938315FE013196AAE2B5E1CE017F
:10E87000459641915191619171914D935D936D9345
:10E880007D93E817F907A9F76091D3157091D41516
:10E890008091D5159091D615ECE095958795779553
:10E8A0006795EA95D1F7F101E85AFF4F8080918092
:10E8B000A280B380A6E0B594A79497948794AA9574
:10E8C000D1F73497C080D180E280F380B5E0F59431
:10E8D000E794D794C794BA95D1F79B01AC010E94F5
:10E8E0004CD26F8B788F898F9A8FA5019401C701C5
:10E8F000B6010E944CD20F89188D298D3A8D600F78
:10E90000711F821F931F40E06115710581059105FC
:10E9100009F448C08B019C01002711272227307E73
:10E92000012B022B032B49F452E0660F771F881F3F
:10E93000991F5A95D1F74F5FE7CF1616170618069D
:10E94000190684F5BB2797FDB095AB2F042F10E077
:10E95000473098F00E94F365AA2797FDA095BA2F3B
:10E96000DC01992788270650110904C0B595A795A1
:10E97000979587950A95D2F718C00E94F365AA2744
:10E9800097FDA095BA2FDC019927882726E030E073
:10E99000201B310B04C0880F991FAA1FBB1F2A958B
:10E9A000D2F703C080E090E0DC01409180155091E7
:10E9B00081156091821570918315C090D315D09008
:10E9C000D415E090D515F090D6159101245B3F4FFA
:10E9D0008101005B1F4FF9014C155D056E057F0538
:10E9E00054F4C082D182E282F382F801C082D182E3
:10E9F000E282F38209C04083518362837383F8010A
:10EA00004083518362837383F101E85BFF4F408150
:10EA1000518162817381759684179507A607B707A0
:10EA20001CF081E0808301C0108281E0F101E45A92
:10EA3000FF4F808377961082F397108211821282A3
:10EA40001382F10184859585A685B785892B8A2B4C
:10EA50008B2B41F480899189A289B389892B8A2BD8
:10EA60008B2BD9F0F9A5F11118C08091B9159091AF
:10EA7000BA15A091BB15B091BC15892B8A2B8B2B95
:10EA800009F58091B5159091B615A091B715B09183
:10EA9000B815892B8A2B8B2BA9F4D101DB961C92FC
:10EAA000DB97DD961C921E92DC97DF961C921E92DD
:10EAB000DE97F101EC5BFF4F1182108232961182DA
:10EAC000108203C081E0F10183AF93018201B301A1
:10EAD000A201C1010E940766FAA5F093B80D4FB7D5
:10EAE000F894EEE3F5E122E535E1C190D190E190B3
:10EAF000F190D901CD92DD92ED92FD929D01B5E1AB
:10EB0000E235FB0791F74FBF0E944D6DF101808503
:10EB10009185A285B385892B8A2B8B2B09F476C02E
:10EB200080916B15882309F471C020916A1580E9E2
:10EB300091E0289FA001299F500D1124662757FDC1
:10EB40006095762F8091461590914715A0914815B4
:10EB5000B091491584179507A607B7070CF456C05E
:10EB600010926B1587E090E00E9435A481EE9AE048
:10EB70000E94AFA489E090E00E9435A461E070E0BB
:10EB800081E0E8960FB6F894DEBF0FBECDBFDF91EF
:10EB9000CF911F910F91FF90EF90DF90CF90BF909A
:10EBA000AF909F908F907F906F905F904F903F902D
:10EBB0002F900C94703C81E0809306020C94C56DFC
:10EBC000D8016D917D918D919C910E94BBD23B01AA
:10EBD0008C01A50194010E94BBD29B01AC01EF897D
:10EBE000F88D80819181A281B381772766270E9469
:10EBF0004CD2BB2797FDB095AB2FEF89F88D808362
:10EC00009183A283B383430158014ACBE8960FB6A0
:10EC1000F894DEBF0FBECDBFDF91CF911F910F9152
:10EC2000FF90EF90DF90CF90BF90AF909F908F902C
:10EC30007F906F905F904F903F902F9008958093BA
:10EC40006B1560E080E592E00E94009E80936A155B
:10EC5000089580916B15089580936B1508950F9317
:10EC60001F93CF93CFB7F894FC0180819181A2814B
:10EC7000B3818093521590935315A0935415B0937C
:10EC80005515FB0180819181A281B3818093561536
:10EC900090935715A0935815B0935915FA01808198
:10ECA0009181A281B38180935A1590935B15A093B3
:10ECB0005C15B0935D15F90180819181A281B381CA
:10ECC00080935E1590935F15A0936015B0936115C6
:10ECD000F80180819181A281B38180936215909324
:10ECE0006315A0936415B09365158091B80D90914C
:10ECF000B70D891B8F7061F402E615E12EE535E151
:10ED00004AE555E166E575E182E595E10E94C36457
:10ED1000CFBFCF911F910F91089540E063E97AE151
:10ED20008BE096E10C94F4CE2F923F924F925F923B
:10ED30006F927F928F929F92AF92BF92CF92DF920B
:10ED4000EF92FF920F931F93CF93DF93CDB7DEB770
:10ED500067970FB6F894DEBF0FBECDBF898B8823AF
:10ED6000B1F060E082E090E00E94009EF82E60E04A
:10ED700084E090E00E94009E8E8360E08EE092E04E
:10ED80000E94009E813729F00E94C03702C01E8277
:10ED9000F12C40E356E15F8B4E8B07E012E080E2FE
:10EDA00092E09A838983A2E1B2E0B887AF83EBE077
:10EDB000F2E0FA87E98749E152E05D834C8397E20C
:10EDC000292E92E0392E8FE793E09C878B87A6E46B
:10EDD000B2E0BE87AD87A12CB12C812C912CC12C27
:10EDE000D12CEF2DF0E0FB8BEA8BEE24E394F12C99
:10EDF0005E81452F50E05D8B4C8BCB8289898823C7
:10EE000009F490C19E8197FF0AC08C899D890C2CC2
:10EE100002C0959587950A94E2F7817001C081E060
:10EE2000AE89BF898C93F401E05DF94EF88BEF87D2
:10EE30008A899B890C2C02C0959587950A94E2F7E4
:10EE400081708183F501E757FC4F408151816281D8
:10EE50007381C5018C559E4F0E94409E0E94B9D47B
:10EE600020E034E244E759E40E94E6D3AE89BF894A
:10EE700012966D937D938D939C931597EB85FC85EE
:10EE8000608171818D859E850E941D9EBC0180E000
:10EE900090E00E94B9D4AE89BF8916966D937D9398
:10EEA0008D939C931997F501E559FC4F4081518151
:10EEB00062817381C501805F9D4F0E94409E0E94C8
:10EEC000BBD4EE89FF8922813381448155810E9420
:10EED000BFD520E030E04AE754E40E94BFD50E944D
:10EEE00088D428EE33E040E050E00E9488D6290123
:10EEF0003A01FB81F23011F118F0F53008F443C00B
:10EF0000C301B20122E030E040E050E00E9488D628
:10EF1000AE89BF8950962D933D934D935C93539743
:10EF200088279927DC01821B930BA40BB50BEE8974
:10EF3000FF8984879587A687B78737C040E050E070
:10EF4000BA01C5018C5D9D4F0E94409E0E94B9D4BC
:10EF5000AE89BF8912962D913D914D915C91159787
:10EF60000E94BFD50E9488D4461A570A680A790AB7
:10EF7000EE89FF89408A518A628A738A14861586CF
:10EF80001686178612C0EE89FF89208B318B428B43
:10EF9000538B7094609450944094411C511C611C9C
:10EFA000711C4486558666867786D8011C96ED913D
:10EFB000FC911D972081C701AF81B8850C9002C0DC
:10EFC000880F991F0A94E2F7282B2083D801159601
:10EFD000ED91FC9116972081C701A985BA850C9007
:10EFE00002C0880F991F0A94E2F7282B2083D801CA
:10EFF0001E96ED91FC911F972081C701AC81BD81C8
:10F000000C9002C0880F991F0A94E2F7282B2083E6
:10F01000D8015396ED91FC9154972081C701AC81A2
:10F02000BD810C9002C0880F991F0A94E2F7282B2B
:10F030002083F801848D958D892B79F101A0F2A1AF
:10F04000E02D2081C701D1010C9002C0880F991FCB
:10F050000A94E2F7809582238083EE89FF8990816C
:10F06000D8015C96ED91FC915D97D1018C91208146
:10F07000992349F0A70102C0440F551F8A95E2F772
:10F08000242B20830AC0D70102C0AA0FBB1F8A9578
:10F09000E2F7CD01809582238083F80185899689E6
:10F0A000892B89F1028CF38DE02D2081C701A98184
:10F0B000BA810C9002C0880F991F0A94E2F78095DC
:10F0C00082238083EE89FF899081D8015596ED9146
:10F0D000FC915697A981BA818C912081992349F09E
:10F0E000A70102C0440F551F8A95E2F7242B208305
:10F0F0000AC0D70102C0AA0FBB1F8A95E2F7CD0153
:10F10000809582238083F601EE0FFF1FEE0FFF1F15
:10F11000E45EF94E1082118212821382EF85F88923
:10F1200012861386F601E95EF94E1082F401E05D65
:10F13000F94E81E04B81433008F480E0818FAE8945
:10F14000BF895D961D921D921D921C929097B1E011
:10F15000B28F138E148AEE89FF89158A168A178A50
:10F16000108EDF0111A212A213A214A215A216A2E0
:10F1700017A210A6FFEFCF1ADF0A49E2840E911CF6
:10F18000CD0189969F8B8E8B0D5D1F4FA981BA8112
:10F190009396BA83A983EF81F885B396F887EF83B6
:10F1A00049855A854D5D5F4F5A8749878C819D817E
:10F1B00083969D838C8393E2290E311CA4E0AA0ED2
:10F1C000B11CEB85FC853296FC87EB874D855E850F
:10F1D0004E5F5F4F5E874D8755E0C516D10409F03D
:10F1E0000CCE8989882321F01092121610921116E4
:10F1F00010921416109213161092161610921516DD
:10F2000067960FB6F894DEBF0FBECDBFDF91CF91EA
:10F210001F910F91FF90EF90DF90CF90BF90AF9034
:10F220009F908F907F906F905F904F903F902F9026
:10F23000089599E2899FF0011124E05DF94E628101
:10F240007381848195810895CF93DF931F92CDB709
:10F25000DEB749830E94BBD4498129E2429FF00175
:10F260001124E05DF94E22813381448155810E9451
:10F27000E6D30F90DF91CF9108954F925F926F92F6
:10F280007F928F929F92AF92BF92CF92DF92EF9236
:10F29000FF920F931F93CF93DF93142F20E030E062
:10F2A0004AE754E40E94BFD50E944ED429013A0196
:10F2B0004B01D82FC92F89E2189FF0011124E05D7E
:10F2C000F94E62817381848195810E944ED45901E7
:10F2D0006A017B018C019201A301B4018D2F9C2F47
:10F2E0000E94CED6E8EEAE2EF3E0BF2EC12CD12C7C
:10F2F000E12CF12C00E010E00E9454D7B901CA01C2
:10F30000DF91CF911F910F91FF90EF90DF90CF9001
:10F31000BF90AF909F908F907F906F905F904F9035
:10F32000089540E063E97AE18DEF96E10C94F4CE24
:10F330001F93CF93DF93C8E4D7E110E0612FCE0194
:10F340000E94879D2B961F5F1530C1F7DF91CF91EB
:10F350001F91089580914717811103C0809146172E
:10F36000089581E008956F927F929F92AF92BF922D
:10F37000CF92DF92EF92FF920F931F93CF93DF9381
:10F3800000D000D0CDB7DEB79FB6F89408E312E006
:10F39000612C712C40E050E0BA01C8010E94409EEF
:10F3A0006B017C01862D0E9419799B01AC01B30190
:10F3B00086E097E129833A834B835C830E94C64EA3
:10F3C0005C01C701B6010E94BBD429813A814B81FF
:10F3D0005C810E94BFD520E030E04AE754E40E94FF
:10F3E000E6D30E9488D4F50160837183828393837E
:10F3F000FFEF6F1A7F0A0C5F1F4F83E068167104DE
:10F4000049F602E010E0B80186E097E10E94C64E9E
:10F41000FC0110821182128213820F5F1F4F053090
:10F42000110589F700E010E0B8018AE197E10E9438
:10F43000C64EFC0110821182128213820F5F1F4F91
:10F440000530110589F79FBE0F900F900F900F9018
:10F45000DF91CF911F910F91FF90EF90DF90CF90B0
:10F46000BF90AF909F907F906F9008951092471734
:10F470001092461781E00E9494760E9498794FEF8F
:10F480005FEFBA0188E392E00E94409E6F3F7F4F9A
:10F490008F4F9F4F11F40C94253708958F929F92B0
:10F4A000AF92BF92DF92EF92FF920F931F93CF9391
:10F4B000DF93CDB7DEB764970FB6F894DEBF0FBE0B
:10F4C000CDBF24E1FC01DE01119601900D922A9539
:10F4D000E1F78BE3E82E86E1F82E00E010E0DD2472
:10F4E000D394F701D082B801809104179091051749
:10F4F0000E94C64EFC0180809180A280B380B8013A
:10F50000CE0101960E94C64EFC014081518162816C
:10F510007381480D591D6A1D7B1D40835183628391
:10F5200073830F5F1F4FF9E2EF0EF11C05301105D9
:10F53000C1F664E070E0CE0101960E94C64E8C01D7
:10F5400063E070E0CE0101960E94C64E4C0162E07D
:10F5500070E0CE0101960E94C64E5C0161E070E051
:10F56000CE0101960E94C64E7C0160E070E0CE01A3
:10F5700001960E94C64E9401A501B7010E942F7604
:10F5800064960FB6F894DEBF0FBECDBFDF91CF916A
:10F590001F910F91FF90EF90DF90BF90AF909F90E1
:10F5A0008F900895AF92BF92CF92DF92EF92FF9229
:10F5B0000F931F93CF93DF93CDB7DEB764970FB64A
:10F5C000F894DEBF0FBECDBF24E1FC01DE01119631
:10F5D00001900D922A95E1F781E080933B1680938C
:10F5E000641680938D168093B6168093DF1664E0C0
:10F5F00070E0CE0101960E94C64E8C0163E070E07F
:10F60000CE0101960E94C64E5C0162E070E0CE0120
:10F6100001960E94C64E6C0161E070E0CE01019639
:10F620000E94C64E7C0160E070E0CE0101960E940F
:10F63000C64E9501A601B7010E942F7664960FB6BB
:10F64000F894DEBF0FBECDBFDF91CF911F910F9118
:10F65000FF90EF90DF90CF90BF90AF9008955F92B2
:10F660006F927F928F929F92AF92BF92CF92DF92D2
:10F67000EF92FF920F931F93CF93DF93CDB7DEB737
:10F6800064970FB6F894DEBF0FBECDBF3C010E9459
:10F690008A4E5FB6F89480905E1590905F15A090AA
:10F6A0006015B0906115C0905A15D0905B15E09030
:10F6B0005C15F0905D15009156151091571520912D
:10F6C000581530915915409152155091531560912C
:10F6D000541570915515809165158F93809164151F
:10F6E0008F93809163158F93809162158F93CE01D4
:10F6F00001960E948B4E84E1FE013196D301019068
:10F700000D928A95E1F70F900F900F900F9000E007
:10F7100010E0B80180910417909105170E94C64E21
:10F72000FC01C080D180E280F380B801C3010E9457
:10F73000C64EFC0140815181628173814C195D0983
:10F740006E097F0940835183628373830F5F1F4F6C
:10F7500005301105F1F65FBEC30164960FB6F8944B
:10F76000DEBF0FBECDBFDF91CF911F910F91FF90F4
:10F77000EF90DF90CF90BF90AF909F908F907F9051
:10F780006F905F9008956F927F928F929F92AF9249
:10F79000BF92CF92DF92EF92FF920F931F93CF937E
:10F7A000DF93CDB7DEB765970FB6F894DEBF0FBE17
:10F7B000CDBF3C01CE0145967C018E010F5E1F4FEF
:10F7C0009E01235F3F4FAE01475F5F4FBE016B5FFE
:10F7D0007F4F44970E9410658D8981708D8B813099
:10F7E00029F426E0C22E27E1D22E04C09AE1C92EC8
:10F7F00097E1D92EFE0131967F0100E010E0B801BB
:10F80000C6010E94C64EF701408151816281738119
:10F81000FC0180819181A281B381481B590B6A0B45
:10F820007B0BF70141935193619371937F010F5FBC
:10F830001F4F0530110519F78D849E84AF84B88859
:10F84000C984DA84EB84FC840D811E812F81388584
:10F8500049815A816B817C818C898F938B898F93AD
:10F860008A898F9389898F93C3010E948B4E0F9051
:10F870000F900F900F90C30165960FB6F894DEBFFE
:10F880000FBECDBFDF91CF911F910F91FF90EF90F1
:10F89000DF90CF90BF90AF909F908F907F906F90B0
:10F8A00008958093301708954F925F926F927F92E0
:10F8B0008F929F92AF92BF92CF92DF92EF92FF9280
:10F8C0000F931F93CF93DF93CDB7DEB728970FB673
:10F8D000F894DEBF0FBECDBF6C019A01AB01FEE311
:10F8E000EF2EF5E1FF2E00E010E0B801C6012D83F8
:10F8F0003E834F8358870E94BF4EFC0180809180D9
:10F90000A280B380B80180910417909105170E94DE
:10F91000C64EFC0180819181A281B381880D991D21
:10F92000AA1DBB1DF70181939193A193B1937F0110
:10F930000F5F1F4F2D813E814F8158850530110586
:10F94000A1F6C0904615D0904715E0904815F0906C
:10F9500049158091921690919316A0919416B091AA
:10F960009516C816D906EA06FB0614F4D701C60197
:10F970008093461590934715A0934815B093491569
:10F9800062E575E104E815E1EEE34E2EE5E15E2E59
:10F99000712C612CC12CD12C7601F20181919191B5
:10F9A000A191B1912F01FB0181909190A190B19013
:10F9B000BF0188199909AA09BB09B7FF07C0B0950B
:10F9C000A095909581959F4FAF4FBF4FF8018193C0
:10F9D0009193A193B1938F01C816D906EA06FB064D
:10F9E0001CF4672C6C017D017394F5E07F12D5CF78
:10F9F00060929815C0929915D0929A15E0929B1535
:10FA0000F0929C15CD28CE28CF2839F160E472E41D
:10FA10008FE090E00E9488D629833A834B835C83F1
:10FA2000E090031700E023E037E1AE014F5F5F4F46
:10FA300060E070E0CB010E94976D8091B80D9091CD
:10FA4000B70D891B8F7090914517891720F081E0C1
:10FA50008093471702C01092471728960FB6F89464
:10FA6000DEBF0FBECDBFDF91CF911F910F91FF90F1
:10FA7000EF90DF90CF90BF90AF909F908F907F904E
:10FA80006F905F904F9008954F925F926F927F9228
:10FA90008F929F92AF92BF92CF92DF92EF92FF929E
:10FAA0000F931F93CF93DF93CDB7DEB728970FB691
:10FAB000F894DEBF0FBECDBF5C014D835E836F83C4
:10FAC00078871EE3E12E15E1F12E02E5C02E05E157
:10FAD000D02E00E010E0822E912CC401002E02C036
:10FAE000959587950A94E2F780FF0AC0F601408059
:10FAF000518062807380B801C5010E94BF4E10C062
:10FB0000B801C5010E94BF4EFC0140805180628057
:10FB10007380B80180910417909105170E94C64E1A
:10FB2000FC0180819181A281B381840D951DA61D68
:10FB3000B71DF70180839183A283B3830F5F1F4FAB
:10FB4000F4E0CF0ED11C84E0E80EF11C0530110565
:10FB500021F64091461550914715609148157091D6
:10FB600049158091921690919316A0919416B09198
:10FB70009516481759076A077B0714F4DB01CA0179
:10FB80008093461590934715A0934815B093491557
:10FB900064E875E1A2E56A2EA5E17A2EBEE38B2E1C
:10FBA000B5E19B2E10E0A12C20E030E0A901F4018A
:10FBB00081919191A191B1914F01F301C190D190A7
:10FBC000E190F1903F018C199D09AE09BF09B7FF83
:10FBD00007C0B095A095909581959F4FAF4FBF4FAF
:10FBE000FB0181939193A193B193BF01281739072A
:10FBF0004A075B071CF4A12E9C01AD011F5F153065
:10FC0000B1F6A09298152093991530939A154093C8
:10FC10009B1550939C15211531054105510569F13E
:10FC20006D817E818F8198850E9488D660E472E420
:10FC30008FE090E00E9488D629833A834B835C83CF
:10FC4000E090031700E023E037E1AE014F5F5F4F24
:10FC500060E070E0CB010E94976D8091B80D9091AB
:10FC6000B70D891B8F7090914517891720F081E09F
:10FC70008093471702C01092471728960FB6F89442
:10FC8000DEBF0FBECDBFDF91CF911F910F91FF90CF
:10FC9000EF90DF90CF90BF90AF909F908F907F902C
:10FCA0006F905F904F9008952F923F924F925F9286
:10FCB0006F927F928F929F92AF92BF92CF92DF927C
:10FCC000EF92FF920F931F93CF93DF93CDB7DEB7E1
:10FCD00066970FB6F894DEBF0FBECDBF3C014D87CF
:10FCE0005E876F87788B47015801DA8AC98AAEE34D
:10FCF0004A2EA5E15A2EB2E52B2EB5E13B2E00E0AF
:10FD000010E0422F50E05E834D838D819E81002E56
:10FD100002C0959587950A94E2F780FF0AC0F10129
:10FD2000C080D180E280F380B801C3010E94BF4E41
:10FD300010C0B801C3010E94BF4EFC01C080D18039
:10FD4000E280F380B80180910417909105170E941A
:10FD5000C64EFC0180819181A281B3818C0D9D1DD5
:10FD6000AE1DBF1DF20180839183A283B3830F5F19
:10FD70001F4FF4E02F0E311C24E0420E511C0530C1
:10FD8000110519F640914615509147156091481597
:10FD9000709149158091921690919316A0919416A6
:10FDA000B0919516481759076A077B0714F4DB01D1
:10FDB000CA018093461590934715A0934815B093B8
:10FDC000491510929815F4E86F2EF5E17F2E41E366
:10FDD00057E158874F8301EA15E182E595E19A875B
:10FDE0008987EEE3F5E1FC87EB871D82212C312C1E
:10FDF0002101EB85FC856191719181919191FC8745
:10FE0000EB87E985FA85C190D190E190F190FA876E
:10FE1000E9876C197D098E099F09F301608371835D
:10FE2000828393836B017C0197FF07C0CC24DD2480
:10FE30007601C61AD70AE80AF90AC114F0E8DF0603
:10FE4000E104F10464F4EF81F8852081318142817D
:10FE50005381CB01772766270E944CD224C00E9491
:10FE6000BBD46B8B7C8B8D8B9E8BEF81F8856081F7
:10FE70007181828193810E94BBD420E030E040E810
:10FE800057E30E94BFD59B01AC016B897C898D89AA
:10FE90009E890E94BFD520E030E040E857E40E94F0
:10FEA000BFD50E9488D4F8016083718382839383D5
:10FEB000F301C082D182E282F3822C143D044E040D
:10FEC0005F042CF4FD81F09398151601270124E0BE
:10FED000620E711C3D813F5F3D834F8158854C5FB1
:10FEE0005F4F58874F830C5F1F4F353009F081CF2C
:10FEF0002092991530929A1540929B1550929C151C
:10FF000023282428252809F459C020E030E0A9013D
:10FF1000C501B4010E94E2D3882309F44FC020E058
:10FF200030E040E857E4C501B4010E94BFD50E940B
:10FF300088D460939D1570939E1580939F15909320
:10FF4000A0152091B702222379F0E989FA89BF012F
:10FF5000882777FD8095982F3AE0660F771F881FD6
:10FF6000991F3A95D1F703C060E070E0CB01E090B3
:10FF70000317222319F00091B60201C000E02D857D
:10FF80003E854F85588929833A834B835C8323E0E0
:10FF900037E1AE014F5F5F4F0E94976D8091B80DC2
:10FFA0009091B70D891B8F7090914517891720F09C
:10FFB00081E08093471702C01092471766960FB6EC
:10FFC000F894DEBF0FBECDBFDF91CF911F910F918F
:10FFD000FF90EF90DF90CF90BF90AF909F908F9069
:10FFE0007F906F905F904F903F902F9008952F9249
:10FFF0003F924F925F926F927F928F929F92AF92B9
:020000021000EC
:10000000BF92CF92DF920F931F93CF93DF93CDB721
:10001000DEB768970FB6F894DEBF0FBECDBF782E5F
:10002000A62E1092B602CE0101962D8B3E8B4F8BE1
:10003000588F0E94C37BEAE38E2EE6E19E2E00E0FD
:1000400010E0B12C66246394588D4F893E892D8928
:10005000C801895E994E6C01C501002E02C09595BC
:1000600087950A94E2F780FD03C0F601108228C04C
:10007000B801CE0101962D8B3E8B4F8B588F0E947D
:10008000C64E2D893E894F89588D772039F022241C
:100090002A94322C422C7FE3572E05C0212C312C80
:1000A000412C60EC562EFC01208231824282538228
:1000B000F6016082023011F460922F17F401608221
:1000C0000F5F1F4FF9E28F0E911C0530110509F0EB
:1000D000BFCFBA01A901CE0101960E94547C81E0F4
:1000E0008093461768960FB6F894DEBF0FBECDBF5B
:1000F000DF91CF911F910F91DF90CF90BF90AF9084
:100100009F908F907F906F905F904F903F902F9037
:100110000895853098F49091121621E030E0082E71
:1001200001C0220F0A94EAF7662321F0922B9093E4
:100130001216089520952923209312160895809170
:1001400012160895853040F42BE0829FC0011124DF
:10015000885B984E0C948D9D08958093B602089507
:10016000817080930317813019F486E097E102C013
:100170008AE197E190930517809304170895809181
:10018000690290916A02892B99F0E0916B02F091DB
:100190006C02808190E000906D0202C09595879579
:1001A0000A94E2F7817021E090918216891301C0D0
:1001B00020E040E2249F90011124809162029091FE
:1001C0006302892BA1F0E0916402F09165028081C5
:1001D00090E00090660202C0959587950A94E2F738
:1001E000482F417081E090918216491301C080E050
:1001F00040E1849FC0011124822B932B2091460261
:1002000030914702232BA1F0E0914802F09149027E
:10021000208130E000904A0202C0359527950A946B
:10022000E2F7422F417021E030915916431301C08B
:1002300020E048E0249F90011124282B392B809145
:100240003F0290914002892BA1F0E0914102F09190
:100250004202808190E00090430202C0959587950C
:100260000A94E2F7482F417081E0909159164913A2
:1002700001C080E044E0849FC0011124822B932BB5
:100280002091230230912402232BA1F0E09125023A
:10029000F0912602208130E00090270202C03595BF
:1002A00027950A94E2F7422F417021E030913016F1
:1002B000431301C020E030E0220F331F282B392BDD
:1002C00080911C0290911D02892BA1F0E0911E02E9
:1002D000F0911F02808190E00090200202C095956D
:1002E00087950A94E2F7482F417081E0909130168B
:1002F000491301C080E0822B08959091B7029111BB
:1003000001C080E00C94E4653F924F925F926F923F
:100310007F928F929F92AF92BF92CF92DF92EF9295
:10032000FF920F931F93CF93DF9300D000D000D0A4
:10033000CDB7DEB780E00E9494760E949879109243
:100340002E1710922F170E94B37980E00E94B08080
:100350006FEF88E891E00E94009E803811F00E94C3
:100360003F3560E08EE691E00E94009E81708093B0
:10037000B7028093B60281E00E947D8191E3E92E6D
:1003800097E1F92E10E0812F0E9419799B01AC01B1
:1003900060E070E080E89FE30E94E6D320E030E078
:1003A00040E857E40E94BFD50E9488D4F7016193CA
:1003B0007193819391937F011F5F153021F768EE50
:1003C00073E082E791E00E941D9EA0E0B0E0809380
:1003D000F7159093F815A093F915B093FA1568EEF8
:1003E00073E084E791E00E941D9EA0E0B0E080935E
:1003F000FB159093FC15A093FD15B093FE1566E9CF
:1004000070E086E791E00E941D9EA0E0B0E080933E
:10041000FF1590930016A0930116B093021660EAA0
:100420007FE088E791E00E941D9EA0E0B0E080930D
:10043000031690930416A0930516B093061660EA6F
:100440007FE08AE791E00E941D9EA0E0B0E08093EB
:10045000071690930816A0930916B0930A1687EF13
:1004600095E19E838D83BDEBAB2EB5E1BB2E0CE6F3
:1004700015E1312CCC24CA94DC2C76018D809E8031
:10048000F4014080518062807380832D0E9419792D
:100490009B01AC0160EF7FEF8FE799E40E94E6D308
:1004A0000E948DD4641575058605970598F4832DF3
:1004B0000E9419799B01AC0160EF7FEF8FE799E40F
:1004C0000E94E6D30E948DD4ED81FE81608371830A
:1004D000828393838D819E8104969E838D83F40114
:1004E00060817181828193810E94B9D42B013C018A
:1004F000832D0E9419799B01AC01C301B2010E94B6
:10050000BFD50E948DD49B01AC01F501619371931D
:10051000819391935F01C701B6010E9466D6F801ED
:1005200021933193419351938F013394F5E03F121E
:10053000A5CF60ED77E080E791E00E941D9EA0E0EE
:10054000B0E0813127E29207A105B10520F080E1FA
:1005500097E2A0E0B0E08093F3159093F415A09398
:10056000F515B093F61560EA7FE086E891E00E9409
:100570001D9EA0E0B0E08131E7E29E07A105B10534
:1005800020F080E197E2A0E0B0E08093EF15909337
:10059000F015A093F115B093F21560E070E080EED5
:1005A00091E00E941D9E9093AC0D8093AB0D60E096
:1005B00070E082EE91E00E941D9E9093AE0D8093BC
:1005C000AD0D6AE070E08CE791E00E941D9EBC01D9
:1005D00080E090E00E94B9D420E030E040E857E4A9
:1005E0000E94BFD50E9488D46093D7157093D81508
:1005F0008093D9159093DA156AE070E08EE791E068
:100600000E941D9EBC0180E090E00E94B9D420E0D1
:1006100030E040E857E40E94BFD50E9488D4609340
:10062000DB157093DC158093DD159093DE156AE081
:1006300070E080E891E00E941D9EBC0180E090E0A7
:100640000E94B9D420E030E040E857E40E94BFD5D2
:100650000E9488D46093DF157093E0158093E115B4
:100660009093E2156EE170E082E891E00E941D9E99
:10067000BC0180E090E00E94B9D420E030E040E886
:1006800057E40E94BFD50E9488D46093E31570930D
:10069000E4158093E5159093E6156EE170E084E82B
:1006A00091E00E941D9EBC0180E090E00E94B9D4C0
:1006B00020E030E040E857E40E94BFD50E9488D493
:1006C0006093E7157093E8158093E9159093EA1508
:1006D000E7EDF5E18091DF159091E015A091E1152E
:1006E000B091E2154191519161917191481759076B
:1006F0006A077B0714F4DB01CA0125E1EB3EF20730
:1007000089F78093EB159093EC15A093ED15B093BA
:10071000EE1542E553E060E070E088ED91E00E9464
:10072000409E0E94B9D420E030E543EC57E40E949B
:10073000E6D320E030E040E857E40E94BFD50E94B5
:1007400088D46B017C0144E853E060E070E08CEDFC
:1007500091E00E94409E0E94B9D420E030E543EC35
:1007600057E40E94E6D320E030E040E857E40E94DE
:10077000BFD50E9488D49B01AC018EE195E0A0E03A
:10078000B0E08093661590936715A0936815B093B9
:10079000691580E090E0A2E0B0E08093D3159093DB
:1007A000D415A093D515B093D61561E084EE91E0F1
:1007B00029833A834B835C830E94009E29813A817E
:1007C0004B815C81882329F184E090E09093D215DD
:1007D0008093D1150E94455029813A814B815C81DB
:1007E00081110AC08091D1159091D215880F991F5F
:1007F0009093D2158093D1158091D1159091D215F7
:1008000009975CF088E090E09093D2158093D11521
:1008100004C01092D2151092D11581E08093A90DD9
:100820008093AA0D8091B1169091B216A091B31643
:10083000B091B4168093A10D9093A20DA093A30D37
:10084000B093A40D8091DA169091DB16A091DC167E
:10085000B091DD168093A50D9093A60DA093A70DE2
:10086000B093A80D8FE08093451700913017C70112
:10087000B6010E94536D26960FB6F894DEBF0FBEE8
:10088000CDBFDF91CF911F910F91FF90EF90DF903F
:10089000CF90BF90AF909F908F907F906F905F9020
:1008A0004F903F900C9422640E946E6510924717FF
:1008B0001092461780E00E9494768091B702809350
:1008C000B60281E00C947D810E943B53811110920D
:1008D000471780914617882331F11092461780E020
:1008E00090E0FC01E95EF94E208130914617232B00
:1008F0002093461701968330910599F7809146170A
:10090000811111C00E946E6580912F17882339F0E4
:1009100080912E178F5F80932E1710922F17809142
:10092000B7028093B60208950C94EC6280912E1762
:100930000895CF93DF9300D000D000D0CDB7DEB7BD
:1009400040E063E97AE18FE797E10E94F4CE45E069
:1009500063EA7AE1CE0101960E94F4CE4DE953E0BC
:10096000BE016F5F7F4F88E497E10E94139D46E0D0
:1009700065E97AE1CE0101960E94F4CE4DE953E09B
:10098000BE016F5F7F4F83E597E10E94139D43E0B7
:1009900065E97AE1CE0101960E94F4CE4DE953E07B
:1009A000BE016F5F7F4F8EE597E10E94139D44E08B
:1009B00069EA7AE1CE0101960E94F4CE4DE953E056
:1009C000BE016F5F7F4F89E697E10E94139D47E06C
:1009D00069E97AE1CE0101960E94F4CE4DE953E037
:1009E000BE016F5F7F4F84E797E10E94139D8AE10C
:1009F00097E10E948A4E86E097E10E948A4E2696F1
:100A00000FB6F894DEBF0FBECDBFDF91CF91089532
:100A100094EA9093BC009091BC0097FFFCCF90911A
:100A2000B900987F983061F58093BB0084E880938B
:100A3000BC008091BC0087FFFCCF8091B900887F0B
:100A4000883101F5FB0150E024E8CF01861B970BAC
:100A50008417950784F481918093BB002093BC0098
:100A60008091BC0087FFFCCF8091B900887F8832DD
:100A700061F383E0089584E98093BC0080E00895E9
:100A800081E0089582E008951092B90080E2809399
:100A9000B800089580918C17089510928C1781E00A
:100AA00080938517089581E040918A1750918B17A4
:100AB0002091881730918917421753070CF080E076
:100AC000089580918A1790918B1720918817309103
:100AD0008917821793077CF4E0918617F0918717A6
:100AE0009C012F5F3F4F30938B1720938A17E80F9D
:100AF000F91F8491089580E00895809185170895E5
:100B0000CF93C82F81E080938C1710928B1710928F
:100B10008A1710928517C13081F060F0C23001F55C
:100B20008093851783E591E19093871780938617CB
:100B3000C3E01AC02EEB32E306C00E94FF358823C3
:100B400039F028E83AE230938717209386170CC0D3
:100B500082E592E29093871780938617C2E004C0E3
:100B600010928C1780E00EC0EC2FF0E0EE0FFF1F0C
:100B7000E35EFC4C8591949190938917809388173C
:100B800080918C17CF91089510928C1781E08093FB
:100B90008517089540E063E97AE18DE897E10C94C8
:100BA000F4CECF93DF9300D000D000D0CDB7DEB726
:100BB000109295171092941740E251EA67E070E0A6
:100BC000FC0140A351A362A373A3E4E0F1E08081A0
:100BD00087788083E5E0F1E080818778808342E058
:100BE0006DE97AE1CE0101960E94F4CE60E0CE017B
:100BF00001960E9423CF26960FB6F894DEBF0FBE53
:100C0000CDBFDF91CF9108957F928F929F92AF9247
:100C1000BF92CF92DF92EF92FF920F931F93CF93E9
:100C2000DF93CDB7DEB72F970FB6F894DEBF0FBEB8
:100C3000CDBF8C01FC0181818111A4C0F090030122
:100C4000FF2DF8778F2E92B2292D2470922E80914D
:100C500094178227909195179F27892BF801329638
:100C60006F01882351F080E291EAA7E0B0E0F8013B
:100C700080A391A3A2A3B3A313C0F8018281882308
:100C800031F0C6010E94CED0882309F47BC040EA2F
:100C900056E861E070E0F80140A351A362A373A39A
:100CA000C6010E94FDD098012F5E3F4F5901F3FC11
:100CB0000FC080919317811119C040E856E968E987
:100CC00070E0C9010E94AAD081E0809393170EC002
:100CD000CE0101960E94A6D08FE0FE013196D5018B
:100CE00001900D928A95E1F710929317C5010E9429
:100CF000CED0882389F0F801108281E08183CE0173
:100D000001960E94A6D08FE0FE013196D501019098
:100D10000D928A95E1F736C091100CC082E0F8017F
:100D2000808381E0818340A151A162A173A1C601AA
:100D30000E94AAD083E0E82EF12CA82CB12C7724B5
:100D40007394C5010E2C02C0959587950A94E2F71D
:100D500080FD0DC0F8018181811109C0E08271829E
:100D600040A151A162A173A1C6010E94AAD0FFEFC8
:100D7000EF1AFF0A27E0E216F10419F79092941790
:100D8000809295172F960FB6F894DEBF0FBECDBF99
:100D9000DF91CF911F910F91FF90EF90DF90CF9057
:100DA000BF90AF909F908F907F900895FC01F89432
:100DB0008181208111827894882321F030E0FB0129
:100DC000318320830895FC0140A351A362A373A340
:100DD000089540E063E97AE186E997E10C94F4CE66
:100DE0002F923F924F925F926F927F928F929F923B
:100DF000AF92CF92DF92EF92FF920F931F93CF9318
:100E0000DF93EC01D62E1A012901602F47010E94C1
:100E1000B48983EA93E09E838D83DF823E0188E07C
:100E2000680E711C8AE0E80EF11CAE014B5F5F4F4B
:100E3000AD2CCC24C39400E910ED23E030E0BE01DA
:100E4000C3010E94DB9FB101CE018E579F4F0E94CC
:100E50000BCFFE01E857FF4FD082A401465E5F4FE3
:100E60009201B301CE0187579F4F0E94B79CC35692
:100E7000DF4F99828882DF91CF911F910F91FF9070
:100E8000EF90DF90CF90AF909F908F907F906F907A
:100E90005F904F903F902F900895CF93DF93EC0198
:100EA00008960E94C4A2CE0187579F4FDF91CF9131
:100EB0000C94CD9C87579F4F61110C947A9C0C9495
:100EC000869C882321F080919000806803C08091E7
:100ED00090008F73809390000895882321F0809173
:100EE0009000886003C080919000837F8093900081
:100EF00008950F931F93CF93DF9300D000D000D0BD
:100F0000CDB7DEB7162F0FB7F894FC01828181119F
:100F100012C08FEF860F8E3F28F080E00E946D8711
:100F200045E013C070E070939D0060939C00809139
:100F30009000886021C0813009F58FEF860F8E3FC9
:100F400098F080E00E94618743E061EA7AE1CE0197
:100F500001960E94F4CE61E01F3F09F060E0CE01EF
:100F600001960E9443CF0AC070E07093990060938D
:100F70009800809190008068809390000FBF269623
:100F80000FB6F894DEBF0FBECDBFDF91CF911F919A
:100F90000F91089540E063E97AE18CE997E10C94C0
:100FA000F4CE0F931F93CF93DF93EC018C010E5778
:100FB0001F4F60E0C8010E9443CF61E0C8010E945A
:100FC00023CFCE0108960E94F19ECE010E94938904
:100FD000CE0187579F4FDF91CF911F910F910C94B6
:100FE0008A9C0F931F93CF93DF9300D000D000D043
:100FF000CDB7DEB7062F142F94E09D838E8342E099
:10100000BE016B5F7F4F84EC0E94088587EC90E007
:101010000197F1F700C0000083E08B830C8342E06E
:10102000BE016D5F7F4F84EC0E94088587EC90E0E5
:101030000197F1F700C0000082E089831A8342E043
:10104000BE016F5F7F4F84EC0E94088526960FB625
:10105000F894DEBF0FBECDBFDF91CF911F910F91EE
:1010600008958F929F92AF92BF92CF92DF92EF92AC
:10107000FF9261E080E491E00E94009EB82E4FEF65
:101080005FEFBA0184E491E00E94409E6B017C0115
:101090008B2D90E089309105E0F5FC01E555FF4F7F
:1010A0000C94A7D621E04FEF6FEF06C021E04FEF81
:1010B00024C021E040E060E08FEF21C021E040E06B
:1010C0006FEF1CC021E040E062E308C021E046E48D
:1010D00060E086E414C021E048EC60E088EC0FC0DA
:1010E0008D2C9E2CAF2CBB24B7018827992721E09B
:1010F000482D8F2D04C021E040E060E080E0FF90AB
:10110000EF90DF90CF90BF90AF909F908F900C9416
:10111000F187FF90EF90DF90CF90BF90AF909F90BE
:101120008F900895CF93DF9300D000D000D0CDB73B
:10113000DEB70E9444851D8281E08E8342E0BE01BD
:101140006B5F7F4F84EC0E94088587EC90E00197ED
:10115000F1F700C0000081E08B8384E18C8342E0E2
:10116000BE016D5F7F4F84EC0E94088587EC90E0A4
:101170000197F1F700C0000088E089838AEA8A833A
:1011800042E0BE016F5F7F4F84EC0E94088587ECD0
:1011900090E00197F1F700C000000E943188269688
:1011A0000FB6F894DEBF0FBECDBFDF91CF9108958B
:1011B0001F93CF93DF93CDB7DEB728970FB6F89480
:1011C000DEBF0FBECDBF182F81E08F831123E1F169
:1011D00084E3888742E0BE01695F7F4F84EC0E9410
:1011E000088587EC90E00197F1F700C0000088E0E7
:1011F0008D838FE38E8342E0BE016B5F7F4F84EC73
:101200000E94088587EC90E00197F1F700C000008C
:1012100086E08B8380E88C8342E0BE016D5F7F4F68
:1012200084EC0E94088587EC90E00197F1F700C0FC
:10123000000087E089831A8342E0BE016F5F7F4F21
:1012400084EC0E94088544C084E1888742E0BE01A6
:10125000695F7F4F84EC0E94088587EC90E00197DE
:10126000F1F700C0000088E08D838AE28E8342E0BF
:10127000BE016B5F7F4F84EC0E94088587EC90E095
:101280000197F1F700C000001C821B8286E08B836F
:1012900042E0BE016D5F7F4F84EC0E94088587ECC1
:1012A00090E00197F1F700C000001A82198287E0F0
:1012B000898342E0BE016F5F7F4F84EC0E94088506
:1012C00087EC90E00197F1F700C000000E943188A0
:1012D00028960FB6F894DEBF0FBECDBFDF91CF9139
:1012E0001F91089521E040E060E08FEF0E94F187B8
:1012F0008CE00C94D8881F93CF93DF93C82FD62F00
:10130000142F0E94F83421E0412F6D2F8C2FDF9194
:10131000CF911F910C94F18740E063E97AE182EA72
:1013200097E10C94F4CEFC011382128208950F937E
:101330001F93CF93DF9300D0CDB7DEB78C01AE0102
:101340004F5F5F4FFC01648187E199E00E94878ACB
:1013500029813A81F801338322830F900F90DF9126
:10136000CF911F910F91089529EA33E0FC01318359
:1013700020836483089540E063E97AE188EA97E195
:101380000C94F4CEAF92BF92CF92DF92EF92FF9285
:101390000F931F93CF93DF93EC017B016A015901F7
:1013A000B8010E940BCFB601CE0106960E940BCF6A
:1013B000B701CE010C960E940BCFB501CE0142962B
:1013C000DF91CF911F910F91FF90EF90DF90CF9021
:1013D000BF90AF900C940BCFAF92BF92CF92DF92A1
:1013E000EF92FF920F931F93CF93DF93EC018C0149
:1013F0000A5F1F4F60E0C8010E9443CF1A8E1B8E08
:1014000088E78C8FEBA0FCA0FCA6EBA6B0E1CB2E6E
:10141000D12C5E018CE0A80EB11C6E2D6170C5014F
:101420000E9443CFF694E79461E0C8010E9443CF45
:1014300060E0C8010E9443CF81E0C81AD108C114FE
:10144000D10459F7F0E1EF2EF12C629660E0C5016E
:101450000E9443CF61E0C8010E9443CFCE010E94A9
:1014600036CF60E0C8010E9443CF81E0E81AF1085E
:10147000E114F10459F760E0C801DF91CF911F91A9
:101480000F91FF90EF90DF90CF90BF90AF900C94B2
:1014900043CF0F931F93CF93DF93EC0161E00C9642
:1014A0000E9423CF8E010A5F1F4F61E0C8010E9496
:1014B00023CF60E0CE0142960E9423CF61E0CE01AF
:1014C0000E9423CF80E396E49CA38BA38CE396E455
:1014D0009EA38DA380E09EE498A78FA318A21F8EE1
:1014E0001AA219A21E8E1D8E60E0CE010E9443CF6B
:1014F00060E0C8010E9443CF1AA619A6198E188E63
:10150000CE01DF91CF911F910F910C94EC89FC01DA
:10151000611103C0878D90A102C081A192A1DA015F
:101520008D939C93808D918D08954F925F926F92D1
:101530007F928F929F92AF92BF92CF92DF92EF9263
:10154000FF920F931F93CF93DF93EC017C0186E012
:10155000E80EF11C60E0C7010E9443CF5E0182E10A
:10156000A80EB11CC5010E9436CF8111B6C08A8D6C
:10157000813049F028F0823049F44FA058A408C0C7
:101580004BA05CA005C04DA05EA002C0412C512C18
:10159000620130E1632E712C00E010E04E018CE01E
:1015A000880E911C6C2D6170C4010E9443CFD694AB
:1015B000C79461E0C7010E9443CF000F111FC5010E
:1015C0000E9436CF8111016060E0C7010E9443CFC5
:1015D00081E0681A71086114710421F780E1C82E56
:1015E000D12C60E0C4010E9443CF61E0C7010E949A
:1015F00043CFC5010E9436CF60E0C7010E9443CFB0
:1016000081E0C81AD108C114D10459F760E0C701BC
:101610000E9443CF8B8D813071F180F0823009F0D0
:1016200040C040E951E062E0C801969587959695E3
:1016300087950E94ABCF9E8F8D8F33C00F3F8FE772
:10164000180719F483E090E013C040E951E061E02D
:10165000C8010E94ABCF2D8D3E8D280F391F213937
:1016600081E038071CF438A32F8F19C084E090E084
:10167000998F888F16C00F3F8FE7180719F340E93D
:1016800051E061E0C8010E94ABCF2D8D3E8D280F47
:10169000391F213981E038074CF73AA329A3198E65
:1016A000188E8B8D90E09AA789A78A8D8B8F4BA679
:1016B0005CA6813039F018F0823069F010C081E00A
:1016C0008A8F0EC08C8D8F5F8C8F883720F01C8E98
:1016D00082E08A8F04C01A8E02C080E001C081E0DF
:1016E000DF91CF911F910F91FF90EF90DF90CF90FE
:1016F000BF90AF909F908F907F906F905F904F9032
:10170000089540E063E97AE18EEA97E10C94F4CE23
:101710004F925F926F927F92AF92BF92CF92DF9281
:10172000EF92FF920F931F93CF93DF9300D0CDB72B
:10173000DEB75C018B01009709F447C06230710588
:1017400008F443C0DC0116964D905D906D907C903E
:101750001997000F111F73016201C00ED11EE11C09
:10176000F11CD501ED91FC910190F081E02D22E07A
:1017700030E0AE014F5F5F4FC701B6010995882386
:1017800021F109811A8101151105E9F0C80140967E
:101790000897D8F0083FBFEF1B0710F000E010E0FB
:1017A0001A821982D501ED91FC910480F581E02D1A
:1017B00022E030E0AE014F5F5F4FC701B6010995EF
:1017C0000115110531F681E001C080E00F900F9006
:1017D000DF91CF911F910F91FF90EF90DF90CF900D
:1017E000BF90AF907F906F905F904F9008952F9231
:1017F0003F924F925F926F927F928F929F92AF92A1
:10180000BF92CF92DF92EF92FF920F931F93CF93ED
:10181000DF93CDB7DEB72C970FB6F894DEBF0FBEBF
:10182000CDBF6C011B015A01009709F45AC0DC01BD
:10183000ED91FC91808191819C878B87A481B581FA
:10184000BC83AB83D60116968D919D910D90BC9172
:10185000A02D8D839E83AF83B887F601E28CF38C35
:1018600082859385A485B585B695A7959795879527
:101870009A878987138E128E812C912C00E010E0BC
:101880000AC089819A81892B99F18FEFE81AF80AA9
:101890009FEF891A990AA985BA85A815B90509F48F
:1018A00050C0F2E0EF16F104F8F089859A85E81649
:1018B000F906D0F4C701880F991F4D805E806F80B4
:1018C0007884480E591E611C711C22E030E0AE0184
:1018D0004F5F5F4FC301B201EB85FC850995811114
:1018E000D0CF80E090E04AC032E0E32EF12CE2CF8E
:1018F000A114B10431F4D6015B96FC92EE925A9792
:1019000022C00115110529F4EFEFFFEFFA83E983F7
:1019100002C01A83098322E030E0AE014F5F5F4FBF
:10192000C301B201EB81FC810995811105C0B801A9
:10193000C6010E94888BD5CFF1E0AF1AB1088701AC
:10194000A4CFAB28A1F7B2E02B163104B0F01A8374
:101950000983220C331C6D817E818F819885620DF5
:10196000731D811D911D22E030E0AE014F5F5F4F7E
:10197000EB81FC8109958823D1F2C8012C960FB622
:10198000F894DEBF0FBECDBFDF91CF911F910F91B5
:10199000FF90EF90DF90CF90BF90AF909F908F908F
:1019A0007F906F905F904F903F902F90089580E1CF
:1019B00090E008950F931F93FC01009799F0623017
:1019C000710580F09B0122503109A089B1890E94E4
:1019D000ADD60289138924893589600F711F821F52
:1019E000931F03C060E070E0CB011F910F91089539
:1019F000FC01819191E0219180FB879587F9820F0D
:101A00009F5F9B30C1F70895CF92DF92EF92FF92D4
:101A10000F931F93CF93DF93CDB7DEB761970FB6C8
:101A2000F894DEBF0FBECDBF6C017901D9010D91D5
:101A30001C91119712968D919C91139780961396F5
:101A40009C938E931297F6018081853E11F081114F
:101A500004C0D70114961C924BC0F60183858F30C9
:101A600009F048C0D90114968C91882319F0958506
:101A7000891789F08BE2F80111928A95E9F7D6016E
:101A80001D968C91F7018483D80197964D935D93B1
:101A90006D937C939A97F60180818F7390E0019704
:101AA0004DE0489F9001499F300D1124E4EDF2E094
:101AB000DE01119601900D924A95E1F7FE013196F3
:101AC000020F131FAE01425F5F4F2E1B3F0BC90178
:101AD0008E0F9F1F4F9760F48191B601680F711DA3
:101AE000DB018C91D8018D938D01E417F50779F70F
:101AF00081E08AC0F8018081882309F456C0C601BC
:101B00004E875F87688B798B0E94F88CD70114967B
:101B10009C914E855F8568897989981346C02AC053
:101B2000FA019083F601248523FD4FC08F5F119643
:101B30004F5F5F4F883019F09C91903289F7D80140
:101B40009C91953011F495EE9C93F601908590321E
:101B500069F0F801E80FF11D9EE29083F6013896D6
:101B600034E0380F8F5F90819032C1F5F801E80FB3
:101B7000F11D1082F6018385D80190968C93909781
:101B8000828D938D92969C938E939197848D958D53
:101B9000A68DB78DF80183A394A3A5A3B6A381E076
:101BA000D70115968C9380E02FC08BE2F80111923B
:101BB0008A95E9F7D80197964D935D936D937C9341
:101BC0009A97D601A80180E0B7CF2C9121542A31F1
:101BD00008F0ACCF905EFA019083A8CFA801480F1F
:101BE000511DDA019C93D6011C962C9124FF07C04D
:101BF000208121542A3118F4905EDA019C938F5F82
:101C000031968313B0CFB2CF61960FB6F894DEBF92
